:08000000446B04000200000043
:04004800EE56000070
:04005400F85400005C
:040094009C58000074
:0400A000D655000031
:0400E400905B00002D
:0400F400706900002F
:100400003220EF00C3202000008041001040BA00DD
:100410000160EF00000006005365000072690000F3
:10042000616C0000204200006F6F0000742000002B
:100430004C6F000061640000203F000000000000DD
:100440003220EF00C3222000008041001040BA009B
:100450000160EF000000060020200000486F00004F
:100460006C6400002042000075740000746F00008E
:100470006E200000696E00002020000000000000D7
:100480003220EF00C3242000008041001040BA0059
:100490000160EF0000000600666F0000722000009F
:1004A000342000007365000063200000746F0000BA
:1004B000205300007461000072740000000000000E
:1004C0003220EF00C3262000008041001040BA0017
:1004D0000160EF0000000600202000002042000024
:1004E0006F6F0000742000006C6F000061640000FA
:1004F00065720000202000002020000000000000A5
:100500003220EF00C3282000008041001040BA00D4
:100510000160EF0000000600202000002020000005
:1005200025660000207300006563000020200000A5
:100530002020000020200000200000003220EF00DA
:10054000A32A2000008041001040BA000160EF00A3
:1005500000000600204200006F6F0000746C000075
:100560006F6100006420000053740000617200009D
:100570007465000064200000000000003220EF00DD
:10058000A32C2000008041001040BA000160EF0061
:100590000000060020200000202000002025000090
:1005A000730000003220EF00E32D200000804100A6
:1005B0001040BA000160EF0000000600303100007A
:1005C0002D4A0000756E00002D300000390000003B
:1005D0003220EF00432F2000008041001040BA007D
:1005E0000160EF0000000600204900006E69000075
:1005F00074690000616C00007A650000204500000D
:1006000045500000726F00006D20000000000000E7
:100610003220EF0043312000008041001040BA003A
:100620000160EF000000060020450000455000007A
:10063000726F00006D200000496E000069740000B8
:10064000696100006C7A0000656400002000000011
:100650003220EF0043332000008041001040BA00F8
:100660000160EF0000000600204C00006F610000F8
:10067000646900006E6700002044000065660000A9
:10068000617500006C740000732000000000000021
:100690003220EF0043352000008041001040BA00B6
:1006A0000160EF0000000600202000002020000074
:1006B000496E000069740000204D0000757800004C
:1006C00020200000200000003220EF00033720002F
:1006D000008041001040BA000160EF0000000600F9
:1006E0002020000020200000205200006573000040
:1006F00065740000204D0000757800002025000082
:1007000075200000000000003220EF0003392000B7
:10071000008041001040BA000160EF0000000600B8
:100720002020000020200000496E000069740000B5
:100730002056000069640000656F00002020000062
:1007400020200000000000003220EF00033B2000CA
:10075000008041001040BA000160EF000000060078
:1007600020200000496E0000697400002053000042
:10077000756200005379000073740000656D00001D
:1007800020200000000000003220EF00033D200088
:10079000008041001040BA000160EF000000060038
:1007A00020460000696E0000646900006E6700006A
:1007B00020430000616D000065720000617300005D
:1007C000000000003220EF00E33E200000804100E6
:1007D0001040BA000160EF00000006002020000079
:1007E0002020000020200000202000002020000009
:1007F00020200000202000002020000020200000F9
:10080000200000003220EF00E34020000080410083
:100810001040BA000160EF000000060043680000CD
:10082000656300006B730000756D000020520000CE
:10083000656100006420000025320000782C000073
:1008400020430000616C0000637500006C610000D3
:10085000746500006420000025320000780A000062
:100860000D0000003220EF00E34320000080410033
:100870001040BA000160EF000000060020200000D8
:10088000204300006F6E00006669000067200000D2
:100890005361000076650000642000002020000005
:1008A000000000003220EF00E345200000804100FE
:1008B0001040BA000160EF0000000600436F000026
:1008C0006E6600006967000020530000617600003A
:1008D000656400000A0D0000000000003220EF00F7
:1008E000A3472000008041001040BA000160EF00E3
:1008F00000000600537400006F72000065200000C5
:1009000046610000637400006F72000079200000EF
:1009100044650000666100007574000073200000EB
:1009200046610000696C0000656400000A0D00006B
:10093000000000003220EF00634A200000804100E8
:100940001040BA000160EF00000006005265000090
:10095000616400002045000045500000726F0000F7
:100960006D20000046610000696C000065640000B5
:100970000A0D0000000000003220EF00834C200030
:10098000008041001040BA000160EF000000060046
:10099000537400006F720000652000004465000081
:1009A000666100007574000073200000466100005D
:1009B000696C0000656400000A0D00000000000082
:1009C0003220EF0063022000830150000500310057
:1009D000C34F2000008041001040BA000160EF00CA
:1009E00000000600C04F200083814100808141004B
:1009F0001380BA0000000600446F4C004C6F580092
:100A0000616420005072630065736800657465005E
:100A10002025630032786B00202573003278750042
:100A200020256D004C583D00202525004C583200F3
:100A3000202558004C580A0020250D004C58000075
:100A4000202500003220EF00E30220008301500047
:100A500005003100E3532000008041001040BA003F
:100A60000160EF0000000600E05320008381410098
:100A7000808141001380BA0000000600446F4300EB
:100A80004C6F610061646D00507220006573250039
:100A9000657432003A2078004320200025644C0021
:100AA0002C20690050207600256465002C28200049
:100AB0006B3D4300254C610058296D002042200009
:100AC00061642500202D32002050640072650A0008
:100AD00073650D00742000003220EF008357200062
:100AE000008041001040BA000160EF0000000600E5
:100AF000446F00004C6F0000616400005072000001
:100B000065730000657400003A2000004320000077
:100B100063680000656300006B730000756D000082
:100B20003D25000032580000202100003D2000003B
:100B300025320000580A00000D0000003220EF00AE
:100B4000030220008301500005003100A35B200058
:100B5000008041001040BA000160EF000000060074
:100B6000A05B200083814100808141001380BA0096
:100B7000000006004C6F650063206E002532740093
:100B8000782C2000205043006F72610074206D00AB
:100B9000256465002C507200726561007365250044
:100BA00074203200256464002C200A0043750D0077
:100BB000727200003220EF00030220008301500017
:100BC00005003100635F2000008041001040BA0042
:100BD0000160EF0000000600605F2000838141009B
:100BE000808141001380BA0000000600536120009C
:100BF0007665630020256800327865002025630053
:100C000032786B00202573004C58750020256D004C
:100C10004C583D00202525004C5832002025580016
:100C20004C580A0020250D004C5800003220EF00DF
:100C300023622000008041001040BA000160EF00F4
:100C4000000006000A0D00005361000076650000F8
:100C50002044000065660000617500006C740000AF
:100C6000204C000053470000205000007265000037
:100C7000736500007420000025320000642000002D
:100C800061740000202500004C58000000000000A6
:100C90003220EF0043652000008041001040BA0080
:100CA0000160EF0000000600536F00006E79000045
:100CB00020450000564900002D440000333000005C
:100CC0002020000020200000202000002000000044
:100CD0003220EF0043672000008041001040BA003E
:100CE0000160EF0000000600536F00006E79000005
:100CF00020450000564900002D440000333000001C
:100D00002F440000333100002020000020000000AC
:100D10003220EF0043692000008041001040BA00FB
:100D20000160EF00000006005661000064640000EE
:100D3000696F000020410000646400002D61000024
:100D40002D430000616D0000202000002000000005
:100D50003220EF00436B2000008041001040BA00B9
:100D60000160EF0000000600536F00006E79000084
:100D700020450000564900002D440000313000009D
:100D80003020000020200000202000002000000073
:100D90003220EF00436D2000008041001040BA0077
:100DA0000160EF00000006005641000044440000CE
:100DB000494F000020480000442D00003138000059
:100DC0002020000020200000202000002000000043
:100DD0003220EF00436F2000008041001040BA0035
:100DE0000160EF0000000600536F00006E79000004
:100DF00020450000564900002D4400003730000017
:100E00002020000020200000202000002000000002
:100E10003220EF0043712000008041001040BA00F2
:100E20000160EF0000000600536F00006E790000C3
:100E300020420000524300002D33000030300000FB
:100E400020200000202000002020000020000000C2
:100E50003220EF0043732000008041001040BA00B0
:100E60000160EF0000000600536F00006E79000083
:100E700020420000524300002D480000373000009F
:100E80003020000020200000202000002000000072
:100E90003220EF0043752000008041001040BA006E
:100EA0000160EF0000000600536F00006E79000043
:100EB00020420000524300002D5A0000373000004D
:100EC0003020000020200000202000002000000032
:100ED0003220EF0043772000008041001040BA002C
:100EE0000160EF0000000600536F00006E79000003
:100EF00020420000524300002D5A0000333300000E
:100F000030200000202000002020000020000000F1
:100F10003220EF0043792000008041001040BA00E9
:100F20000160EF0000000600536F00006E790000C2
:100F300020450000564900002D48000044310000C3
:100F400020200000202000002020000020000000C1
:100F50003220EF00437B2000008041001040BA00A7
:100F60000160EF0000000600506100006E610000AB
:100F7000736F00006E69000063200000415700009D
:100F80002D480000453100003030000020000000F6
:100F90003220EF00437D2000008041001040BA0065
:100FA0000160EF000000060043650000696C00006E
:100FB000696E000067560000494500005720000098
:100FC0002020000020200000202000002000000041
:100FD0003220EF00437F2000008041001040BA0023
:100FE0000160EF0000000600436100006E6E00002B
:100FF0006F6E000020560000432D000043350000B6
:10100000306900002F720000202000002000000046
:101010003220EF0043812000008041001040BA00E0
:101020000160EF0000000600556E00006B6E0000CE
:101030006F7700006E200000436100006D650000C6
:10104000726100002020000020200000200000002D
:101050003220EF0043832000008041001040BA009E
:101060000160EF0000000600537900007374000077
:10107000656D000020430000616D00002049000004
:101080006E690000742000003A20000055730000D3
:101090006520000050720000657300006574000058
:1010A00031320000000000003220EF0003862000F3
:1010B000008041001040BA000160EF00000006000F
:1010C0005379000073740000656D00002043000038
:1010D000616D0000204900006E690000742000006E
:1010E0003A200000486F00006D65000020430000BA
:1010F000616D0000657200006120000000000000CA
:101100003220EF00C3882000008041001040BA0068
:101110000160EF0000000600457800007420000028
:10112000507200006573000065740000733A00009F
:1011300020430000616D000031200000312D0000CF
:10114000313200002C200000436100006D320000AD
:10115000204E00006F6E0000650000003220EF009E
:10116000A38B2000008041001040BA000160EF0016
:101170000000060045780000742000005072000056
:101180006573000065740000733A0000204300009E
:10119000616D000031200000312D0000362C000070
:1011A00020430000616D000032200000312D00005E
:1011B000360000003220EF00638E200000804100E6
:1011C0001040BA000160EF0000000600436100001B
:1011D0006D200000536500006C200000466F000089
:1011E0006C6C00006F7700007320000050720000EC
:1011F0006576000069650000773A00002045000030
:101200006E610000626C0000656400000000000078
:101210003220EF0043912000008041001040BA00CE
:101220000160EF0000000600436100006D20000037
:10123000536500006C200000466F00006C6C0000DD
:101240006F77000073200000507200006576000088
:1012500069650000773A00002044000069730000CF
:10126000616200006C650000640000003220EF0045
:1012700023942000008041001040BA000160EF007C
:1012800000000600507200006573000065740000E5
:10129000204C00006F63000061740000696F000063
:1012A0006E3A0000203100002D3600002049000079
:1012B0006E430000616D00002C3600002D310000EF
:1012C000322000004C6F0000636100006C000000E1
:1012D0003220EF0043972000008041001040BA0008
:1012E0000160EF000000060050720000657300000E
:1012F00065740000204C00006F6300006174000002
:10130000696F00006E3A0000203100002D310000AE
:10131000322000004C6F0000636100006C00000090
:101320003220EF00C3992000008041001040BA0035
:101330000160EF0000000600486F000073740000B9
:101340002053000065720000696100006C200000FD
:10135000496E000070750000743A000020450000DE
:101360006E610000626C0000656400000000000017
:101370003220EF00439C2000008041001040BA0062
:101380000160EF0000000600486F00007374000069
:101390002053000065720000696100006C200000AD
:1013A000496E000070750000743A0000204400008F
:1013B00069730000616200006C6500006400000059
:1013C0003220EF00C39E2000008041001040BA0090
:1013D0000160EF0000000600536500007269000024
:1013E000616C000020450000636800006F3A000057
:1013F000204500006E610000626C00006564000022
:10140000000000003220EF00E3A020000080410037
:101410001040BA000160EF000000060053650000B4
:1014200072690000616C00002045000063680000E4
:101430006F3A000020440000697300006162000000
:101440006C650000640000003220EF0003A3200060
:10145000008041001040BA000160EF00000006006B
:101460005365000072690000616C000020490000B3
:101470006E6600006F3A0000204F00006E00000012
:101480003220EF00C3A42000008041001040BA00C9
:101490000160EF0000000600536500007269000063
:1014A000616C0000204900006E6600006F3A000089
:1014B000204F000066660000000000003220EF00B0
:1014C000A3A62000008041001040BA000160EF0098
:1014D00000000600546100006C6C000079200000E0
:1014E0004C650000766500006C3A00002041000069
:1014F0006374000069760000652000004C6F0000F6
:10150000770000003220EF00E3A8200000804100B7
:101510001040BA000160EF000000060054610000B6
:101520006C6C0000792000004C65000076650000BE
:101530006C3A0000204100006374000069760000EE
:101540006520000048690000676800000000000096
:101550003220EF0043AB2000008041001040BA0071
:101560000160EF0000000600000000003220EF00E4
:1015700023AC2000008041001040BA000160EF0061
:10158000000006005379000073740000656D0000D0
:10159000204D00006F640000653A0000204100000B
:1015A000757400006F0000003220EF0003AE2000D1
:1015B000008041001040BA000160EF00000006000A
:1015C0005379000073740000656D0000204D000029
:1015D0006F640000653A0000204D0000616E00005D
:1015E000756100006C0000003220EF0003B02000A5
:1015F000008041001040BA000160EF0000000600CA
:1016000044690000616700006E6F000073740000A1
:1016100069630000204D00006F640000653A00001F
:10162000204F00006E0000003220EF0003B22000C7
:10163000008041001040BA000160EF000000060089
:1016400044690000616700006E6F00007374000061
:1016500069630000204D00006F640000653A0000DF
:10166000204F000066660000000000003220EF00FE
:1016700023B42000008041001040BA000160EF0058
:10168000000006005365000072690000616C0000F4
:101690002044000069610000672000004D6F0000D9
:1016A000646500003A2000004F6E0000000000005A
:1016B0003220EF0043B62000008041001040BA0005
:1016C0000160EF0000000600536500007269000031
:1016D000616C000020440000696100006720000088
:1016E0004D6F0000646500003A2000004F66000066
:1016F000660000003220EF0063B820000080410047
:101700001040BA000160EF000000060054720000B3
:10171000616E000073690000746900006F6E000064
:10172000204D00006F640000653A00002043000077
:1017300075740000000000003220EF0083BA200022
:10174000008041001040BA000160EF000000060078
:1017500054720000616E000073690000746900003B
:101760006F6E0000204D00006F640000653A0000BD
:10177000204D000069780000000000003220EF00DA
:10178000A3BC2000008041001040BA000160EF00BF
:101790000000060054720000616E000073690000D2
:1017A000746900006F6E0000204D00006F6400003F
:1017B000653A0000205700006970000065000000D5
:1017C0003220EF00C3BE2000008041001040BA006C
:1017D0000160EF0000000600466100006465000043
:1017E0002D5400006F5F0000426C00006163000038
:1017F0006B2000004D6F0000646500003A2000007F
:10180000416300007469000076650000000000007C
:101810003220EF0043C12000008041001040BA0098
:101820000160EF00000006004661000064650000F2
:101830002D5400006F5F0000426C000061630000E7
:101840006B2000004D6F0000646500003A2000002E
:10185000496E000041630000746900007665000075
:10186000000000003220EF00E3C3200000804100B0
:101870001040BA000160EF00000006005669000049
:10188000646500006F200000737700006974000039
:10189000636800003A20000044750000616C00009D
:1018A0002053000077690000746300006865000041
:1018B000722000004D6F0000646500000000000011
:1018C0003220EF00C3C62000008041001040BA0063
:1018D0000160EF000000060056690000646500002A
:1018E0006F200000737700006974000063680000D7
:1018F0003A200000536900006E6700006C6500002C
:1019000020530000776900007463000068650000E0
:10191000722000004D6F00006465000000000000B0
:101920003220EF00C3C92000008041001040BA00FF
:101930000160EF0000000600546100006B650000CC
:10194000204D00006F640000653A00002041000057
:10195000757400006F0000003220EF0083CB200080
:10196000008041001040BA000160EF000000060056
:10197000546100006B650000204D00006F640000A2
:10198000653A0000204D0000616E000075610000A6
:101990006C0000003220EF0063CD20000080410089
:1019A0001040BA000160EF0000000600426C000029
:1019B0006F6300006B200000496D0000616700004C
:1019C00065200000436F00006E740000726F00001D
:1019D0006C7300003A200000456E00006162000058
:1019E0006C65000064200000000000003220EF0061
:1019F00023D02000008041001040BA000160EF00B9
:101A000000000600426C00006F6300006B200000C5
:101A1000496D00006167000065200000436F000011
:101A20006E740000726F00006C7300003A200000BA
:101A30004469000073610000626C0000656400008E
:101A4000200000003220EF00E3D22000008041009F
:101A50001040BA000160EF00000006005472000060
:101A6000616E000073690000746900006F6E000011
:101A70002053000077610000703A0000204500000C
:101A80006E610000626C00006564000020000000D0
:101A90003220EF0043D52000008041001040BA0002
:101AA0000160EF000000060054720000616E00004B
:101AB00073690000746900006F6E0000205300001D
:101AC00077610000703A0000204400006973000054
:101AD000616200006C6500006420000000000000EE
:101AE0003220EF00C3D72000008041001040BA0030
:101AF0000160EF0000000600507200006F670000F8
:101B0000726100006D200000536500006C650000EC
:101B1000637400003A200000446900007361000013
:101B2000626C000065640000200000003220EF00BD
:101B300023DA2000008041001040BA000160EF006D
:101B4000000006005769000070650000204C00008E
:101B500065660000742000002D3E00002052000049
:101B60006967000068740000000000003220EF0088
:101B700023DC2000008041001040BA000160EF002B
:101B80000000060057690000706500002052000048
:101B90006967000068740000202D00003E200000EE
:101BA0004C65000066740000000000003220EF0069
:101BB00023DE2000008041001040BA000160EF00E9
:101BC0000000060057690000706500002042000018
:101BD0006F740000202D00003E200000546F0000B4
:101BE000700000003220EF00E3DF200000804100A1
:101BF0001040BA000160EF000000060057690000C5
:101C000070650000205400006F700000202D00005F
:101C10003E200000426F0000740000003220EF0000
:101C2000A3E12000008041001040BA000160EF00F5
:101C30000000060057690000706500002055000094
:101C40004C2000002D3E0000204C000052000000FF
:101C50003220EF0043E32000008041001040BA0032
:101C60000160EF0000000600576900007065000089
:101C700020550000522000002D3E0000204C0000A6
:101C80004C0000003220EF00E3E42000008041001F
:101C90001040BA000160EF00000006005769000024
:101CA00070650000204C00004C2000002D3E00001C
:101CB00020550000520000003220EF0083E6200093
:101CC000008041001040BA000160EF0000000600F3
:101CD0005769000070650000204C00005220000091
:101CE0002D3E0000205500004C0000003220EF0087
:101CF00023E82000008041001040BA000160EF009E
:101D000000000600576900007065000020430000D5
:101D1000656E0000742000002D3E0000204F000082
:101D200075740000000000003220EF0003EA20007C
:101D3000008041001040BA000160EF000000060082
:101D40004E6F00006E650000000000003220EF00C2
:101D500023EB2000008041001040BA000160EF003A
:101D6000000006004D65000064690000756D00000C
:101D7000000000003220EF0063EC200000804100F2
:101D80001040BA000160EF00000006004C61000046
:101D900072670000650000003220EF0083ED200034
:101DA000008041001040BA000160EF000000060012
:101DB000536D0000616C00006C0000003220EF00E9
:101DC000A3EE2000008041001040BA000160EF0047
:101DD000000006004C6F00007765000072200000D4
:101DE0004C650000667400002D25000073000000A3
:101DF0003220EF0043F02000008041001040BA0084
:101E00000160EF00000006005570000070650000E2
:101E1000722000005269000067680000742D000005
:101E200025730000000000003220EF0003F22000C4
:101E3000008041001040BA000160EF000000060081
:101E40004C6F0000776500007220000052690000AE
:101E500067680000742D000025730000000000007A
:101E60003220EF00C3F32000008041001040BA0090
:101E70000160EF0000000600557000007065000072
:101E8000722000006C650000667400002D250000C3
:101E9000730000003220EF0063F520000080410055
:101EA0001040BA000160EF00000006004D65000020
:101EB00064690000756D00002C2000004E6F00006A
:101EC00020540000726100006E73000000000000EA
:101ED0003220EF0043F72000008041001040BA009C
:101EE0000160EF00000006004D650000646900001D
:101EF000756D00002C20000054720000616E00001F
:101F0000732000002575000025250000000000005A
:101F10003220EF0043F92000008041001040BA0059
:101F20000160EF00000006004C61000072670000D5
:101F3000652C0000204E00006F200000547200004D
:101F4000616E0000730000003220EF0003FB2000F0
:101F5000008041001040BA000160EF000000060060
:101F60004C61000072670000652C000020540000E6
:101F7000726100006E7300002025000075250000CE
:101F8000250000003220EF00E3FC2000008041002B
:101F90001040BA000160EF00000006004675000026
:101FA0006C6C00002C2000004E6F000020540000DC
:101FB000726100006E730000000000003220EF002C
:101FC000A3FE2000008041001040BA000160EF0035
:101FD00000000600467500006C6C00002C2000001C
:101FE00054720000616E000073200000257500002F
:101FF00025250000000000003220EF0083002100B2
:10200000008041001040BA000160EF0000000600AF
:10201000536D0000616C00006C2C0000204E00002D
:102020006F20000054720000616E00007300000019
:102030003220EF0043022100008041001040BA002E
:102040000160EF0000000600536D0000616C0000AD
:102050006C2C000020540000726100006E730000C0
:102060002025000075250000250000003220EF002B
:1020700023042100008041001040BA000160EF00FD
:102080000000060048440000203100003038000005
:102090003070000020350000392E00003934000077
:1020A000487A0000000000003220EF000306210003
:1020B000008041001040BA000160EF0000000600FF
:1020C000484400002031000030380000307000002B
:1020D00020350000304800007A2000002020000059
:1020E000000000003220EF00E307210000804100E3
:1020F0001040BA000160EF000000060048440000F4
:102100002031000030380000306900002035000028
:10211000392E000039340000487A00000000000029
:102120003220EF00C3092100008041001040BA00B6
:102130000160EF000000060048440000203100006C
:1021400030380000306900002035000030480000C1
:102150007A20000020200000000000003220EF0064
:10216000A30B2100008041001040BA000160EF0085
:102170000000060048440000202000003732000024
:102180003050000020200000353900002E390000BA
:10219000344800007A0000003220EF00830D210057
:1021A000008041001040BA000160EF00000006000E
:1021B000484400002020000037320000305000006A
:1021C0002020000035300000487A00002020000068
:1021D000200000003220EF00630F2100008041004A
:1021E0001040BA000160EF000000060048560000F1
:1021F0002020000036340000307800002034000039
:102200003830000020360000304800007A0000001E
:102210003220EF0043112100008041001040BA003D
:102220000160EF000000060048560000202000007A
:1022300036340000307800002034000038300000D0
:1022400020370000354800007A0000003220EF00FF
:1022500023132100008041001040BA000160EF000C
:102260000000060048560000202000003830000022
:1022700030780000203600003030000020360000AA
:10228000304800007A0000003220EF0003152100E2
:10229000008041001040BA000160EF00000006001D
:1022A0004856000020310000303200003478000031
:1022B000203700003638000020360000304800008B
:1022C0007A0000003220EF00E31621000080410078
:1022D0001040BA000160EF00000006004856000000
:1022E0002031000030320000347800002037000038
:1022F0003638000020370000354800007A00000022
:102300003220EF00C3182100008041001040BA00C5
:102310000160EF0000000600485600002031000078
:1023200032380000307800003130000032340000D4
:1023300020360000304800007A0000003220EF0014
:10234000A31A2100008041001040BA000160EF0094
:10235000000006004856000020310000323800001E
:1023600030780000203700003638000020360000AA
:10237000304800007A0000003220EF00831C21006A
:10238000008041001040BA000160EF00000006002C
:102390004856000020310000333600003678000037
:1023A000203700003638000020360000304800009A
:1023B0007A0000003220EF00631E210000804100FF
:1023C0001040BA000160EF0000000600485600000F
:1023D000203100003430000030780000313000003F
:1023E0003530000020360000304800007A00000040
:1023F0003220EF0043202100008041001040BA004D
:102400000160EF0000000600485600002031000087
:1024100036300000307800003132000030300000EB
:1024200020360000304800007A0000003220EF0023
:1024300023222100008041001040BA000160EF001B
:10244000000006004856000020310000393200002C
:1024500030780000313200003030000020360000BB
:10246000304800007A0000003220EF0003242100F1
:10247000008041001040BA000160EF00000006003B
:10248000202000004E6F0000742000004176000004
:10249000616900006C610000626C00006520000052
:1024A000200000003220EF00E325210000804100E1
:1024B0001040BA000160EF00000006005344000025
:1024C000203400003830000069200000323900005C
:1024D0002E390000374800007A0000003220EF005B
:1024E000A3272100008041001040BA000160EF00E6
:1024F0000000060053440000204E0000545300002A
:1025000043200000532D0000566900006465000060
:102510006F0000003220EF0063292100008041009D
:102520001040BA000160EF000000060053440000B4
:1025300020350000373600006920000032350000E9
:10254000487A0000000000003220EF00032B210039
:10255000008041001040BA000160EF00000006005A
:102560005344000020500000414C00002053000064
:102570002D56000069640000656F00000000000037
:102580003220EF00C32C2100008041001040BA002F
:102590000160EF000000060053440000204E0000E0
:1025A0005453000043200000436F00006D70000092
:1025B0006F73000069740000650000003220EF00B6
:1025C000A32E2100008041001040BA000160EF00FE
:1025D000000006005344000020500000414C000061
:1025E000204300006F6D0000706F000073690000F1
:1025F00074650000000000003220EF0083302100ED
:10260000008041001040BA000160EF0000000600A9
:10261000446F0000466900006E64000041630000E2
:102620007469000076650000507200006573000058
:102630006574000073200000506F00007274000089
:10264000202500006420000062610000640A000090
:102650000D0000003220EF00030220008301500033
:102660000500310063342100008041001040BA00B1
:102670000160EF000000060060342100838141000A
:10268000808141001380BA00000006000A0D72002C
:10269000446F6500466973006E64650041637400B1
:1026A0007469200076653100507220006573250042
:1026B00065744C007320580043613A006D2020007F
:1026C000256420003A2020002D5000003220EF0029
:1026D00023372100008041001040BA000160EF0064
:1026E00000000600553800005F490000535200000A
:1026F000202500003258000020250000325800003C
:10270000202500003258000020250000325800002B
:1027100020250000325800000A0D000000000000D3
:102720003220EF00C3392100008041001040BA0080
:102730000160EF0000000600553800005F42000015
:102740003020000049530000522D00004572000067
:1027500072200000253200005820000025320000C1
:1027600058200000253200005820000025320000CB
:10277000582000005B250000325800005D0A000070
:102780000D0000003220EF00E33C210000804100FA
:102790001040BA000160EF0000000600553800004C
:1027A0005F4200003120000049530000522D00001C
:1027B0004572000072200000253200005820000001
:1027C000253200005820000025320000582000006B
:1027D0005B250000325800005D200000253200001B
:1027E000580A00000D0000003220EF0003402100D5
:1027F000008041001040BA000160EF0000000600B8
:10280000553800005F4200003220000049530000AC
:10281000522D000045720000722000002532000099
:102820005820000025320000582000005B250000E1
:10283000325800005D2000002532000058200000C2
:1028400025320000580A00000D0000003220EF0081
:1028500023432100008041001040BA000160EF00D6
:1028600000000600553800005F42000033200000E1
:1028700049530000522D00004572000072200000F4
:1028800025320000582000005B250000325800006F
:102890005D20000025320000582000002532000095
:1028A0005820000025320000582000000A0D0000CA
:1028B000000000003220EF0063462100008041004C
:1028C0001040BA000160EF0000000600553800001B
:1028D0005F4200003420000049530000522D0000E8
:1028E00045720000722000005B2500003258000095
:1028F0005D20000025320000582000002532000035
:102900005820000025320000582000002532000029
:10291000582000000A0D0000000000003220EF00E7
:10292000A3492100008041001040BA000160EF007F
:1029300000000600553900005F49000053520000B6
:102940002025000032580000202800002532000019
:1029500078290000253200005820000025320000B0
:1029600058200000253200005820000025320000C9
:10297000580A00000D0000003220EF00834C2100B7
:10298000008041001040BA000160EF000000060026
:10299000553900005F42000030200000495300001C
:1029A000522D000045720000722000002532000008
:1029B0005820000025320000582000002532000079
:1029C0005820000025320000582000005B25000040
:1029D000325800005D0A00000D0000003220EF00B8
:1029E000A34F2100008041001040BA000160EF00B9
:1029F00000000600553900005F4200003120000051
:102A000049530000522D0000457200007220000062
:102A10002532000058200000253200005820000018
:102A200025320000582000005B25000032580000CD
:102A30005D20000025320000580A00000D00000053
:102A40003220EF00C3522100008041001040BA0044
:102A50000160EF0000000600553900005F420000F1
:102A60003220000049530000522D00004572000042
:102A7000722000002532000058200000253200009E
:102A8000582000005B250000325800005D20000047
:102A9000253200005820000025320000580A0000AE
:102AA0000D0000003220EF00E30120008301500000
:102AB00005003100E3562100008041001040BA00BB
:102AC0000160EF0000000600E05621008381410014
:102AD000808141001380BA000000060055393200A1
:102AE0005F4258003320200049532500522D320008
:102AF00045725800722020002532250058203200EF
:102B00002825580032780A00295B0D002532000084
:102B1000585D0000202500003220EF00E301200076
:102B20008301500005003100835A210000804100DC
:102B30001040BA000160EF0000000600805A21003A
:102B400083814100808141001380BA0000000600AB
:102B5000553932005F425800352020004953250086
:102B6000522D320045725800722020002532250077
:102B7000582032002825580032780A00295B0D00C1
:102B800025320000585D0000202500003220EF00B3
:102B9000235D2100008041001040BA000160EF0079
:102BA00000000600553900005F420000342000009C
:102BB00049530000522D00004572000072200000B1
:102BC0005B250000325800005D2000002532000027
:102BD0005820000025320000582000002532000057
:102BE0005820000025320000580A00000D000000A7
:102BF0003220EF0043602100008041001040BA0005
:102C00000160EF0000000600427400006E28000022
:102C1000254C0000582F0000256C0000752900008D
:102C20002D47000072700000312000000A0D0000E6
:102C3000000000003220EF006362210000804100AC
:102C40001040BA000160EF000000060020200000E4
:102C5000504700004D2000004D6F000064650000EB
:102C600020410000637400006976000065200000C8
:102C7000200000003220EF0063642100008041004A
:102C80001040BA000160EF0000000600506F000025
:102C900077650000722000004F660000660A0000A1
:102CA0000D0000003220EF00E365210000804100AC
:102CB0001040BA000160EF0000000600506F0000F5
:102CC00077650000722000004F6E00000A0D0000C2
:102CD000000000003220EF00636721000080410007
:102CE0001040BA000160EF00000006002020000044
:102CF0002020000020410000757400006F200000BB
:102D00004D6F0000646500002020000020200000BE
:102D1000000000003220EF006369210000804100C4
:102D20001040BA000160EF0000000600417500008D
:102D3000746F00004D6F0000646500000A0D000014
:102D4000000000003220EF00E36A21000080410013
:102D50001040BA000160EF000000060020200000D3
:102D6000204D0000616E0000756100006C200000C5
:102D70004D6F00006465000020200000202000004E
:102D8000000000003220EF00E36C210000804100D1
:102D90001040BA000160EF00000006004D61000025
:102DA0006E4D00006F640000650A00000D00000019
:102DB0003220EF00436E2100008041001040BA0035
:102DC0000160EF0000000600204100007574000063
:102DD0006F2000004D6F000064650000204100007E
:102DE00063740000697600006520000000000000A8
:102DF0003220EF0043702100008041001040BA00F3
:102E00000160EF000000060020200000204D0000BF
:102E1000616E0000756100006C200000466F0000CC
:102E200063750000732000002020000000000000F7
:102E30003220EF0043722100008041001040BA00B0
:102E40000160EF0000000600466F0000637500009F
:102E5000734D0000616E00000A0D000000000000CC
:102E60003220EF00C3732100008041001040BA00FF
:102E70000160EF000000060020200000202000007C
:102E800041750000746F0000204600006F63000071
:102E900075730000202000002020000000000000CA
:102EA0003220EF00C3752100008041001040BA00BD
:102EB0000160EF0000000600466F0000637500002F
:102EC00073410000757400006F0A00000D000000DF
:102ED0003220EF0043772100008041001040BA000B
:102EE0000160EF000000060020200000202000000C
:102EF000204600006F63000075730000206E000024
:102F00002F610000202000002020000000000000B1
:102F10003220EF0043792100008041001040BA00C8
:102F20000160EF00000006004E6F0000204300002B
:102F3000616D0000657200006120000053650000B3
:102F40006C65000063740000656400000000000010
:102F50003220EF00437B2100008041001040BA0086
:102F60000160EF0000000600204300004355000010
:102F7000204D00006F6400006520000041630000E8
:102F80007469000076650000200000003220EF0028
:102F9000237D2100008041001040BA000160EF0055
:102FA00000000600204E00006F7400002073000037
:102FB00075700000706F000072740000656400009E
:102FC00020200000200000003220EF00037F2100BD
:102FD000008041001040BA000160EF0000000600D0
:102FE000204D0000616E0000756100006C20000043
:102FF000576800006974000065200000426100000D
:103000006C200000000000003220EF00038121004E
:10301000008041001040BA000160EF00000006008F
:10302000574200004D6100006E750000616C0000A9
:103030000A0D0000000000003220EF008382210012
:10304000008041001040BA000160EF00000006005F
:10305000204F00006E6500002050000075730000D6
:1030600068200000574200002020000020200000BF
:1030700020200000000000003220EF0083842100A7
:10308000008041001040BA000160EF00000006001F
:103090004F500000574200000A0D000000000000E1
:1030A0003220EF00C3852100008041001040BA00AB
:1030B0000160EF0000000600204F000050570000A4
:1030C000422000004E6F0000207300007570000069
:1030D000706F000072740000200000003220EF00CA
:1030E000A3872100008041001040BA000160EF007A
:1030F0000000060041750000746F000020570000BA
:10310000686900007465000020420000616C0000E6
:10311000616E000063650000000000003220EF00D7
:10312000A3892100008041001040BA000160EF0037
:10313000000006005742000041750000746F000057
:103140000A0D0000000000003220EF00038B210078
:10315000008041001040BA000160EF00000006004E
:10316000576800006974000065200000426100009B
:103170006C6100006E630000652000006E2F00008F
:1031800061200000000000003220EF00038D2100CC
:10319000008041001040BA000160EF00000006000E
:1031A00020200000204D0000616E000075610000CD
:1031B0006C200000497200006973000020200000AC
:1031C00020200000000000003220EF00038F2100CB
:1031D000008041001040BA000160EF0000000600CE
:1031E00049720000697300004D6100006E0A000022
:1031F0000D0000003220EF006390210000804100AC
:103200001040BA000160EF0000000600202000001E
:1032100020410000757400006F200000497200001A
:103220006973000020200000202000002020000002
:10323000000000003220EF00639221000080410076
:103240001040BA000160EF00000006004972000063
:103250006973000041750000746F00000A0D0000E2
:10326000000000003220EF00E393210000804100C5
:103270001040BA000160EF000000060020200000AE
:10328000202000004972000069730000206E0000D9
:103290002F610000202000002020000020200000DE
:1032A000000000003220EF00E39521000080410083
:1032B0001040BA000160EF0000000600426100000B
:1032C000636B00006C6900006768000074200000F8
:1032D000436F00006D700000204F00006666000024
:1032E000000000003220EF00E39721000080410041
:1032F0001040BA000160EF0000000600424C0000E0
:10330000432000004F660000660A00000D00000028
:103310003220EF0043992100008041001040BA00A4
:103320000160EF000000060042610000636B0000D6
:103330006C6900006768000074200000436F0000A3
:103340006D700000204F00006E20000000000000A3
:103350003220EF00439B2100008041001040BA0062
:103360000160EF0000000600424C00004320000016
:103370004F6E00000A0D0000000000003220EF0038
:10338000A39C2100008041001040BA000160EF00C2
:103390000000060042610000636B00006C690000E1
:1033A0006768000074200000436F00006D7000002B
:1033B000206E00002F610000000000003220EF00AE
:1033C000A39E2100008041001040BA000160EF0080
:1033D0000000060020200000204800006F6D000063
:1033E00065200000436100006D650000726100000F
:1033F00020200000200000003220EF0083A02100E8
:10340000008041001040BA000160EF00000006009B
:10341000486F00006D650000436100006D0A000008
:103420000D0000003220EF00E3A1210000804100E8
:103430001040BA000160EF000000060020480000C4
:103440006F6D000065200000436100006D650000A5
:1034500072610000206E00002F610000000000007B
:103460003220EF00C3A32100008041001040BA00C9
:103470000160EF0000000600427400006E280000AA
:10348000256C0000782F0000256C000075290000D5
:103490002D47000072700000332000000A0D00006C
:1034A000000000003220EF00E3A521000080410071
:1034B0001040BA000160EF000000060050720000EA
:1034C0006F67000020430000257500000A0D000012
:1034D000000000003220EF0063A7210000804100BF
:1034E0001040BA000160EF000000060050720000BA
:1034F0006F670000204C0000736700000A0D000099
:10350000000000003220EF00E3A82100008041000D
:103510001040BA000160EF00000006005072000089
:103520006F67000020500000697000000A0D000065
:10353000000000003220EF0063AA2100008041005B
:103540001040BA000160EF00000006005072000059
:1035500065760000204C0000736700000A0D000033
:10356000000000003220EF00E3AB210000804100AA
:103570001040BA000160EF00000006005072000029
:103580006576000020430000257500000A0D00004C
:10359000000000003220EF0063AD210000804100F8
:1035A0001040BA000160EF000000060050720000F9
:1035B0006576000020500000697000000A0D0000D0
:1035C000000000003220EF00E3AE21000080410047
:1035D0001040BA000160EF000000060042740000D5
:1035E0006E280000254C0000582F0000256C0000BC
:1035F000752900002D470000727000003420000083
:103600000A0D0000000000003220EF0003B121008D
:10361000008041001040BA000160EF000000060089
:103620002020000020200000436100006D650000A4
:1036300072610000202500006420000020200000AE
:1036400020200000200000003220EF0003B3210002
:10365000008041001040BA000160EF000000060049
:103660004E6F000020500000726F00006772000073
:10367000616D00002073000075700000706F000025
:1036800072740000000000003220EF0003B521003A
:10369000008041001040BA000160EF000000060009
:1036A000506700006D2000004D6F00006465000051
:1036B00020250000750A00000D0000003220EF00F8
:1036C000A3B62100008041001040BA000160EF0065
:1036D0000000060020500000726F000067720000BA
:1036E000616D0000204D00006F6400006520000047
:1036F0002020000020200000000000003220EF0009
:10370000A3B82100008041001040BA000160EF0022
:1037100000000600436100006D650000726100005A
:1037200020250000640A00000D0000003220EF0098
:1037300023BA2100008041001040BA000160EF0070
:10374000000006004E6F000020430000616D000085
:103750006572000061200000466F0000756E000079
:103760006420000020200000000000003220EF0054
:1037700023BC2100008041001040BA000160EF002E
:1037800000000600204900006E2000004361000098
:103790006D6500007261000020530000746F00002E
:1037A0007265000020250000640000003220EF0058
:1037B00023BE2100008041001040BA000160EF00EC
:1037C00000000600537400006F72000065200000C6
:1037D000256400000A0D0000000000003220EF0008
:1037E000A3BF2100008041001040BA000160EF003B
:1037F0000000060020200000526500006164000007
:10380000696E000067200000436100006D650000E4
:103810007261000020200000000000003220EF0054
:10382000A3C12100008041001040BA000160EF00F8
:103830000000060020200000537400006F7200009A
:10384000696E000067200000507200006573000080
:103850006574000020200000200000003220EF00EE
:10386000A3C32100008041001040BA000160EF00B6
:103870000000060020530000746F00007265000015
:103880002050000072650000736500007420000085
:103890002532000064200000200000003220EF00EC
:1038A000A3C52100008041001040BA000160EF0074
:1038B00000000600452D0000537400006F720000E8
:1038C00065200000253200006420000046610000F1
:1038D000696C000065640000000000003220EF0009
:1038E000A3C72100008041001040BA000160EF0032
:1038F0000000060020530000746F00007265000095
:1039000020250000326400002046000061690000AC
:103910006C650000640000003220EF0083C92100C4
:10392000008041001040BA000160EF000000060076
:10393000496E0000436100006D6500007261000087
:1039400020500000726500007365000074200000C4
:1039500025320000640000003220EF0083CB2100FC
:10396000008041001040BA000160EF000000060036
:10397000507200006573000065740000202500008F
:10398000640A00000D0000003220EF0003CD21008A
:10399000008041001040BA000160EF000000060006
:1039A0002020000050720000657300006574000064
:1039B0002025000032640000000000003220EF00EB
:1039C000A3CE2100008041001040BA000160EF004A
:1039D000000006002020000042610000642000007A
:1039E000507200006573000065740000202500001F
:1039F0003264000020200000000000003220EF00B0
:103A0000A3D02100008041001040BA000160EF0007
:103A100000000600202000004E6F00002050000033
:103A200072650000736500007420000025320000FC
:103A300064200000200000003220EF0083D221002B
:103A4000008041001040BA000160EF000000060055
:103A500045720000722000002D2000005049000037
:103A6000502000004163000074690000766500008A
:103A700020200000000000003220EF0083D421004D
:103A8000008041001040BA000160EF000000060015
:103A90004C53000047200000507200006573000086
:103AA000657400002532000064200000736100008E
:103AB00076650000640000003220EF0083D621000C
:103AC000008041001040BA000160EF0000000600D5
:103AD0004C53000047200000507200006573000046
:103AE000657400002532000064200000657200004B
:103AF000726F0000720000003220EF0083D82100B6
:103B0000008041001040BA000160EF000000060094
:103B10004C530000472000004E6F00002050000072
:103B200072650000736500007420000025320000FB
:103B300064200000200000003220EF0083DA210022
:103B4000008041001040BA000160EF000000060054
:103B5000427400006E280000254C0000582F000021
:103B6000256C0000752900002D47000072700000D0
:103B7000350A00000D0000003220EF0083DC210038
:103B8000008041001040BA000160EF000000060014
:103B90005769000070650000555200000A0D0000D2
:103BA000000000003220EF00E3DD21000080410032
:103BB0001040BA000160EF000000060057690000E5
:103BC00070650000435200000A0D00000000000074
:103BD0003220EF0043DF2100008041001040BA0096
:103BE0000160EF00000006005769000070650000EA
:103BF0004C5200000A0D0000000000003220EF00CF
:103C0000A3E02100008041001040BA000160EF00F5
:103C10000000060057690000706500005543000071
:103C20000A0D0000000000003220EF0003E2210036
:103C3000008041001040BA000160EF000000060063
:103C40005769000070650000434300000A0D000042
:103C5000000000003220EF0063E3210000804100FB
:103C60001040BA000160EF00000006005769000034
:103C7000706500004C4300000A0D000000000000C9
:103C80003220EF00C3E42100008041001040BA0060
:103C90000160EF0000000600576900007065000039
:103CA000554C00000A0D0000000000003220EF001B
:103CB00023E62100008041001040BA000160EF00BF
:103CC000000006005769000070650000434C0000CA
:103CD0000A0D0000000000003220EF0083E7210001
:103CE000008041001040BA000160EF0000000600B3
:103CF00057690000706500004C4C00000A0D000080
:103D0000000000003220EF00E3E8210000804100C5
:103D10001040BA000160EF00000006005769000083
:103D2000706500000A0D0000000000003220EF0066
:103D300023EA2100008041001040BA000160EF003A
:103D40000000060043750000740A00000D0000002A
:103D50003220EF0043EB2100008041001040BA0008
:103D60000160EF0000000600537700006974000056
:103D70006368000065720000204D00006F64000061
:103D80006520000025320000780A00000D000000C8
:103D90003220EF0043ED2100008041001040BA00C6
:103DA0000160EF00000006004D690000782F000060
:103DB00046540000420A00000D0000003220EF00CF
:103DC000A3EE2100008041001040BA000160EF0026
:103DD0000000060020200000202000005374000096
:103DE0006172000074200000546100006B650000E7
:103DF0002020000020200000000000003220EF0002
:103E0000A3F02100008041001040BA000160EF00E3
:103E10000000060020200000202000005461000067
:103E20006B650000204300006F6D0000706C0000A7
:103E30006574000065200000000000003220EF00E3
:103E4000A3F22100008041001040BA000160EF00A1
:103E500000000600202000004C73000067200000D6
:103E6000496E000063720000204D00006F64000086
:103E70006520000020200000000000003220EF003C
:103E8000A3F42100008041001040BA000160EF005F
:103E90000000060050690000705500004C0A000048
:103EA0000D0000003220EF00E3F52100008041000A
:103EB0001040BA000160EF00000006002020000062
:103EC0004C7300006720000044650000637200002E
:103ED000204D00006F6400006520000020200000DD
:103EE000000000003220EF00E3F7210000804100D5
:103EF0001040BA000160EF000000060050690000A9
:103F0000704C00004C0A00000D0000003220EF0051
:103F100023F92100008041001040BA000160EF0049
:103F2000000006005069000070550000520A0000B1
:103F30000D0000003220EF0063FA210000804100F4
:103F40001040BA000160EF00000006005069000058
:103F5000704C0000520A00000D0000003220EF00FB
:103F6000A3FB2100008041001040BA000160EF0077
:103F7000000006004C73000067440000656E0000FE
:103F80000A0D0000000000003220EF0003FD2100B8
:103F9000008041001040BA000160EF000000060000
:103FA0004C73000067530000697A0000650A000046
:103FB0000D0000003220EF0063FE21000080410070
:103FC0001040BA000160EF0000000600546F0000CE
:103FD000676700006C650000207400006F2000001F
:103FE000496E000063720000656D0000656E0000A0
:103FF000740A00000D0000003220EF008300220050
:10400000008041001040BA000160EF00000006008F
:10401000546F0000676700006C65000020740000AA
:104020006F2000004465000063720000656D0000B1
:10403000656E0000740A00000D0000003220EF00E1
:10404000A3022200008041001040BA000160EF008E
:1040500000000600507200006F64000075630000ED
:10406000746900006F6E00005669000065770000FB
:1040700048440000257300000A0D00000000000005
:104080003220EF00C3042200008041001040BA003B
:104090000160EF000000060020200000202000004A
:1040A000436F00006D700000696C000065640000E3
:1040B0003A200000257300002061000074200000F9
:1040C000257300000A0D0000000000003220EF0000
:1040D00023072200008041001040BA000160EF0079
:1040E00000000600313400003A350000333A000089
:1040F00030360000000000003220EF00830822006C
:10410000008041001040BA000160EF00000006008E
:10411000202000002053000061760000696E00003E
:1041200067200000436F00006E66000069670000B2
:1041300020200000000000003220EF00830A22004F
:10414000008041001040BA000160EF00000006004E
:1041500020200000205200006573000065740000FC
:104160002056000069640000656F000020200000F8
:10417000000000003220EF00630C220000804100AC
:104180001040BA000160EF0000000600204300006C
:104190006C65000061720000696E0000672000001D
:1041A0005072000065730000657400007300000029
:1041B0003220EF00430E2200008041001040BA0080
:1041C0000160EF0000000600204300006C65000065
:1041D00061720000696E000067200000416C000001
:1041E0006C20000020200000000000003220EF00C2
:1041F00023102200008041001040BA000160EF004F
:104200000000060020520000657300007461000089
:104210007274000020530000797300007465000080
:104220006D200000000000003220EF000312220089
:10423000008041001040BA000160EF00000006005D
:10424000202000004E6F0000742000006F6E000000
:1042500020500000726500007365000074200000AB
:10426000000000003220EF00E31322000080410034
:104270001040BA000160EF0000000600456E00002B
:10428000616200006C650000204800006F73000050
:10429000742000005365000072690000616C00002A
:1042A000000000003220EF00E315220000804100F2
:1042B0001040BA000160EF000000060044690000F1
:1042C00073610000626C000065200000536500000F
:1042D00072690000616C00002020000020200000B6
:1042E000000000003220EF00E317220000804100B0
:1042F0001040BA000160EF00000006000A0D000047
:10430000436F00006D6D0000616E000064200000CE
:10431000436F00006D7000006C6500007465000064
:104320000A0D00003E0000003220EF00031A2200B8
:10433000008041001040BA000160EF00000006005C
:10434000202000005368000075740000646F0000B6
:10435000776E000020410000637400006976000061
:1043600065200000000000003220EF00031C220046
:10437000008041001040BA000160EF00000006001C
:1043800020430000616D00006572000061200000A4
:10439000506F000077650000726400006F770000C6
:1043A0006E200000000000003220EF00031E2200FB
:1043B000008041001040BA000160EF0000000600DC
:1043C000204C00006F610000646900006E6700000F
:1043D000205000007265000073650000742000002A
:1043E00031320000000000003220EF0003202200E4
:1043F000008041001040BA000160EF00000006009C
:10440000536500006172000063680000696E00007F
:1044100067200000666F00007220000041740000F9
:1044200074610000636800006564000020430000C0
:10443000616D000065720000617300000D0A0000EC
:10444000000000003220EF00E32222000080410043
:104450001040BA000160EF0000000600506F00003D
:104460007274000020250000643A00000A0D00006C
:10447000000000003220EF00632422000080410091
:104480001040BA000160EF00000006004361000028
:104490006D6500007261000020530000656100003E
:1044A0007263000068200000436F00006D70000020
:1044B0006C650000746500000A0D00000A00000031
:1044C0003220EF00C3262200008041001040BA00D5
:1044D0000160EF000000060020560000432D0000A0
:1044E000433500003069000020200000205000000B
:1044F0006F720000742000003020000020000000D7
:104500003220EF00C3282200008041001040BA0092
:104510000160EF0000000600436100006E6F0000C4
:104520006E200000446500007465000063740000A4
:10453000656400000D0A0000000000003220EF005A
:10454000A32A2200008041001040BA000160EF0061
:1045500000000600204E00006F20000043610000B4
:104560006D20000020200000205000006F7200002D
:104570007420000030200000200000003220EF00F6
:10458000A32C2200008041001040BA000160EF001F
:10459000000006000D0A0000506100006E6100007E
:1045A000736F00006E690000632000004157000037
:1045B0002D48000045310000303000000D0A000099
:1045C000000000003220EF00E32E220000804100B6
:1045D0001040BA000160EF0000000600204100001A
:1045E000572D000048450000313000003020000009
:1045F000205000006F720000742000003020000086
:10460000200000003220EF00E33022000080410053
:104610001040BA000160EF000000060020470000D3
:104620006574000038200000000000003220EF0018
:1046300023322200008041001040BA000160EF00E8
:104640000000060020200000202D00002D2000008A
:1046500025320000582000002D2D00000A0D00001A
:10466000000000003220EF00E33322000080410010
:104670001040BA000160EF00000006000A0D0000C3
:104680002020000020670000657400003136000023
:10469000200000003220EF0063352200008041003E
:1046A0001040BA000160EF0000000600202000006A
:1046B000202D00002D200000254C00005820000077
:1046C0002D2D0000200A00000D0000003220EF0018
:1046D00023372200008041001040BA000160EF0043
:1046E000000006000A0D00002020000020670000E6
:1046F0006574000033320000200000003220EF001B
:10470000A3382200008041001040BA000160EF0091
:104710000000060020200000202D00002D200000B9
:10472000254C0000582000002D2D00000A0D00002F
:10473000000000003220EF00633A220000804100B8
:104740001040BA000160EF00000006000A0D0000F2
:1047500020430000616D000065720000615400009C
:104760007970000065200000000000003220EF009A
:10477000233C2200008041001040BA000160EF009D
:10478000000006000D0A0000536F00006E79000063
:1047900020450000564900002D4400003330000041
:1047A00028720000290D00000A0000003220EF00EE
:1047B000233E2200008041001040BA000160EF005B
:1047C0000000060020450000564900002D4400006E
:1047D0003330000028720000295000006F72000082
:1047E0007420000030200000200000003220EF0084
:1047F00023402200008041001040BA000160EF0019
:1048000000000600496E0000766100006C6900003F
:1048100064200000436100006D65000072610000CB
:104820000D0A0000000000003220EF0003422200C9
:10483000008041001040BA000160EF000000060057
:10484000204900006E760000616C00006964000081
:1048500020430000616D00006572000061000000EF
:104860003220EF00C3432200008041001040BA0014
:104870000160EF00000006000D0A0000536F000009
:104880006E79000020450000564900002D440000CC
:10489000333000002F330000312000000D0A0000EB
:1048A000000000003220EF00E345220000804100BC
:1048B0001040BA000160EF00000006002045000033
:1048C000564900002D440000333000002F33000013
:1048D000315000006F720000742000003020000092
:1048E000200000003220EF00E3472200008041005A
:1048F0001040BA000160EF00000006000D0A000041
:10490000536F00006E7900002045000056490000FA
:104910002D440000333000000D0A000000000000AC
:104920003220EF00C3492200008041001040BA004D
:104930000160EF000000060020450000564900001D
:104940002D440000333000002020000020500000E3
:104950006F72000074200000302000002000000072
:104960003220EF00C34B2200008041001040BA000B
:104970000160EF00000006000D0A00005661000013
:1049800064640000696F000020410000646400005E
:104990002D4100002D430000616D00000D0A000054
:1049A000000000003220EF00E34D220000804100B3
:1049B0001040BA000160EF00000006002041000036
:1049C000646400002D4100002D430000616D000073
:1049D000205000006F7200007420000030200000A2
:1049E000200000003220EF00E34F22000080410051
:1049F0001040BA000160EF00000006000D0A000040
:104A0000536F00006E7900002045000056490000F9
:104A10002D44000031300000300D00000A0000007D
:104A20003220EF00C3512200008041001040BA0044
:104A30000160EF000000060020450000564900001C
:104A40002D440000313000003020000020500000D4
:104A50006F72000074200000302000002000000071
:104A60003220EF00C3532200008041001040BA0002
:104A70000160EF00000006000D0A00005641000032
:104A800044440000494F000020480000442D00002D
:104A9000313800000D0A0000000000003220EF0055
:104AA000A3552200008041001040BA000160EF00D1
:104AB000000006005641000044440000494F000039
:104AC000204800004431000038200000506F0000F2
:104AD0007274000020300000000000003220EF005F
:104AE000A3572200008041001040BA000160EF008F
:104AF000000006000D0A0000536F00006E790000F0
:104B000020450000564900002D44000037300000C9
:104B10000D0A0000000000003220EF00835922003F
:104B2000008041001040BA000160EF000000060064
:104B300020450000564900002D4400003730000099
:104B400020200000205000006F7200007420000040
:104B500030200000200000003220EF00835B2200A4
:104B6000008041001040BA000160EF000000060024
:104B70000D0A0000536F00006E7900002042000013
:104B800052430000482D000037300000300D000077
:104B90000A0000003220EF00635D22000080410027
:104BA0001040BA000160EF00000006002042000043
:104BB00052430000482D0000373000003020000034
:104BC000205000006F7200007420000030200000B0
:104BD000200000003220EF00635F220000804100CF
:104BE0001040BA000160EF00000006000D0A00004E
:104BF000456C00006D6F000020430000616D0000F7
:104C000065720000610D00000A0000003220EF0014
:104C100023612200008041001040BA000160EF00D3
:104C200000000600204500006C6D00006F200000B1
:104C30002020000020200000205000006F720000A3
:104C40007420000030200000200000003220EF001F
:104C500023632200008041001040BA000160EF0091
:104C6000000006000D0A0000536F00006E7900007E
:104C700020420000524300002D330000303000007D
:104C80000D0A0000000000003220EF000365220042
:104C9000008041001040BA000160EF0000000600F3
:104CA00020420000524300002D330000303000004D
:104CB00020200000205000006F72000074200000CF
:104CC00030200000200000003220EF0003672200A7
:104CD000008041001040BA000160EF0000000600B3
:104CE0000D0A0000536F00006E79000020420000A2
:104CF000524300002D5A000037300000300D0000F4
:104D00000A0000003220EF00E3682200008041002A
:104D10001040BA000160EF000000060020420000D1
:104D2000524300002D5A00003730000030200000B0
:104D3000205000006F72000074200000302000003E
:104D4000200000003220EF00E36A220000804100D2
:104D50001040BA000160EF00000006000D0A0000DC
:104D6000536F00006E7900002042000052430000A3
:104D70002D5A000033330000300D00000A000000FF
:104D80003220EF00C36C2200008041001040BA00C6
:104D90000160EF00000006002042000052430000C6
:104DA0002D5A000033330000302000002050000056
:104DB0006F7200007420000030200000200000000E
:104DC0003220EF00C36E2200008041001040BA0084
:104DD0000160EF00000006000D0A0000536F0000A4
:104DE0006E79000020450000564900002D48000063
:104DF000443100000D0A0000000000003220EF00E6
:104E0000A3702200008041001040BA000160EF0052
:104E10000000060020450000564900002D48000013
:104E20004431000020200000205000006F7200007C
:104E30007420000030200000200000003220EF002D
:104E4000A3722200008041001040BA000160EF0010
:104E5000000006000D0A00005661000064640000B6
:104E6000696F000020430000656900006C69000064
:104E70006E67000056490000455700000D0A00000B
:104E8000000000003220EF00E374220000804100A7
:104E90001040BA000160EF0000000600204300004F
:104EA000562F0000435600004D5000002020000007
:104EB000205000006F7200007420000030200000BD
:104EC000200000003220EF00E37622000080410045
:104ED0001040BA000160EF0000000600556E0000AF
:104EE0006B6E00006F7700006E20000043610000D1
:104EF0006D650000726100000D0A000000000000F6
:104F00003220EF00C3782200008041001040BA0038
:104F10000160EF0000000600205500006E6B0000ED
:104F20006E6F0000776E000020200000205000000F
:104F30006F7200007420000030200000200000008C
:104F40003220EF00C37A2200008041001040BA00F6
:104F50000160EF00000006000A0D00002041000083
:104F6000542F00004D4400005F4D00006F640000AE
:104F7000654900006E710000200000003220EF0043
:104F8000A37C2200008041001040BA000160EF00C5
:104F9000000006000D0A00002057000061690000B3
:104FA000745300006F6E000079410000636B0000D5
:104FB000000000003220EF00637E220000804100EC
:104FC0001040BA000160EF00000006000D0A00006A
:104FD0002057000061690000745300006F6E0000EC
:104FE000790000003220EF00E37F220000804100C2
:104FF0001040BA000160EF00000006002A570000D0
:1050000061690000745300006F6E000079000000B9
:105010003220EF0043812200008041001040BA009E
:105020000160EF0000000600202D00002054000069
:10503000696D0000656F0000757400002025000098
:1050400075200000286D0000732900000D0A000083
:10505000000000003220EF00638322000080410046
:105060001040BA000160EF0000000600436100003C
:105070006E630000656C00002053000031200000CA
:10508000000000003220EF00E38422000080410095
:105090001040BA000160EF0000000600436100000C
:1050A0006E630000656C0000205300003220000099
:1050B000000000003220EF006386220000804100E3
:1050C0001040BA000160EF00000006000A0D000069
:1050D00020200000204700006574000042520000BC
:1050E00043500000616E0000546900006C740000C1
:1050F000506F000073200000000000003220EF001D
:10510000A3882200008041001040BA000160EF0037
:105110000000060020200000202D00002D200000AF
:10512000503A0000254C0000582C0000543A000072
:10513000254C0000582000002D2D00000A0D000015
:10514000000000003220EF00E38A220000804100CE
:105150001040BA000160EF0000000600205D000072
:105160000A0D0000000000003220EF00038C220036
:10517000008041001040BA000160EF00000006000E
:105180000D0A000020570000616900007443000010
:10519000616E00006F6E0000000000003220EF0022
:1051A000A38D2200008041001040BA000160EF0092
:1051B00000000600202D000020540000696D000052
:1051C000656F000075740000202500006C750000FC
:1051D000202800006D730000290D00000A00000067
:1051E0003220EF00C38F2200008041001040BA003F
:1051F0000160EF00000006000D0A000020570000CB
:105200006169000074500000616E0000617300006D
:105210006F6E000069630000000000003220EF00A4
:10522000A3912200008041001040BA000160EF000D
:105230000000060020200000466F0000637500009B
:10524000732000004E650000617200000000000045
:105250003220EF0043932200008041001040BA004A
:105260000160EF000000060020200000466F0000F3
:1052700063750000732000004661000072000000AA
:105280003220EF00C3942200008041001040BA0099
:105290000160EF000000060020200000466F0000C3
:1052A0006375000073200000506F00007320000041
:1052B0006E2F0000610000003220EF008396220074
:1052C000008041001040BA000160EF0000000600BD
:1052D00020200000466F000063750000732000006E
:1052E0004E65000061720000202500006C75000012
:1052F000000000003220EF0063982200008041008F
:105300001040BA000160EF000000060020200000FD
:10531000466F0000637500007320000046610000C6
:1053200072200000256C0000750000003220EF00A4
:10533000239A2200008041001040BA000160EF0073
:105340000000060020200000466F0000637500008A
:1053500073200000506F000073200000256C0000D7
:10536000750000003220EF00E39B22000080410026
:105370001040BA000160EF0000000600202000008D
:105380002049000072690000733A000020250000E7
:10539000730000003220EF00639D22000080410076
:1053A0001040BA000160EF0000000600202000005D
:1053B000204900007269000073200000257300007E
:1053C000000000003220EF00E39E22000080410038
:1053D0001040BA000160EF0000000600202000002D
:1053E000204900007269000073200000256C000055
:1053F000750000003220EF0063A022000080410011
:105400001040BA000160EF000000060020200000FC
:105410004D610000782000005A6F00006F6D0000A1
:1054200020250000750000003220EF0003A22200BA
:10543000008041001040BA000160EF00000006004B
:10544000202000004D610000782000005061000025
:105450006E20000025750000000000003220EF00E3
:10546000A3A32200008041001040BA000160EF00B9
:1054700000000600202000004D61000078200000A0
:10548000546900006C7400002025000075000000C5
:105490003220EF0043A52200008041001040BA00F6
:1054A0000160EF00000006003E25000073200000B0
:1054B0004E6F000074200000466F0000756E000003
:1054C000640A00000D3E0000000000003220EF00E2
:1054D00023A72200008041001040BA000160EF00C5
:1054E00000000600436F00006D700000696C000052
:1054F000656400003A200000257300002061000070
:1055000074200000257300000A0D00000000000058
:105510003220EF00A302200083015000050031007B
:1055200043AA2200008041001040BA000160EF0051
:105530000000060040AA22008381410080814100D2
:105540001380BA00000006000D0A4400537965007C
:1055500073746600656D61002053750065746C009E
:10556000746974006E672000733A50000A0D72006F
:105570000A0D65004465730066616500756C740012
:1055800074203A00436120006D652500726164005B
:105590003A200A0025640D000A0D00003220EF00B9
:1055A000A3AD2200008041001040BA000160EF006E
:1055B000000006000D0A0000576900007065000039
:1055C00020440000657300006372000069700000F1
:1055D000746900006F6E00003A200000257300001F
:1055E0000A0D0000000000003220EF0003B022008E
:1055F000008041001040BA000160EF00000006008A
:105600005069000070200000204400006573000015
:105610006372000069700000746900006F6E000022
:105620003A200000257300000A0D00000000000071
:105630003220EF0043B22200008041001040BA0047
:105640000160EF00000006004C73000067200000BE
:105650002044000065730000637200006970000060
:10566000746900006F6E00003A200000257300008E
:105670000A0D0000000000003220EF0083B4220079
:10568000008041001040BA000160EF0000000600F9
:105690000D0A0000507200006F6700007261000088
:1056A0006D2D000057690000706500002044000067
:1056B0006573000063720000697000007469000087
:1056C0006F6E00003A200000257300000A0D0000F4
:1056D000000000003220EF0063B72200008041008C
:1056E0001040BA000160EF00000006005072000098
:1056F0006F670000726100006D2D000050690000AE
:1057000070200000204400006573000063720000F8
:1057100069700000746900006F6E00003A2000009C
:10572000257300000A0D0000000000003220EF0089
:1057300023BA2200008041001040BA000160EF004F
:1057400000000600507200006F67000072610000E8
:105750006D2D00004C730000672000002044000005
:1057600065730000637200006970000074690000D6
:105770006F6E00003A200000257300000A0D000043
:10578000000000003220EF00E3BC22000080410056
:105790001040BA000160EF00000006000D0A000092
:1057A000507200006576000069650000772D0000EA
:1057B0005769000070650000204400006573000018
:1057C0006372000069700000746900006F6E000071
:1057D0003A200000257300000A0D000000000000C0
:1057E0003220EF00C3BF2200008041001040BA0009
:1057F0000160EF00000006005072000065760000B6
:1058000069650000772D00005069000070200000DD
:10581000204400006573000063720000697000009E
:10582000746900006F6E00003A20000025730000CC
:105830000A0D0000000000003220EF0083C22200A9
:10584000008041001040BA000160EF000000060037
:10585000507200006576000069650000772D000039
:105860004C730000672000002044000065730000B6
:105870006372000069700000746900006F6E0000C0
:105880003A200000257300000A0D0000000000000F
:105890003220EF0043C52200008041001040BA00D2
:1058A0000160EF0000000600507200006F6700000A
:1058B000726100006D2000004F75000074700000E0
:1058C00075740000204600006F7200006D610000DA
:1058D000743A000020250000730A00000D0000004B
:1058E0003220EF00C3C72200008041001040BA0000
:1058F0000160EF00000006005072000065760000B5
:1059000069650000772000004F750000747000008A
:1059100075740000204600006F7200006D61000089
:10592000743A000020250000730A00000D000000FA
:105930003220EF0043CA2200008041001040BA002C
:105940000160EF0000000600506F0000727400005C
:105950002025000075200000496E000070750000D1
:1059600074200000466F0000726D0000617400003A
:105970003A200000257300000A0D0000000000001E
:105980003220EF00C30220008301500005003100E7
:10599000C3CD2200008041001040BA000160EF003A
:1059A00000000600C0CD22008381410080814100BB
:1059B0001380BA00000006000A0D740050617500E3
:1059C0006E53720070656E00656420002020200018
:1059D00020205000546961006C746E0053706500A3
:1059E00065656C006420200020204C005A6F69001F
:1059F0006F6D670053706800656574006420730004
:105A000020490A00646C0D0065200000526500000A
:105A10003220EF0083022000830150000500310096
:105A200043D22200008041001040BA000160EF0024
:105A30000000060040D222008381410080814100A5
:105A40001380BA00000006002020250020256400F5
:105A50006420200020202000202020002020200082
:105A6000202020002020200025642000202020006D
:105A700020202000202020002020200020202500A1
:105A80002564640020200A0020200D0020200A0048
:105A900020200D00202000003220EF0083D52200BE
:105AA000008041001040BA000160EF0000000600D5
:105AB0004A6F00007973000074690000636B000096
:105AC0002053000065740000757000003A0A000061
:105AD0000D0000003220EF00E3022000830150009F
:105AE0000500310063D82200008041001040BA0058
:105AF0000160EF000000060060D8220083814100B1
:105B0000808141001380BA00000006000A0D640085
:105B100020503A00616E2000205020006F7231004A
:105B200074202000446920007265320063742000F4
:105B3000696F20006E3A33002020200031202000C1
:105B40002032340020202000332020002034350073
:105B500020202000352020002036360020200A009A
:105B600053700D00656500003220EF0003DC220059
:105B7000008041001040BA000160EF000000060004
:105B80002020000020200000202000002020000015
:105B90002020000020200000202000002020000005
:105BA0002020000020200000200000003220EF0014
:105BB00023DE2200008041001040BA000160EF00A7
:105BC000000006002020000020200000202000000F
:105BD00020200000000000003220EF00E30220003F
:105BE000830150000500310083E022000080410065
:105BF0001040BA000160EF000000060080E02200C3
:105C000083814100808141001380BA0000000600BA
:105C10000D0A640054693A006C7420002050200082
:105C20006F723100742020004469200072653200D8
:105C300063742000696F20006E3A3300202020003A
:105C4000312020002032340020202000332020008A
:105C5000203435002020200035202000203636005A
:105C600020200A0053700D00656500003220EF000F
:105C7000E3022000830150000500310023E52200EB
:105C8000008041001040BA000160EF0000000600F3
:105C900020E5220083814100808141001380BA0009
:105CA000000006000D0A64005A6F3A006F6D200074
:105CB000205020006F7231007420200044692000C1
:105CC0007265320063742000696F20006E3A330001
:105CD000202020003120200020323400202020000D
:105CE00033202000203435002020200035202000E3
:105CF0002036360020200A0053700D006565000034
:105D00003220EF00C3E82200008041001040BA00BA
:105D10000160EF00000006000D0A00004E65000063
:105D200075740000726100006C2000005A6F000062
:105D30006E6500003A200000506100006E200000F7
:105D4000546900006C740000205A00006F6F00005E
:105D50006D0A00000D0000003220EF0083EB2200EE
:105D6000008041001040BA000160EF000000060012
:105D70002020000020200000202000002020000023
:105D8000202000002020000020200000202500000E
:105D9000327800002020000025320000782000002A
:105DA0002020000025320000780000003220EF00A3
:105DB00023EE2200008041001040BA000160EF0095
:105DC000000006000A0D000050720000657300001C
:105DD00065740000733A00000A0D00000A0D00000F
:105DE000000000003220EF00A302200083015000D9
:105DF00005003100E3F02200008041001040BA00AD
:105E00000160EF0000000600E0F022008381410005
:105E1000808141001380BA00000006004361200029
:105E20006D20200050725A0065206F004D6F6F008A
:105E300064656D006C20200020202000202046009A
:105E400020206F0020206300202075002020730098
:105E50002020200020202000506149006E20720088
:105E60002020690020207300546900006C74000039
:105E70003220EF0043F42200008041001040BA00BD
:105E80000160EF0000000600205B00004972000086
:105E9000697300002C4600006F63000075730000FA
:105EA0002C41000057420000202C0000424C000012
:105EB000432000005D0A00000D0A00000D000000F4
:105EC0003220EF00C3F62200008041001040BA00EB
:105ED0000160EF00000006004F6E0000202000006F
:105EE000200000003220EF00E3F722000080410094
:105EF0001040BA000160EF00000006004F6600008D
:105F000066200000200000003220EF0003F922008C
:105F1000008041001040BA000160EF000000060060
:105F20004F6E00000A0D0000000000003220EF005C
:105F300023FA2200008041001040BA000160EF0007
:105F4000000006004F660000660A00000D00000019
:105F50003220EF0043FB2200008041001040BA00D5
:105F60000160EF00000006000A0D00004361000020
:105F70006D2000004D6F0000646500006C0A000099
:105F80000D0000003220EF00E3FC22000080410001
:105F90001040BA000160EF0000000600202500005C
:105FA00064200000204E00006F20000043610000CC
:105FB0006D650000726100000A0D00000000000025
:105FC0003220EF00C3FE2200008041001040BA00E2
:105FD0000160EF000000060045450000507200001F
:105FE0006F6D000020440000756D0000703A0000E5
:105FF0000A0D0000000000003220EF0083002300A3
:10600000008041001040BA000160EF00000006006F
:1060100020200000202000002020000000000000C0
:106020003220EF00C3012300008041001040BA007D
:106030000160EF00000006000A0D00003E20000095
:1060400041570000423D00004F6E00000A0D000065
:106050003E200000000000003220EF0083032300F8
:10606000008041001040BA000160EF00000006000F
:106070000A0D00003E20000041570000423D000094
:106080004F660000660A00000D3E00002000000080
:106090003220EF0043052300008041001040BA0089
:1060A0000160EF00000006000A0D00003E20000025
:1060B000424C0000433D00004F6E00000A0D0000FE
:1060C0003E200000000000003220EF000307230004
:1060D000008041001040BA000160EF00000006009F
:1060E0000A0D00003E200000424C0000433D00002D
:1060F0004F660000660A00000D3E00002000000010
:106100003220EF00C3082300008041001040BA0095
:106110000160EF00000006000A0D000020500000A2
:10612000726F000067720000616D00002F50000068
:106130007265000076690000657700002069000044
:106140006E740000657200006C6100006365000001
:1061500072200000746F0000206F00006E0A0000C3
:106160000D0000003220EF00E30B2300008041000F
:106170001040BA000160EF00000006000A0D0000A8
:1061800020500000726F000067720000616D000017
:106190002F500000726500007669000065770000EE
:1061A000206900006E740000657200006C610000E0
:1061B0006365000072200000746F0000206F000013
:1061C000666600000A0D0000000000003220EF00AB
:1061D000230F2300008041001040BA000160EF004F
:1061E000000006000A0D00000A0D0000205000000B
:1061F000726F000067720000616D0000206900008E
:106200006E740000657200006C6100006365000040
:106210007220000069730000206F00006E0A000009
:106220000D0000003220EF00E31123000080410048
:106230001040BA000160EF00000006000A0D0000E7
:106240000A0D000020500000726F0000677200000D
:10625000616D0000206900006E740000657200002E
:106260006C6100006365000072200000697300002B
:10627000206F0000666600000A0D000000000000AC
:106280003220EF00C3142300008041001040BA0008
:106290000160EF0000000600205000007265000061
:1062A0007669000065770000206900006E740000C8
:1062B000657200006C6100006365000072200000E0
:1062C00069730000206F00006E0A00000D000000DE
:1062D0003220EF0043172300008041001040BA0035
:1062E0000160EF0000000600205000007265000011
:1062F0007669000065770000206900006E74000078
:10630000657200006C61000063650000722000008F
:1063100069730000206F0000666600000A0D00002F
:10632000000000003220EF00E3192300008041004C
:106330001040BA000160EF00000006000A0D0000E6
:106340000A0D0000204900006E760000616C00001C
:106350006964000020490000326300002041000011
:106360006464000072650000737300002028000060
:1063700025730000290A00000D0000003220EF0004
:10638000A31C2300008041001040BA000160EF0010
:10639000000006000A0D00000A0D00002049000060
:1063A0006E760000616C0000696400002049000006
:1063B000326300002052000065670000697300002E
:1063C0007465000072200000282500007329000079
:1063D0000A0D0000000000003220EF00E301200061
:1063E000830150000500310083202300008041001C
:1063F0001040BA000160EF0000000600802023007A
:1064000083814100808141001380BA0000000600B2
:106410000A0D65000A0D73005265700061646F001B
:1064200020496E0032437300204D650075783D00B1
:1064300020412500646432007265580073730A00BD
:106440003D250D0032580000205200003220EF00A0
:106450004302200083015000050031002324230063
:10646000008041001040BA000160EF00000006000B
:106470002024230083814100808141001380BA00E1
:10648000000006000A0D58000A0D20005265520057
:1064900061646500204973003243700020416F0041
:1064A00064646E0072657300737365003D253D0082
:1064B00032582500205232006567580069730A007F
:1064C00074650D00723D0000253200003220EF009F
:1064D00023272300008041001040BA000160EF0034
:1064E000000006004D750000782000005772000083
:1064F000697400006542000079740000653D000089
:10650000257500000A0D0000000000003220EF0099
:10651000C30120008301500005003100232A23001D
:10652000008041001040BA000160EF00000006004A
:10653000202A230083814100808141001380BA001A
:10654000000006000A0D58000A0D2C005772440086
:1065500069746100652074004932610063203D0068
:106560004D75250078203200416458006472200087
:1065700065730A00733D0D00253200003220EF00E4
:10658000030220008301500005003100A32D2300E9
:10659000008041001040BA000160EF0000000600DA
:1065A000A02D230083814100808141001380BA0027
:1065B000000006000A0D32000A0D580057722C0028
:1065C0006974440065206100416474006472610074
:1065D00065733D00733D250025323200582C58006C
:1065E0005265200067690A0073740D00657200002F
:1065F0003D2500003220EF00633023000080410081
:106600001040BA000160EF00000006000A0D000013
:106610000A0D0000204E00006F20000064610000A1
:10662000746100000A0D0000000000003220EF003D
:1066300023322300008041001040BA000160EF00C7
:10664000000006000A0D000053500000492D000014
:1066500057720000697400006520000025320000B8
:1066600078250000327800000A0D000000000000CC
:106670003220EF0043342300008041001040BA0074
:106680000160EF00000006000A0D000045720000E6
:10669000726F0000722D0000204900007269000036
:1066A00073200000696E0000204100007574000036
:1066B0006F2000004D6F0000646500000A0D0000AF
:1066C000000000003220EF00E3362300008041008C
:1066D0001040BA000160EF0000000600202000001A
:1066E000204900007269000073200000436F000021
:1066F0006D6D0000616E000064200000466F0000B8
:10670000726D0000617400000A0D000000000000BE
:106710003220EF0043392300008041001040BA00CE
:106720000160EF000000060020200000204900006A
:10673000726900007320000041750000746F000052
:1067400028630000722900002C200000497200001C
:1067500069730000204D0000616E0000756100004B
:106760006C28000063720000290A00000D00000080
:106770003220EF00433C2300008041001040BA006B
:106780000160EF000000060020200000204900000A
:106790007269000073200000557000002C34000066
:1067A00028630000722900002C20000049720000BC
:1067B00069730000204400006F7700006E2C000019
:1067C0003428000063720000290A00000D00000058
:1067D0003220EF00433F2300008041001040BA0008
:1067E0000160EF00000006002020000020490000AA
:1067F0007269000073200000257500000000000091
:106800003220EF00C3402300008041001040BA0056
:106810000160EF00000006000A0D00003E200000AD
:1068200044690000616700003D4F00006E0A0000EF
:106830000D3E0000200000003220EF0083422300C4
:10684000008041001040BA000160EF000000060027
:106850000A0D00003E20000044690000616700004E
:106860003D4F0000666600000A0D00003E2000005B
:10687000000000003220EF0063442300008041004C
:106880001040BA000160EF00000006000A0D000091
:106890003E200000506F000077650000723D000050
:1068A0004F6E00000A0D00003E20000000000000B6
:1068B0003220EF0043462300008041001040BA0020
:1068C0000160EF00000006000A0D00003E200000FD
:1068D000506F000077650000723D00004F660000B9
:1068E000660A00000D3E0000200000003220EF008C
:1068F00023482300008041001040BA000160EF00EF
:10690000000006000A0D00003E2000005344000075
:1069100069610000673D00004F6E00000A0D000035
:106920003E200000000000003220EF00034A230058
:10693000008041001040BA000160EF000000060036
:106940000A0D00003E200000534400006961000071
:10695000673D00004F660000660A00000D3E000023
:10696000200000003220EF00E34B230000804100B4
:106970001040BA000160EF00000006000A0D0000A0
:106980003E200000546100006C6C0000793D000066
:10699000416300007469000076650000204C00002F
:1069A0006F7700000A0D00003E200000000000008C
:1069B0003220EF00434E2300008041001040BA0017
:1069C0000160EF00000006000A0D00003E200000FC
:1069D000546100006C6C0000793D000041630000D0
:1069E0007469000076650000204300006C6F0000B1
:1069F000736500000A0D00003E200000000000004A
:106A00003220EF00C3502300008041001040BA0044
:106A10000160EF00000006000A0D00003E200000AB
:106A2000546100006C6C0000793D0000416300007F
:106A30007469000076650000204800006967000066
:106A4000680A00000D3E0000200000003220EF0028
:106A500023532300008041001040BA000160EF0082
:106A6000000006000A0D00003E20000054610000F6
:106A70006C6C0000793D0000416300007469000007
:106A800076650000204F0000706500006E0A00006F
:106A90000D3E0000200000003220EF00835523004F
:106AA000008041001040BA000160EF0000000600C5
:106AB00045720000726F0000722D00002046000039
:106AC0006F63000075730000206900006E200000F5
:106AD00041750000746F0000204D00006F640000DD
:106AE000650A00000D0000003220EF00035823006B
:106AF000008041001040BA000160EF000000060075
:106B000020200000204600006F6300007573000025
:106B1000204300006F6D00006D6100006E64000096
:106B2000204600006F7200006D610000740A0000D2
:106B30000D0000003220EF00635A23000080410066
:106B40001040BA000160EF000000060020200000A5
:106B5000204600006F6300007573000020410000B4
:106B6000757400006F28000063720000292C00007B
:106B700020200000204600006F63000075730000B5
:106B8000204D0000616E0000756100006C2800005F
:106B900063720000290A00000D0000003220EF009F
:106BA000A35D2300008041001040BA000160EF00A7
:106BB0000000060020200000204600006F63000057
:106BC0007573000020550000702C00003428000070
:106BD00063720000292C00002020000020460000E5
:106BE0006F63000075730000204400006F770000A1
:106BF0006E2C00003428000063720000290A000097
:106C00000D0000003220EF00C3012000830150007E
:106C100005003100E3612300008041001040BA000C
:106C20000160EF0000000600E06123008381410065
:106C3000808141001380BA000000060020206F0010
:106C4000204677006F636E0075732C00205530006E
:106C5000702C6100306130003028280063726300BE
:106C6000292C7200204629006F630A0075730D00FD
:106C7000204400003220EF006364230000804100C4
:106C80001040BA000160EF00000006002020000064
:106C9000204600006F63000075730000202500008F
:106CA000750000003220EF00E36523000080410002
:106CB0001040BA000160EF00000006000A0D00005D
:106CC0003E200000436100006D650000726100001D
:106CD00020250000642000004E6F0000742000009A
:106CE00061760000616900006C610000626C000068
:106CF000650A00000D3E0000200000003220EF0079
:106D0000A3682300008041001040BA000160EF003A
:106D1000000006000A0D00003E200000537700002E
:106D20004D6F0000646500003D4400007561000087
:106D30006C0A00000D3E0000200000003220EF0031
:106D4000A36A2300008041001040BA000160EF00F8
:106D5000000006000A0D00003E20000053770000EE
:106D60004D6F0000646500003D530000696E000037
:106D7000676C0000650A00000D3E00002000000066
:106D80003220EF00C36C2300008041001040BA00A5
:106D90000160EF0000000600333A00005049000097
:106DA000502000004C6F000077650000722000004A
:106DB0005269000067680000740000003220EF0094
:106DC000A36E2300008041001040BA000160EF0074
:106DD00000000600343A0000504900005020000036
:106DE00055700000706500007220000052690000BC
:106DF00067680000740000003220EF0083702300F9
:106E0000008041001040BA000160EF000000060061
:106E1000323A000050490000502000004C6F000042
:106E200077650000722000004C6500006674000069
:106E3000000000003220EF00637223000080410058
:106E40001040BA000160EF0000000600313A000077
:106E5000504900005020000055700000706500008F
:106E6000722000004C650000667400000000000005
:106E70003220EF0043742300008041001040BA002C
:106E80000160EF0000000600203A00004E6F000095
:106E90006E65000020530000656C00006563000013
:106EA00074650000640000003220EF0003762300C8
:106EB000008041001040BA000160EF0000000600B1
:106EC0000A0D00003E20000050690000704C0000D8
:106ED0006F6300003D250000732C0000205300006C
:106EE000697A0000653D0000257300000A0D00006E
:106EF0003E200000000000003220EF0083782300D5
:106F0000008041001040BA000160EF000000060060
:106F100025750000302000005065000072630000FD
:106F2000656E0000740000003220EF00037A230039
:106F3000008041001040BA000160EF000000060030
:106F4000467500006C6C0000000000003220EF006D
:106F5000237B2300008041001040BA000160EF0055
:106F6000000006000A0D00003E2000004C730000E7
:106F700067440000656E00003D250000730A0000B4
:106F80000D3E0000200000003220EF00037D2300B2
:106F9000008041001040BA000160EF0000000600D0
:106FA0000A0D00003E2000007363000053790000CA
:106FB000734D00006F6400003D41000075740000D7
:106FC0006F0A00000D3E0000200000003220EF009C
:106FD000237F2300008041001040BA000160EF00D1
:106FE000000006000A0D00003E2000007363000050
:106FF00053790000734D00006F6400003D4D0000A8
:10700000616E0000756100006C0A00000D3E00001A
:10701000200000003220EF00638123000080410047
:107020001040BA000160EF0000000600313100009E
:107030003A4300006F7200006E650000722000008D
:107040004C5200003E5500004C0000003220EF0082
:1070500023832300008041001040BA000160EF004C
:1070600000000600203600003A570000697000005A
:10707000652000004C3E0000520000003220EF006E
:10708000A3842300008041001040BA000160EF009B
:1070900000000600203300003A4300006F72000039
:1070A0006E65000072200000554C00003E4C000050
:1070B000520000003220EF00638623000080410070
:1070C0001040BA000160EF000000060031300000FF
:1070D0003A5700006970000065200000426F000010
:1070E000743E0000546F0000700000003220EF007A
:1070F00023882300008041001040BA000160EF00A7
:1071000000000600203700003A57000069700000B8
:1071100065200000436500006E7400006572000089
:10712000203E00004F750000740000003220EF0088
:10713000238A2300008041001040BA000160EF0064
:1071400000000600203400003A570000697000007B
:1071500065200000546F0000703E0000426F000088
:10716000740000003220EF00E38B23000080410018
:107170001040BA000160EF00000006002038000057
:107180003A5700006970000065200000523E000080
:107190004C0000003220EF00638D2300008041008E
:1071A0001040BA000160EF0000000600203500002A
:1071B0003A4300006F7200006E650000722000000C
:1071C000555200003E4C00004C0000003220EF0001
:1071D000238F2300008041001040BA000160EF00BF
:1071E00000000600202000003A4E00006F6E0000F4
:1071F00065200000536500006C65000063740000AA
:1072000065640000000000003220EF0003912300BD
:10721000008041001040BA000160EF00000006004D
:107220000A0D00003E200000576900007065000054
:10723000536500006C3D0000257300000A0D00003E
:107240003E200000000000003220EF0003932300E6
:10725000008041001040BA000160EF00000006000D
:107260000A0D00003E200000496400006C6500002B
:10727000527400006E3D00002564000020530000A1
:10728000656300006F6E0000647300000A0D00006B
:107290003E200000000000003220EF008395230014
:1072A000008041001040BA000160EF0000000600BD
:1072B0000A0D00003E2000004A500000616E0000F0
:1072C00053700000643A0000205000006F7200000C
:1072D0007420000020310000202000003220000037
:1072E0002033000020200000342000002035000062
:1072F00020200000360A00000D0000003220EF00C0
:10730000E30120008301500005003100A399230010
:10731000008041001040BA000160EF00000006004C
:10732000A099230083814100808141001380BA002D
:1073300000000600202064002020200020202500DE
:107340002020320020206400202020002020250062
:10735000202032002532640064200A0025320D000E
:1073600064203E0025320000642000002532000029
:107370003220EF00439C2300008041001040BA00FF
:107380000160EF00000006000D0A00003E4A000008
:10739000506100006E44000069720000202000006F
:1073A000446900007265000063740000696F0000AA
:1073B0006E3A00002031000020320000203300002F
:1073C0002034000020350000203600000A0D0000A7
:1073D000000000003220EF00C301200083015000B4
:1073E0000500310063A02300008041001040BA0076
:1073F0000160EF000000060060A0230083814100CF
:10740000808141001380BA00000006002020630044
:1074100020202000202025002020630020202000A4
:10742000202025002020630020202000202025008F
:107430002020630020250A0063200D0025633E0004
:10744000202500003220EF00E3A22300008041004D
:107450001040BA000160EF00000006000A0D0000B5
:107460003E2000004C73000067530000697A000062
:10747000653D0000257300000A0D00003E2000005D
:10748000000000003220EF00E3A423000080410050
:107490001040BA000160EF00000006000A0D000075
:1074A0003E200000506100006E5300007065000037
:1074B000656400003D250000640A00000D3E0000E8
:1074C000200000003220EF00E3A6230000804100EE
:1074D0001040BA000160EF00000006000A0D000035
:1074E0003E2000004A5A00006F6F00006D530000FC
:1074F000706400003A200000506F000072740000B9
:107500002020000031200000203200002020000058
:10751000332000002034000020200000352000002F
:10752000203600000A0D0000000000003220EF00AD
:10753000E3012000830150000500310023AB23004C
:10754000008041001040BA000160EF00000006001A
:1075500020AB230083814100808141001380BA0069
:10756000000006002020320020206400202020009F
:107570002020250020203200202064002020200030
:1075800020202500202532003264640020250A00D6
:1075900032640D0020253E003264000020250000EA
:1075A0003220EF00C3AD2300008041001040BA003C
:1075B0000160EF00000006000D0A00003E4A0000D6
:1075C0005A6F00006F6D00004469000072200000D7
:1075D00020440000697200006563000074690000C7
:1075E0006F6E00003A2000003120000032200000C1
:1075F000332000003420000035200000360A00004F
:107600000D0000003220EF00E30120008301500054
:1076100005003100E3B12300008041001040BA00B2
:107620000160EF0000000600E0B12300838141000B
:10763000808141001380BA00000006002020200055
:10764000202025002020630020202000202025006D
:10765000202063002020200020202500202063001F
:1076600020200A0020200D0025633E002025000078
:1076700063200000256300003220EF0083B4230064
:10768000008041001040BA000160EF0000000600D9
:107690000D0A00003E4A0000546900006C740000AE
:1076A000446900007220000020440000697200005C
:1076B00065630000746900006F6E00003A200000EE
:1076C0003120000032200000332000003420000070
:1076D00035200000360A00000D0000003220EF00C7
:1076E000A3B72300008041001040BA000160EF0002
:1076F000000006000A0D00003E2000004A54000071
:10770000696C000074530000706400003A200000AF
:10771000506F000072740000202000003120000033
:107720002032000020200000332000002034000020
:107730002020000035200000203600000A0D000047
:10774000000000003220EF00E30120008301500020
:1077500005003100E3BB2300008041001040BA0067
:107760000160EF0000000600E0BB230083814100C0
:10777000808141001380BA00000006002020320002
:10778000202064002020200020202500202032001E
:1077900020206400202020002020250020256400D7
:1077A00032640A0020250D0032643E0020250000CE
:1077B00032640000202500003220EF00C3012000C9
:1077C000830150000500310083BF23000080410089
:1077D0001040BA000160EF000000060080BF2300E7
:1077E00083814100808141001380BA0000000600BF
:1077F0000A0D64003E202C00496420006C655A008C
:107800005A6F6F006E656F003A206D0050613D0049
:107810006E3D2500256464002C200A0054690D008B
:107820006C743E003D2500003220EF0003C22300AF
:10783000008041001040BA000160EF000000060027
:107840000A0D00003E200000546900006C74000026
:107850005370000065650000643D00002564000071
:107860000A0D00003E200000000000003220EF0062
:1078700023C42300008041001040BA000160EF00E3
:10788000000006000A0D00003E2000005A6F0000B4
:107890006F6D00005370000065650000643D0000DE
:1078A000256400000A0D00003E20000000000000DA
:1078B0003220EF0043C62300008041001040BA0090
:1078C0000160EF00000006000A0D00003E200000ED
:1078D000436100006D4600006F6C000050720000B4
:1078E000763D0000456E0000616200006C6500009E
:1078F000640A00000D3E0000200000003220EF006E
:10790000A3C82300008041001040BA000160EF00CE
:10791000000006000A0D00003E2000004361000048
:107920006D4600006F6C000050720000763D000054
:107930004469000073610000626C0000656400002F
:107940000A0D00003E200000000000003220EF0081
:1079500023CB2300008041001040BA000160EF00FB
:10796000000006004F6E000020430000616D000023
:107970006572000061200000496E0000697400001B
:107980002C200000736500006E6400002048000099
:107990006F6D000065200000636F00006D6D0000DA
:1079A000616E0000640A00000D3E0000200000002F
:1079B0003220EF0043022000830150000500310017
:1079C00043CF2300008041001040BA000160EF0067
:1079D0000000060040CF23008381410080814100E8
:1079E0001380BA00000006004F6E6E002043640052
:1079F000616D20006572730061206500496E710041
:107A0000697475002C20650073656E006E646300F8
:107A10002050650072650A0073650D0074203E00F9
:107A200031322000206300006F6D00006D610000A6
:107A30003220EF0043D22300008041001040BA0002
:107A40000160EF00000006000A0D00003E2000006B
:107A50005072000065730000657400004C6F0000F8
:107A6000633D000036200000496E000043610000C5
:107A70006D200000362000004C6F000063610000A4
:107A80006C0A00000D3E0000200000003220EF00D4
:107A900023D52300008041001040BA000160EF00B0
:107AA000000006000A0D00003E2000005072000099
:107AB00065730000657400004C6F0000633D0000BA
:107AC000416C00006C2000004C6F000063610000FE
:107AD0006C0A00000D3E0000200000003220EF0084
:107AE000A3D72300008041001040BA000160EF00DE
:107AF000000006002F6E00002F7200000000000042
:107B00003220EF00C3D82300008041001040BA00AB
:107B10000160EF00000006000A0D00003E53000067
:107B2000657400004465000066610000756C00002B
:107B30007420000025640000200A00000D3E0000B3
:107B4000200000003220EF00E3DA23000080410033
:107B50001040BA000160EF00000006000A0D0000AE
:107B60003E44000065660000617500006C74000012
:107B7000436100006D20000025640000200A000021
:107B80000D3E0000200000003220EF0003DD230046
:107B9000008041001040BA000160EF0000000600C4
:107BA0000A0D00003E2000004578000074540000DB
:107BB0007269000067670000657200003D310000D7
:107BC00032200000436100006D3100002C200000D5
:107BD00030200000436100006D3200000A0D0000FB
:107BE0003E200000000000003220EF0003E02300F0
:107BF000008041001040BA000160EF000000060064
:107C00000A0D00003E20000045780000745400007A
:107C10007269000067670000657200003D36000071
:107C200020430000616D0000312C00002036000070
:107C300020430000616D0000320A00000D3E00008C
:107C4000200000003220EF00E3E22300008041002A
:107C50001040BA000160EF00000006000A0D0000AD
:107C60003E2000005365000072690000616C000056
:107C700045630000686F00003D4500006E61000034
:107C8000626C0000656400000A0D00003E200000E8
:107C9000000000003220EF0063E523000080410077
:107CA0001040BA000160EF00000006000A0D00005D
:107CB0003E2000005365000072690000616C000006
:107CC00045630000686F00003D44000069730000D8
:107CD000616200006C650000640A00000D3E000057
:107CE000200000003220EF00E3E723000080410085
:107CF0001040BA000160EF00000006000A0D00000D
:107D00003E2000005365000072690000616C0000B5
:107D1000496E0000666F00003D4500006E61000086
:107D2000626C0000656400000A0D00003E20000047
:107D3000000000003220EF0063EA230000804100D1
:107D40001040BA000160EF00000006000A0D0000BC
:107D50003E2000005365000072690000616C000065
:107D6000496E0000666F00003D440000697300002A
:107D7000616200006C650000640A00000D3E0000B6
:107D8000200000003220EF00E3EC230000804100DF
:107D90001040BA000160EF00000006000A0D00006C
:107DA000416C00006C20000044650000636F00001F
:107DB0006465000072730000206C00006F610000B9
:107DC00064650000640A00000D0000003220EF002E
:107DD00023EF2300008041001040BA000160EF0053
:107DE000000006000A0D0000496E000070750000DA
:107DF00074200000257500003A20000020000000DB
:107E00003220EF00C3F02300008041001040BA0090
:107E10000160EF0000000600313000003830000043
:107E20007020000028350000392E00003934000091
:107E30002920000044650000636F000064650000B5
:107E400072200000436F00006E660000696700004A
:107E5000204400006F6E0000650A00000D00000065
:107E60003220EF00C3F32300008041001040BA002D
:107E70000160EF00000006003130000038300000E3
:107E80007020000028350000302900002044000048
:107E9000656300006F64000065720000204300000D
:107EA0006F6E00006669000067200000446F0000EC
:107EB0006E6500000A0D0000000000003220EF0097
:107EC000A3F62300008041001040BA000160EF00DB
:107ED000000006003130000038300000692000004A
:107EE00028350000392E0000393400002920000018
:107EF00044650000636F00006465000072200000AC
:107F0000436F00006E6600006967000020440000B7
:107F10006F6E0000650A00000D0000003220EF00C7
:107F2000A3F92300008041001040BA000160EF0077
:107F300000000600313000003830000069200000E9
:107F4000283500003029000020440000656300004F
:107F50006F64000065720000204300006F6E000037
:107F60006669000067200000446F00006E65000035
:107F70000A0D0000000000003220EF0083FC230007
:107F8000008041001040BA000160EF0000000600D0
:107F9000373200003070000028350000392E000014
:107FA000393400002920000044650000636F0000A0
:107FB0006465000072200000436F00006E660000E0
:107FC00069670000204400006F6E0000650A000031
:107FD0000D0000003220EF0063FF2300008041000D
:107FE0001040BA000160EF000000060037320000C8
:107FF00030700000283500003029000020440000C7
:10800000656300006F64000065720000204300009B
:108010006F6E00006669000067200000446F00007A
:108020006E6500000A0D0000000000003220EF0025
:1080300023022400008041001040BA000160EF00DC
:1080400000000600363400003020000078200000D8
:1080500034380000302800003630000029200000AD
:10806000456E0000636F0000646500007220000030
:10807000436F00006E660000696700002044000046
:108080006F6E0000650A00000D0000003220EF0056
:1080900023052400008041001040BA000160EF0079
:1080A0000000060036340000302000007820000078
:1080B0003438000030280000373500002920000047
:1080C00044650000636F00006465000072200000DA
:1080D000436F00006E6600006967000020440000E6
:1080E0006F6E0000650A00000D0000003220EF00F6
:1080F00023082400008041001040BA000160EF0016
:108100000000060038300000302000007820000019
:1081100036300000302800003630000029200000F2
:1081200044650000636F0000646500007220000079
:10813000436F00006E660000696700002044000085
:108140006F6E0000650A00000D0000003220EF0095
:10815000230B2400008041001040BA000160EF00B2
:1081600000000600313000003234000020780000AA
:108170002037000036380000283600003029000083
:1081800020440000656300006F6400006572000019
:10819000204300006F6E0000666900006720000049
:1081A000446F00006E6500000A0D00000000000032
:1081B0003220EF00430E2400008041001040BA003E
:1081C0000160EF0000000600313000003234000092
:1081D00020780000203700003638000028370000E3
:1081E0003529000020440000656300006F64000032
:1081F00065720000204300006F6E00006669000099
:1082000067200000446F00006E6500000A0D00004A
:10821000000000003220EF006311240000804100C4
:108220001040BA000160EF0000000600313200008B
:10823000383000002078000020310000303200008B
:10824000342800003630000029200000446500007A
:10825000636F00006465000072200000436F00003F
:108260006E66000069670000204400006F6E000029
:10827000650A00000D0000003220EF008314240086
:10828000008041001040BA000160EF0000000600CD
:108290003132000038300000207800002037000024
:1082A0003638000028360000302900002044000045
:1082B000656300006F6400006572000020430000E9
:1082C0006F6E00006669000067200000446F0000C8
:1082D0006E6500000A0D0000000000003220EF0073
:1082E000A3172400008041001040BA000160EF0095
:1082F0000000060031330000363600002078000010
:1083000020370000363800002836000030290000F1
:1083100020440000656300006F6400006572000087
:10832000204300006F6E00006669000067200000B7
:10833000446F00006E6500000A0D000000000000A0
:108340003220EF00C31A2400008041001040BA0020
:108350000160EF0000000600313400003030000002
:108360002078000020310000303500003028000067
:10837000363000002920000044650000636F0000D3
:108380006465000072200000436F00006E6600000C
:1083900069670000204400006F6E0000650A00005D
:1083A0000D0000003220EF00E31D2400008041009A
:1083B0001040BA000160EF000000060031360000F6
:1083C0003030000020780000203100003230000002
:1083D00030280000363000002920000044650000ED
:1083E000636F00006465000072200000436F0000AE
:1083F0006E66000069670000204400006F6E000098
:10840000650A00000D0000003220EF000321240067
:10841000008041001040BA000160EF00000006003B
:108420003139000032300000207800002031000097
:1084300032300000302000002836000030480000B4
:108440007A2900002D2000004E4F0000542000002B
:1084500073750000707000006F720000746500009A
:10846000640A00000D0000003220EF000324240005
:10847000008041001040BA000160EF0000000600DB
:1084800053440000204E00005453000043200000DD
:1084900028200000532D000056690000646500008C
:1084A0006F29000020440000656300006F64000035
:1084B00065720000204300006F6E000066690000D6
:1084C00067200000446F00006E6500000A0D000088
:1084D000000000003220EF006327240000804100EC
:1084E0001040BA000160EF00000006005344000095
:1084F00020500000414C00002020000028530000C4
:108500002D56000069640000656F000029200000FE
:1085100044650000636F0000646500007220000085
:10852000436F00006E660000696700002044000091
:108530006F6E0000650A00000D0000003220EF00A1
:10854000E30120008301500005003100A32B24002B
:10855000008041001040BA000160EF0000000600FA
:10856000A02B240083814100808141001380BA0048
:10857000000006005344430020206F004E546E005C
:108580005343660020286900204367006F6D200078
:10859000706F440073696F0074656E002920650078
:1085A00044650A00636F0D006465000072200000DE
:1085B0003220EF00C301200083015000050031008C
:1085C000432F2400008041001040BA000160EF00FA
:1085D00000000600402F240083814100808141007B
:1085E0001380BA00000006005344430020506F007F
:1085F000414C6E0020286600204369006F6D6700C3
:10860000706F20007369440074656F0029206E004C
:1086100044656500636F0A0064650D007220000008
:108620003220EF00C3312400008041001040BA0026
:108630000160EF0000000600556E00006B6E000048
:108640006F7700006E0A00000D0000003220EF007E
:1086500023332400008041001040BA000160EF0085
:10866000000006000A0D0000416C00006C200000B4
:10867000456E0000636F00006465000072730000C7
:10868000206C00006F61000064650000640A000057
:108690000D0000003220EF0063352400008041000F
:1086A0001040BA000160EF00000006000A0D000053
:1086B000504700004D3A0000200000003220EF003B
:1086C000A3362400008041001040BA000160EF0092
:1086D000000006000A0D000050520000453A00005C
:1086E000200000003220EF00E3372400008041002A
:1086F0001040BA000160EF000000060031300000B9
:10870000383000007020000028350000392E0000AD
:108710003934000029200000456E0000636F00001E
:108720006465000072200000436F00006E66000068
:1087300069670000204400006F6E0000650A0000B9
:108740000D0000003220EF00E33A240000804100D9
:108750001040BA000160EF00000006003130000058
:10876000383000007020000028350000302900005B
:10877000204500006E6300006F6400006572000019
:10878000204300006F6E0000666900006720000053
:10879000446F00006E6500000A0D0000000000003C
:1087A0003220EF00C33D2400008041001040BA0099
:1087B0000160EF000000060031300000383000009A
:1087C0006920000028350000392E000039340000EF
:1087D00029200000456E0000636F00006465000002
:1087E00072200000436F00006E66000069670000A1
:1087F000204400006F6E0000650A00000D000000BC
:108800003220EF00C3402400008041001040BA0035
:108810000160EF0000000600313000003830000039
:1088200069200000283500003029000020450000A4
:108830006E6300006F64000065720000204300005A
:108840006F6E00006669000067200000446F000042
:108850006E6500000A0D0000000000003220EF00ED
:10886000A3432400008041001040BA000160EF00E3
:10887000000006003732000030700000283500008C
:10888000392E00003934000029200000456E000018
:10889000636F00006465000072200000436F0000F9
:1088A0006E66000069670000204400006F6E0000E3
:1088B000650A00000D0000003220EF00834624000E
:1088C000008041001040BA000160EF000000060087
:1088D00037320000307000002835000030290000D9
:1088E000204500006E6300006F64000065720000A8
:1088F000204300006F6E00006669000067200000E2
:10890000446F00006E6500000A0D000000000000CA
:108910003220EF0043492400008041001040BA009B
:108920000160EF0000000600363400003020000037
:10893000782000003438000030280000373500006F
:1089400029200000456E0000636F00006465000090
:1089500072200000436F00006E660000696700002F
:10896000204400006F6E0000650A00000D0000004A
:108970003220EF00434C2400008041001040BA0038
:108980000160EF00000006003830000030200000D9
:10899000782000003630000030280000363000001B
:1089A00029200000456E0000636F00006465000030
:1089B00072200000436F00006E66000069670000CF
:1089C000204400006F6E0000650A00000D000000EA
:1089D0003220EF00434F2400008041001040BA00D5
:1089E0000160EF000000060031300000323400006A
:1089F00020780000203700003638000028360000BC
:108A000030290000204500006E6300006F64000004
:108A100065720000204300006F6E00006669000070
:108A200067200000446F00006E6500000A0D000022
:108A3000000000003220EF0063522400008041005B
:108A40001040BA000160EF00000006003130000065
:108A50003234000020780000203700003638000053
:108A60002837000035290000204500006E63000013
:108A70006F64000065720000204300006F6E00000C
:108A80006669000067200000446F00006E6500000A
:108A90000A0D0000000000003220EF008355240082
:108AA000008041001040BA000160EF0000000600A5
:108AB0003132000038300000207800002031000002
:108AC0003032000034280000363000002920000039
:108AD000456E0000636F00006465000072200000B6
:108AE000436F00006E6600006967000020440000CC
:108AF0006F6E0000650A00000D0000003220EF00DC
:108B0000A3582400008041001040BA000160EF002B
:108B100000000600313200003830000020780000EC
:108B200020370000363800002836000030290000C9
:108B3000204500006E6300006F6400006572000055
:108B4000204300006F6E000066690000672000008F
:108B5000446F00006E6500000A0D00000000000078
:108B60003220EF00C35B2400008041001040BA00B7
:108B70000160EF00000006003133000036360000CF
:108B8000207800002037000036380000283600002A
:108B900030290000204500006E6300006F64000073
:108BA00065720000204300006F6E000066690000DF
:108BB00067200000446F00006E6500000A0D000091
:108BC000000000003220EF00E35E2400008041003E
:108BD0001040BA000160EF000000060031340000D0
:108BE00030300000207800002031000030350000D7
:108BF000302800003630000029200000456E0000BB
:108C0000636F00006465000072200000436F000085
:108C10006E66000069670000204400006F6E00006F
:108C2000650A00000D0000003220EF0003622400FE
:108C3000008041001040BA000160EF000000060013
:108C40003136000030300000207800002031000074
:108C500032300000302800003630000029200000AB
:108C6000456E0000636F0000646500007220000024
:108C7000436F00006E66000069670000204400003A
:108C80006F6E0000650A00000D0000003220EF004A
:108C900023652400008041001040BA000160EF000D
:108CA000000006003139000032300000207800005A
:108CB0002031000032300000302800003630000043
:108CC00029200000456E0000636F0000646500000D
:108CD00072200000436F00006E66000069670000AC
:108CE000204400006F6E0000650A00000D000000C7
:108CF0003220EF00E3012000830150000500310025
:108D000043692400008041001040BA000160EF0078
:108D100000000600406924008381410080814100F9
:108D20001380BA000000060053444300202D6F005A
:108D300020376E00323066002078690020346700EA
:108D400038302000202844004E546F0053436E00FA
:108D500029206500456E0A00636F0D006465000000
:108D6000722000003220EF00E36B240000804100FD
:108D70001040BA000160EF000000060053440000FC
:108D80002037000036380000207800002035000031
:108D90003736000020280000504100004C29000018
:108DA000204500006E6300006F64000065720000E3
:108DB000204300006F6E000066690000672000001D
:108DC000446F00006E6500000A0D00000000000006
:108DD0003220EF00436F2400008041001040BA00B1
:108DE0000160EF00000006003130000025000000A7
:108DF0003220EF0043702400008041001040BA0090
:108E00000160EF0000000600323000002500000085
:108E10003220EF0043712400008041001040BA006E
:108E20000160EF0000000600333000002500000064
:108E30003220EF0043722400008041001040BA004D
:108E40000160EF0000000600343000002500000043
:108E50003220EF0043732400008041001040BA002C
:108E60000160EF0000000600353000002500000022
:108E70003220EF0043742400008041001040BA000B
:108E80000160EF0000000600363000002500000001
:108E90003220EF0043752400008041001040BA00EA
:108EA0000160EF00000006003730000025000000E0
:108EB0003220EF0043762400008041001040BA00C9
:108EC0000160EF00000006003830000025000000BF
:108ED0003220EF0043772400008041001040BA00A8
:108EE0000160EF000000060039300000250000009E
:108EF0003220EF0043782400008041001040BA0087
:108F00000160EF00000006004E6F0000200000002E
:108F10003220EF0043792400008041001040BA0065
:108F20000160EF00000006004D640000000000003A
:108F30003220EF00437A2400008041001040BA0044
:108F40000160EF00000006004C6700000000000018
:108F50003220EF00437B2400008041001040BA0023
:108F60000160EF00000006004D78000000000000E6
:108F70003220EF00437C2400008041001040BA0002
:108F80000160EF0000000600536D000000000000CB
:108F90003220EF00437D2400008041001040BA00E1
:108FA0000160EF00000006004C530000473A00004B
:108FB000733A0000257300002C5400003A2500008D
:108FC000730000003220EF00E37E240000804100A7
:108FD0001040BA000160EF00000006004C53000092
:108FE000472D0000504700004D3A0000733A000042
:108FF000257300002C5400003A2500007300000087
:109000003220EF00C3802400008041001040BA00ED
:109010000160EF00000006004C530000472D0000E7
:1090200050520000453A0000733A000025730000DA
:109030002C5400003A250000730000003220EF009D
:10904000A3822400008041001040BA000160EF00BC
:10905000000006004C530000473A0000204F00007B
:1090600066660000000000003220EF000384240048
:10907000008041001040BA000160EF0000000600CF
:109080004C530000472D0000504700004D3A0000AF
:10909000204F000066660000000000003220EF0054
:1090A000A3852400008041001040BA000160EF0059
:1090B000000006004C530000472D000050520000F5
:1090C000453A0000204F00006666000000000000E6
:1090D0003220EF0043872400008041001040BA0096
:1090E0000160EF00000006004C4C00000000000092
:1090F0003220EF0043882400008041001040BA0075
:109100000160EF0000000600555200000000000062
:109110003220EF0043892400008041001040BA0053
:109120000160EF00000006004C520000000000004B
:109130003220EF00438A2400008041001040BA0032
:109140000160EF0000000600554C00000000000028
:109150003220EF00438B2400008041001040BA0011
:109160000160EF000000060050490000503A000086
:1091700020250000732C00004C2000002573000007
:10918000000000003220EF00E38C2400008041004A
:109190001040BA000160EF000000060050490000D6
:1091A000502D0000504700004D3A000020250000DF
:1091B000732C00004C20000025730000000000000C
:1091C0003220EF00C38E2400008041001040BA001E
:1091D0000160EF000000060050490000502D000023
:1091E00050520000453A000020250000732C00007A
:1091F0004C20000025730000000000003220EF002A
:10920000A3902400008041001040BA000160EF00EC
:109210000000060050490000503A0000204F0000B6
:1092200066660000000000003220EF000392240078
:10923000008041001040BA000160EF00000006000D
:1092400050490000502D0000504700004D3A0000EA
:10925000204F000066660000000000003220EF0092
:10926000A3932400008041001040BA000160EF0089
:109270000000060050490000502D00005052000030
:10928000453A0000204F0000666600000000000024
:109290003220EF0043952400008041001040BA00C6
:1092A0000160EF0000000600507200006F670000D0
:1092B00020250000750A00000D0000003220EF009C
:1092C000A3962400008041001040BA000160EF0026
:1092D00000000600546100006B6500000A0D0000EC
:1092E000000000003220EF00E397240000804100DE
:1092F0001040BA000160EF0000000600507200004C
:109300006576000020250000750A00000D000000B1
:109310003220EF0043992400008041001040BA0041
:109320000160EF000000060050720000706700004E
:1093300020250000750A00000D0000003220EF001B
:10934000A39A2400008041001040BA000160EF00A1
:10935000000006000A0D0000504700004D280000E4
:10936000772900003A200000000000003220EF00C2
:10937000239C2400008041001040BA000160EF00EF
:10938000000006000A0D00005052000045280000B1
:10939000772900003A200000000000003220EF0092
:1093A000A39D2400008041001040BA000160EF003E
:1093B000000006000A0D0000504700004D28000084
:1093C000722900003A200000000000003220EF0067
:1093D000239F2400008041001040BA000160EF008C
:1093E000000006000A0D0000505200004528000051
:1093F000722900003A200000000000003220EF0037
:10940000A3A02400008041001040BA000160EF00DA
:10941000000006005772000069740000652000001B
:10942000254C0000580A00000D0000003220EF001B
:1094300023A22400008041001040BA000160EF0028
:1094400000000600577200006974000065200000EB
:10945000254C0000582C00002052000065610000DF
:1094600064200000254C0000580A00000D00000098
:109470003220EF0043A42400008041001040BA00D5
:109480000160EF00000006002020000020530000D3
:1094900059530000544500004D2000004D45000088
:1094A0004E55000020200000202000000000000099
:1094B0003220EF0043A62400008041001040BA0093
:1094C0000160EF0000000600202000002053000093
:1094D00065720000696100006C200000496E0000A8
:1094E00070750000742000002020000000000000C3
:1094F0003220EF0043A82400008041001040BA0051
:109500000160EF0000000600202000002053000052
:1095100065720000696100006C2000004563000076
:10952000686F0000202000002020000000000000E4
:109530003220EF0043AA2400008041001040BA000E
:109540000160EF0000000600202000002053000012
:1095500065720000696100006C200000496E000027
:10956000666F0000202000002020000000000000A6
:109570003220EF0043AC2400008041001040BA00CC
:109580000160EF00000006002020000020500000D5
:10959000616E0000656C0000204C000069670000EF
:1095A000687400007320000020200000000000000C
:1095B0003220EF0043AE2400008041001040BA008A
:1095C0000160EF00000006002020000020430000A2
:1095D0006C65000061720000204D0000656D0000A8
:1095E0006F720000792000002020000000000000C1
:1095F0003220EF0043B02400008041001040BA0048
:109600000160EF0000000600202000002043000061
:109610006C6500006172000020500000726500005F
:10962000736500007473000020200000000000003B
:109630003220EF0043B22400008041001040BA0005
:109640000160EF000000060020200000506F0000C5
:109650007765000072200000557000002050000067
:1096600072650000736500007420000000000000B7
:109670003220EF0043B42400008041001040BA00C3
:109680000160EF0000000600202000005072000082
:109690006573000065740000204C00006F630000DB
:1096A00061740000696F00006E200000000000007F
:1096B0003220EF0043B62400008041001040BA0081
:1096C0000160EF0000000600202000002053000091
:1096D0007769000074630000686900006E6700002D
:1096E000204D00006F6400006520000000000000B5
:1096F0003220EF0043B82400008041001040BA003F
:109700000160EF00000006002020000054720000FD
:10971000616E000073690000746900006F6E0000E4
:10972000205300007761000070200000000000005E
:109730003220EF0043BA2400008041001040BA00FC
:109740000160EF0000000600202000002020000043
:1097500053650000747400006C6500002054000024
:10976000696D00006520000020200000000000005E
:109770003220EF0043BC2400008041001040BA00BA
:109780000160EF0000000600202000002020000003
:10979000204600005442000020540000696D000083
:1097A00065200000202000002020000000000000B4
:1097B0003220EF0043BE2400008041001040BA0078
:1097C0000160EF0000000600202000005072000041
:1097D0006F670000726100006D2000004C6F000098
:1097E000636B00006F750000742000000000000033
:1097F0003220EF0043C02400008041001040BA0036
:109800000160EF0000000600202000002020000082
:10981000546100006C6C0000792000004C65000071
:10982000766500006C200000202000000000000091
:109830003220EF0043C22400008041001040BA00F3
:109840000160EF0000000600202000002020000042
:109850005361000076650000204300006F6E000039
:109860006669000067200000202000000000000062
:109870003220EF0043C42400008041001040BA00B1
:109880000160EF000000060020560000494400007F
:10989000454F0000204F0000555400005055000077
:1098A000542000004D4500004E550000000000000F
:1098B0003220EF0043C62400008041001040BA006F
:1098C0000160EF0000000600202000005072000040
:1098D0006F670000726100006D2000004F7500008E
:1098E000747000007574000020200000000000006B
:1098F0003220EF0043C82400008041001040BA002D
:109900000160EF00000006002020000050720000FF
:109910006576000069650000772000004F75000043
:10992000747000007574000020200000000000002A
:109930003220EF0043CA2400008041001040BA00EA
:109940000160EF0000000600202000002050000011
:10995000414E00002044000049520000204D00000C
:10996000454E0000552000002020000000000000AF
:109970003220EF0043CC2400008041001040BA00A8
:109980000160EF00000006002020000020540000CD
:10999000494C0000542000004449000052200000BF
:1099A0004D4500004E550000202000000000000042
:1099B0003220EF0043CE2400008041001040BA0066
:1099C0000160EF000000060020200000205A000087
:1099D0004F4F00004D20000044490000522000007D
:1099E0004D4500004E550000202000000000000002
:1099F0003220EF0043D02400008041001040BA0024
:109A00000160EF00000006002056000049440000FD
:109A1000454F0000204900004E5000005554000002
:109A2000204D0000454E00005520000000000000C1
:109A30003220EF0043D22400008041001040BA00E1
:109A40000160EF00000006002020000043410000FC
:109A50004D200000534500004152000043480000E3
:109A6000204D0000454E0000552000000000000081
:109A70003220EF0043D42400008041001040BA009F
:109A80000160EF00000006002020000043430000BA
:109A9000552000004D4F000044450000204D0000BF
:109AA000454E00005520000020200000000000006E
:109AB0003220EF0043D62400008041001040BA005D
:109AC0000160EF00000006002020000020200000C0
:109AD000204100006C6C0000205000006F720000FC
:109AE000747300002020000020200000000000000F
:109AF0003220EF0043D82400008041001040BA001B
:109B00000160EF000000060020200000202000007F
:109B100020200000506F0000727400002030000010
:109B20003120000020200000202000000000000064
:109B30003220EF0043DA2400008041001040BA00D8
:109B40000160EF000000060020200000202000003F
:109B500020200000506F00007274000020300000D0
:109B60003220000020200000202000000000000023
:109B70003220EF0043DC2400008041001040BA0096
:109B80000160EF00000006002020000020200000FF
:109B900020200000506F0000727400002030000090
:109BA00033200000202000002020000000000000E2
:109BB0003220EF0043DE2400008041001040BA0054
:109BC0000160EF00000006002020000020200000BF
:109BD00020200000506F0000727400002030000050
:109BE00034200000202000002020000000000000A1
:109BF0003220EF0043E02400008041001040BA0012
:109C00000160EF000000060020200000202000007E
:109C100020200000506F000072740000203000000F
:109C2000352000002020000020200000000000005F
:109C30003220EF0043E22400008041001040BA00CF
:109C40000160EF000000060020200000202000003E
:109C500020200000506F00007274000020300000CF
:109C6000362000002020000020200000000000001E
:109C70003220EF0043E42400008041001040BA008D
:109C80000160EF00000006002020000020200000FE
:109C9000204D0000414900004E2000004D450000CD
:109CA0004E55000020200000202000000000000091
:109CB0003220EF0043E62400008041001040BA004B
:109CC0000160EF0000000600202000005265000047
:109CD00073630000616E000020430000616D0000AE
:109CE0006572000061730000202000000000000089
:109CF0003220EF0043E82400008041001040BA0009
:109D00000160EF000000060020200000205200004B
:109D100065730000636100006E200000566900005A
:109D2000646500006F20000020200000000000009B
:109D30003220EF0043EA2400008041001040BA00C6
:109D40000160EF000000060020560000696400007A
:109D5000656F0000204F00007574000070750000F2
:109D6000742000004D6500006E75000000000000CA
:109D70003220EF0043EC2400008041001040BA0084
:109D80000160EF000000060020560000696400003A
:109D9000656F0000204900006E70000075740000BF
:109DA000204D0000656E00007520000000000000DE
:109DB0003220EF0043EE2400008041001040BA0042
:109DC0000160EF000000060020440000656600000E
:109DD000617500006C74000020430000616D00009C
:109DE00065720000612000004E6F0000000000005E
:109DF0003220EF0043F02400008041001040BA0000
:109E00000160EF00000006002044000065660000CD
:109E1000617500006C740000205000007265000045
:109E200073650000742000004E6F00000000000009
:109E30003220EF0043F22400008041001040BA00BD
:109E40000160EF000000060020440000656600008D
:109E5000617500006C74000020490000646C000013
:109E60006520000052740000726E000000000000C7
:109E70003220EF0043F42400008041001040BA007B
:109E80000160EF00000006002020000020500000CC
:109E9000616E00002044000069720000204D000047
:109EA000656E00007520000020200000000000000A
:109EB0003220EF0043F62400008041001040BA0039
:109EC0000160EF0000000600202000002054000088
:109ED000696C0000742000004469000072200000DA
:109EE0004D6500006E75000020200000000000009D
:109EF0003220EF0043F82400008041001040BA00F7
:109F00000160EF000000060020200000205A000041
:109F10006F6F00006D200000446900007220000097
:109F20004D6500006E75000020200000000000005C
:109F30003220EF0043FA2400008041001040BA00B4
:109F40000160EF0000000600205000007265000074
:109F50007365000074200000506100006E20000056
:109F600053700000656500006420000000000000E0
:109F70003220EF0043FC2400008041001040BA0072
:109F80000160EF0000000600205000007265000034
:109F90007365000074200000546900006C740000B8
:109FA00020530000706500006564000000000000A0
:109FB0003220EF0043FE2400008041001040BA0030
:109FC0000160EF00000006002050000072650000F4
:109FD00073650000742000005A6F00006F6D000070
:109FE0002053000070650000656400000000000060
:109FF0003220EF0043002500008041001040BA00ED
:10A000000160EF00000006002045000078740000A9
:10A01000657200006E6100006C2000005472000048
:10A0200069670000676500007273000000000000AF
:10A030003220EF0043022500008041001040BA00AA
:10A040000160EF000000060020530000656C000076
:10A050006563000074200000466F00006C6C000017
:10A060006F770000205000007276000000000000B2
:10A070003220EF0043042500008041001040BA0068
:10A080000160EF0000000600202000004361000096
:10A090006D200000536500006172000063680000DD
:10A0A000204D0000656E00007520000000000000DB
:10A0B0003220EF0043062500008041001040BA0026
:10A0C0000160EF0000000600202000002043000097
:10A0D00043550000204D00006F6400006520000023
:10A0E0004D6500006E75000020200000000000009B
:10A0F0003220EF0043082500008041001040BA00E4
:10A100000160EF0000000600202000002020000079
:10A110005379000073740000656D0000204D00004D
:10A12000656E000075200000202000000000000087
:10A130003220EF00430A2500008041001040BA00A1
:10A140000160EF0000000600202000002020000039
:10A150002020000053740000617200007420000091
:10A16000202000002020000020200000000000002F
:10A170003220EF00430C2500008041001040BA005F
:10A180000160EF00000006002020000020360000E3
:10A1900020430000616D00003120000036200000E7
:10A1A000436100006D32000020200000000000002C
:10A1B0003220EF00430E2500008041001040BA001D
:10A1C0000160EF00000006002020000020200000B9
:10A1D000416C00006C200000313200002043000080
:10A1E000616D000031200000202000000000000010
:10A1F0003220EF0043102500008041001040BA00DB
:10A200000160EF0000000600202000002020000078
:10A2100020200000202000004F4E000020200000E1
:10A22000202000002020000020200000200000004E
:10A230003220EF0043122500008041001040BA0098
:10A240000160EF0000000600202000002020000038
:10A2500020200000204F0000464600002020000083
:10A26000202000002020000020200000200000000E
:10A270003220EF0043142500008041001040BA0056
:10A280000160EF00000006002020000020200000F8
:10A2900020200000202000004F4E00002020000061
:10A2A00020200000202000002020000000000000EE
:10A2B0003220EF0043162500008041001040BA0014
:10A2C0000160EF00000006002020000020200000B8
:10A2D00020200000204F0000464600002020000003
:10A2E00020200000202000002020000000000000AE
:10A2F0003220EF0043182500008041001040BA00D2
:10A300000160EF0000000600202000002020000077
:10A31000204800006F6D00006520000043610000D0
:10A320006D65000072610000202000000000000048
:10A330003220EF00431A2500008041001040BA008F
:10A340000160EF0000000600202000002020000037
:10A35000205000007265000073650000742000004A
:10A36000313200002020000020200000000000000A
:10A370003220EF00431C2500008041001040BA004D
:10A380000160EF00000006002020000020200000F7
:10A39000204100006C6C0000204C00006F63000046
:10A3A000616C000020200000202000000000000060
:10A3B0003220EF00431E2500008041001040BA000B
:10A3C0000160EF00000006002020000036200000A1
:10A3D000496E0000436100006D200000362000003F
:10A3E0004C6F0000636100006C2000000000000062
:10A3F0003220EF0043202500008041001040BA00C9
:10A400000160EF0000000600202000002053000043
:10A41000696E0000676C0000652000004D6F000051
:10A4200064650000202000002020000000000000E3
:10A430003220EF0043222500008041001040BA0086
:10A440000160EF0000000600202000002020000036
:10A4500044750000616C0000204D00006F64000036
:10A4600065200000202000002020000000000000E7
:10A470003220EF0043242500008041001040BA0044
:10A480000160EF00000006002020000020200000F6
:10A4900041630000746900007665000020480000F8
:10A4A0006967000068200000202000000000000014
:10A4B0003220EF0043262500008041001040BA0002
:10A4C0000160EF00000006002020000020200000B6
:10A4D000416300007469000076650000204C0000B4
:10A4E0006F77000020200000202000000000000006
:10A4F0003220EF0043282500008041001040BA00C0
:10A500000160EF0000000600202000005361000001
:10A5100076650000204300006F6E00006669000051
:10A52000672000004E6F0000772000002000000030
:10A530003220EF00432A2500008041001040BA007D
:10A540000160EF0000000600202000002020000035
:10A55000202000004E6F0000726D0000616C000052
:10A56000202000002020000020200000000000002B
:10A570003220EF00432C2500008041001040BA003B
:10A580000160EF00000006002020000020200000F5
:10A5900020200000496E0000766500007274000003
:10A5A00020200000202000002020000000000000EB
:10A5B0003220EF00432E2500008041001040BA00F9
:10A5C0000160EF0000000600204800004420000069
:10A5D00031300000383000007020000035390000B4
:10A5E0002E390000344800007A20000000000000EE
:10A5F0003220EF0043302500008041001040BA00B7
:10A600000160EF0000000600204800004420000028
:10A61000313000003830000070200000353000007C
:10A62000487A0000202000002020000000000000E8
:10A630003220EF0043322500008041001040BA0074
:10A640000160EF00000006002048000044200000E8
:10A65000313000003830000069200000353900003A
:10A660002E390000344800007A200000000000006D
:10A670003220EF0043342500008041001040BA0032
:10A680000160EF00000006002048000044200000A8
:10A690003130000038300000692000003530000003
:10A6A000487A000020200000202000000000000068
:10A6B0003220EF0043362500008041001040BA00F0
:10A6C0000160EF0000000600202000004E6F000037
:10A6D0007420000053750000707000006F7200005D
:10A6E00074650000642000002020000000000000CD
:10A6F0003220EF0043382500008041001040BA00AE
:10A700000160EF000000060020530000442000001C
:10A710004E540000534300002D280000532D00002C
:10A7200056690000646500006F2900000000000009
:10A730003220EF00433A2500008041001040BA006B
:10A740000160EF00000006002053000044200000DC
:10A7500020500000414C00002D280000532D000027
:10A7600056690000646500006F29000000000000C9
:10A770003220EF00433C2500008041001040BA0029
:10A780000160EF0000000600204100007574000029
:10A790006F200000536500006172000063680000D4
:10A7A000204D00006F6400006520000000000000E4
:10A7B0003220EF00433E2500008041001040BA00E7
:10A7C0000160EF00000006002020000020200000B3
:10A7D000205300006F6E0000792000004F6E0000D3
:10A7E0006C79000020200000202000000000000004
:10A7F0003220EF0043402500008041001040BA00A5
:10A800000160EF0000000600202000002020000072
:10A81000436100006E6F00006E2000004F6E00006C
:10A820006C790000202000002020000000000000C3
:10A830003220EF0043422500008041001040BA0062
:10A840000160EF00000006002020000050610000C1
:10A850006E610000736F00006E69000063200000ED
:10A860004F6E00006C790000202000000000000006
:10A870003220EF0043442500008041001040BA0020
:10A880000160EF0000000600202000004469000085
:10A89000726500006374000020430000616D0000D9
:10A8A00020430000747200006C20000000000000D3
:10A8B0003220EF0043462500008041001040BA00DE
:10A8C0000160EF000000060020200000434300006C
:10A8D00055200000436100006D200000436F000020
:10A8E0006E740000726F00006C2000000000000019
:10A8F0003220EF0043482500008041001040BA009C
:10A900000160EF0000000600204800005620000013
:10A910003139000032300000783100003230000060
:10A920003020000036300000487A000000000000AF
:10A930003220EF00434A2500008041001040BA0059
:10A940000160EF00000006002053000044200000DA
:10A950002034000038300000692000003239000047
:10A960002E390000374800007A2000000000000067
:10A970003220EF00434C2500008041001040BA0017
:10A980000160EF000000060020530000442000009A
:10A990002035000037360000692000003235000005
:10A9A000487A000020200000202000000000000065
:10A9B0003220EF00434E2500008041001040BA00D5
:10A9C0000160EF00000006002053000079730000D2
:10A9D000746500006D200000496E000020530000E7
:10A9E000746100006E6400006279000000000000E5
:10A9F0004200F8003600F800801F78002000200098
:10AA00000C000900B01F78009032810000C0B30034
:10AA1000903289002202AE00FEFF37003011800024
:10AA20005226F800E0FF9F005226F900B44F800044
:10AA30000960EF006397200083024200903281009A
:10AA400080429800B44F80000960EF0063972000B7
:10AA500003004200104278006D24E10001003A003A
:10AA6000F969EC00B44F8000614242000440780074
:10AA700000E0B700040820000024E10003003E00CD
:10AA8000F669EF004855040000000000F669EC008C
:10AA9000F809A800B808AF003900370018A9AE00BF
:10AAA0003700370090328100140220000024E100BA
:10AAB0000800320090328100240220000024E100CE
:10AAC0000400320090328100040320000024E100E1
:10AAD0000D003A00A45380004822DE001308200035
:10AAE000041CE10008003E00A45380004822DE0060
:10AAF00093082000041CE10003003900903281001B
:10AB000000C0B30090328900903281006804E100F7
:10AB10000F003A00903281002322AF00FEFF370081
:10AB200024E2B7002562EF0000C2B3002322AF0089
:10AB3000FEFF370024E2B7002562EF00903281006B
:10AB40002322AF00FEFF370024E2B7002562EF00AA
:10AB5000903281007F04E1000900360090328100CC
:10AB6000F40720000024E100050036009032810047
:10AB70002322AF00FEFF370024E2B7002562EF007A
:10AB80009032810075EAB7009560A8008560A90041
:10AB9000A00120000C0009004F1078004F00780041
:10ABA0003600F9004200F900004006004200F800BB
:10ABB0003600F800801F7800200020000C000900FB
:10ABC000B01F78008032810000C0B300803289005D
:10ABD0003202AE00FEFF3700B01180005026F800B0
:10ABE000E0FF9F005026F900B828AE0007003700AC
:10ABF000803281002322AF00FEFF370024E2B7003D
:10AC00002562EF002A5604000000000094538000E3
:10AC10000960EF00A39F2000830242008032810080
:10AC200080429800F829A8009453800061424200B5
:10AC30000440780000E0B700840720000024E10011
:10AC400003003E00726AEF002A5604000000000074
:10AC5000726AEC0097C0A80087C0A900A00120007C
:10AC60000C0009004F1078004F0078003600F90002
:10AC70004200F9000040060004002000A4338900CF
:10AC800004002000B433890004002000C43389008C
:10AC90009033810063006000A0338900803381001D
:10ACA00063006000B0338900A03381002080B200CF
:10ACB000070032001080B200150032002080B20080
:10ACC000230032001080B200310032004000370013
:10ACD000B03381000000E00005003A00C03381007D
:10ACE0000000E900C0338900845604000000000021
:10ACF000B03381006300E10003003A00C0338100FB
:10AD00000000E800C0338900E8560400000000009D
:10AD1000B03381006200E10005003A00C0338100D9
:10AD20000000E900C0338900A456040000000000C0
:10AD3000B03381006100E10003003A00C0338100BC
:10AD40000000E800C0338900E8560400000000005D
:10AD5000B03381006300E10005003A00C033810098
:10AD60000000E900C0338900C45604000000000060
:10AD7000B03381000000E00003003A00C0338100DE
:10AD80000000E800C0338900E8560400000000001D
:10AD9000B03381006100E10005003A00C03381005A
:10ADA0000000E900C0338900E45604000000000000
:10ADB000B03381006200E10003003A00C03381003B
:10ADC0000000E800C0338900E856040000000000DD
:10ADD0007826F8000000F900000006004200F800A4
:10ADE0003600F800801F7800200020000C000900C9
:10ADF000B01F780004002000843289000400200085
:10AE00009432890004002000A4328900040020004C
:10AE1000B432890004002000C4328900D03281009D
:10AE200000C0B300D03289009500A9000828EC00CA
:10AE30004220AF000A28EC000C28EC004220AF00B2
:10AE40000E28EC00C6A2EF00C802F8005226F90056
:10AE5000903281000002780000FC2F0004006000A6
:10AE600090328900903281002088B600A03289009B
:10AE7000A03281000000E0008C003200A03281008E
:10AE80000002780000002C00840260000500E00051
:10AE900013003200903281004E00DE00B032890093
:10AEA000B0328900004180004E00DE00C0328900CF
:10AEB000C03289005626F8007026F9005826F8009E
:10AEC0007226F9003C560200000000008032890022
:10AED00080328100D440800000004200D0408800D1
:10AEE000A03281000002780000002300840260008C
:10AEF0000500E00013003200903281004C00DE00BB
:10AF0000B0328900B0328900004180004C00DE0080
:10AF1000C0328900C03289005626F8007026F90038
:10AF20005826F8007226F9003C5602000000000086
:10AF30008032890080328100B440800000004200ED
:10AF4000B0408800A03281000002780000C02000DC
:10AF5000840260000500E00013003200903281009E
:10AF60004A00DE00B0328900B03289000041800022
:10AF70004A00DE00C0328900C03289005626F8003F
:10AF80007026F9005826F8007226F9003C56020097
:10AF9000000000008032890080328100A4408000DF
:10AFA00000004200A0408800A032810080027800AA
:10AFB0000530B2000500E0001B0032005226F80008
:10AFC0004F0078004800DE005626F800E0FF9F00A2
:10AFD0005626F900B03281000160EF00B0328900DE
:10AFE00021C8BF005826F800E0FF9F005826F9004E
:10AFF000C03281000160EF00C03289005626F8009F
:10B000007026F9005826F8007226F9003C56020016
:10B01000000000008032890080328100944080006E
:10B020000000420090408800A03281008002780039
:10B03000050CB2000500E0001300320090328100E0
:10B040004600DE00B0328900B03289000041800045
:10B050004600DE00C0328900C03289005626F80062
:10B060007026F9005826F8007226F9003C560200B6
:10B07000000000008032890080328100C4408000DE
:10B0800000004200C04088005226F8002008F90065
:10B090002228EF002568A8008500A9009500A800D7
:10B0A0001D00370058580400000000002228EC0062
:10B0B0002003A9002023A8002003AE00FEFF3700D4
:10B0C000001880004200DE005A26F800E0FF9F00D2
:10B0D0005A26F900145D80004822DE0063D8200063
:10B0E00083024200D032810080429800A36BEC00C2
:10B0F000145D80004822DE006324E1000100360078
:10B10000A36BEF00A3CBBF0028E3B7002963EF00D8
:10B110008500A9009500A8008500A900A0012000D5
:10B120000C0009004F1078004F0078003600F9003D
:10B130004200F900004006004200F8003600F80026
:10B14000801F7800200020000C000900B01F78004C
:10B150000400200084328900040020009432890019
:10B1600004002000A432890004002000B4328900C9
:10B17000C032810000C0B300C0328900C0328100FB
:10B180000160EF00C0328900D032810000C0B300FE
:10B19000D0328900D03281000160EF00D0328900C6
:10B1A000E032810000C0B300E0328900E03281006B
:10B1B0000160EF00E0328900F032810000C0B3008E
:10B1C000F0328900F03281000160EF00F032890036
:10B1D0009760A900C6A2EF00C802F8005026F90047
:10B1E0008032810000027800808F2F000400600010
:10B1F00090328900903281001E88B600A03289000A
:10B20000A03281000000E00053003200A032810033
:10B210005A26F800F0FF9F005A26F9005426F8003D
:10B220004F0078004800DE005C26F800E0FF9F0039
:10B230005C26F900D03281004800DE00E432810053
:10B24000044068005826F800E0FF9F005826F900E7
:10B250001EC8BF005E26F800E0FF9F005E26F900D2
:10B260001FC8BF005E26F800F0FF9F005E26F900B1
:10B27000E0328100F4328100044068005826F80072
:10B28000F0FF9F005826F900903281005A26F800FE
:10B29000F0FF9F005A26F900D03281004800DE00FE
:10B2A000F43281004822DE00044068005C26F80089
:10B2B000F0FF9F005C26F90034002000B4328900C2
:10B2C000B03281006800E1001D003100C132810010
:10B2D000B03281000100A500140039005C26F8009E
:10B2E000CF007800C808DE00B03281000100A50060
:10B2F00008003100B0328100E30250004128DD0037
:10B300002481200084024000950AE8009659040038
:10B3100000000000B0328100E30250004128DD004F
:10B320002481200084024000950AE900B0328100A7
:10B330000000E800B03289006059040000000000FD
:10B340005226F8001E08F9002568A8002228EF0000
:10B35000AE590400000000002228EC002003A900E0
:10B360002023A8002003AE00FEFF37000018800055
:10B370004200DE005A26F800E0FF9F005A26F9003E
:10B3800064D82000236C800084824100D032810088
:10B3900080429800A3CBBF000160EF000080B200A4
:10B3A000050032001080B200090032009080B20027
:10B3B0000D0032001200370010C0B300A3EBB7003D
:10B3C00014002000246C8800045A040000000000CF
:10B3D00080C0B300A3EBB70024002000246C8800D9
:10B3E000045A04000000000090C0B300A3EBB700B3
:10B3F00034002000246C8800045A0400000000007F
:10B40000A36BEF00842DEF00A3CBBF0028E3B700B0
:10B410002963EF008760A9009760A8008760A900F2
:10B42000A00120000C0009004F1078004F007800A8
:10B430003600F9004200F900004006000400200038
:10B4400094328900803281002080B2000B003200EB
:10B450001080B2000D0032007080B2000F00320088
:10B460001080B200110032003080B20013003200B0
:10B470007080B2001500320014003700F401200083
:10B48000943289006E5A040000000000040220007B
:10B49000943289006E5A040000000000140220005B
:10B4A000943289006E5A040000000000240220003B
:10B4B000943289006E5A040000000000340220001B
:10B4C000943289006E5A040000000000E40120005C
:10B4D000943289006E5A0400000000005226F800E1
:10B4E0000000F90000000600851F7800705C8000F5
:10B4F0004100DD0004A9200084024000C432810024
:10B5000084029800745C800061024200840278002A
:10B5100005027800F3072000110009000382D8001B
:10B52000715C8800F849A800CF027800000006008E
:10B530000400200054338900403381002080B20091
:10B54000170032001080B200190032007080B20083
:10B550001B0032001080B2001D0032003080B200AB
:10B560001F0032001080B20021003200F080B200D3
:10B57000230032001080B200250032003080B2007B
:10B58000270032001080B200290032007080B20023
:10B590002B003200D080B2002D0032002C0037008A
:10B5A0005402200054338900305B04000000000086
:10B5B0006402200054338900305B04000000000066
:10B5C0007402200054338900305B04000000000046
:10B5D0008402200054338900305B04000000000026
:10B5E0009402200054338900305B04000000000006
:10B5F000A402200054338900305B040000000000E6
:10B60000B402200054338900305B040000000000C5
:10B61000C402200054338900305B040000000000A5
:10B62000D402200054338900305B04000000000085
:10B63000E402200054338900305B04000000000065
:10B64000F402200054338900305B04000000000045
:10B650004402200054338900305B040000000000E5
:10B660006A26F8000000F90000000600040020002F
:10B67000A4328900903281001080B2000B003200A9
:10B680003080B2000D0032001080B2000F00320096
:10B690007080B200110032001080B200130032003E
:10B6A0003080B2001500320018003700E40020009E
:10B6B000A43289008A5B040000000000F40020002E
:10B6C000A43289008A5B040000000000040120000D
:10B6D000A43289008A5B04000000000014012000ED
:10B6E000A43289008A5B04000000000024012000CD
:10B6F000A43289008A5B04000000000034012000AD
:10B70000A43289008A5B040000000000F40F2000CE
:10B71000A43289005426F8000000F9000000060059
:10B720004200F8003600F800801F7800200020005A
:10B730000C000900B01F780099E0A90089E0A90079
:10B740001028EC0084408000430F20000418E10022
:10B750005B003E001028EF001C49E2005800320058
:10B760002508AE00560037001E49E20053003200A3
:10B77000846AAF00510037002468EC001CC9BF0088
:10B78000244180000024E1004A0039002508A90076
:10B790001EC9BF00BC48E3000D0032001EC9BF0037
:10B7A0005026F800E0FF9F005026F900803281000B
:10B7B0000160EF00803289001E5A02000000000084
:10B7C00080027800C5328900745A0200000000002F
:10B7D000F44880000960EF007300200004804100FD
:10B7E000848B2000040040001004E0000F003200B1
:10B7F0001F49E2000D0032001FC9BF006826F80093
:10B80000E0FF9F006826F900403381000160EF00EF
:10B8100040338900985A020000000000800278003E
:10B82000C5328900745A0200000000001EC9BF0022
:10B83000BB48E3001E0032001A09AE000F003700BB
:10B84000144EE2000D003A001EC9BF005226F80057
:10B85000E0FF9F005226F900903281000160EF0066
:10B8600090328900365B0200000000008002780000
:10B87000C5328900745A0200000000001EC9BF00D2
:10B880005226F800E0FF9F005226F9009032810016
:10B890000160EF0090328900365B0200000000007A
:10B8A00080027800C5328900745A0200000000004E
:10B8B0002468EF00605C0400000000002508A90077
:10B8C00099E0A80089E0A900A00120000C0009006F
:10B8D0004F1078004F0078003600F9004200F90060
:10B8E00000400600820020001E0009000000000049
:10B8F000C442A900C042A9001F00090000000000C6
:10B9000081C0D200C462A9004200AF00C062A8009A
:10B910004200AE00C062A900C042A800C242AE0010
:10B92000FEFF37000201E900EFFF3A001E000900A8
:10B9300000000000C442A900C042A90000000000AD
:10B94000C062A8001F000900000000001F000900DD
:10B9500000000000C042A800C242AE00FEFF370057
:10B960001F0009000000000000002000C262AF00BC
:10B970000000A000C442A900C042A900C462A900FE
:10B98000C062A90000000600851F7800C062A80000
:10B990001E00090000000000C042A8001F000900AE
:10B9A00000000000C242AE00FEFF3700C462A900E2
:10B9B000C062A9001E00090000000000C442A900E6
:10B9C000C042A900F1338100725C02000000000057
:10B9D00001348100725C0200000000008026F80043
:10B9E000CF027800C82ADE0085407800725C020031
:10B9F00000000000C062A90000000000C042A800D2
:10BA0000C242AE00FEFF37001E0009000000000029
:10BA10000100090000000000C062A8001E0009002B
:10BA200000000000CF027800000006008200200025
:10BA30001E00090000000000E842A900E442A9003D
:10BA40001F0009000000000081C0D200E862A900C8
:10BA50004200AF00E462A8004200AE00E462A90028
:10BA6000E442A800E642AE00FEFF37000201E90012
:10BA7000EFFF3A001E00090000000000E842A900A4
:10BA8000E442A90000000000E462A8001F000900D1
:10BA9000000000001F00090000000000E442A800B0
:10BAA000E642AE00FEFF37001F0009000000000064
:10BAB00000002000E662AF000000A000E842A900FC
:10BAC000E442A900E862A900E462A90000000600BF
:10BAD000851F7800E462A8001E0009000000000035
:10BAE000E442A8001F00090000000000E642AE008A
:10BAF000FEFF3700E862A900E462A9001E00090009
:10BB000000000000E842A900E442A90011348100CD
:10BB1000165D02000000000021348100165D020065
:10BB2000000000008426F800CF027800C82ADE005A
:10BB300085407800165D020000000000E462A90064
:10BB400000000000E442A800E642AE00FEFF37001D
:10BB50001E000900000000000100090000000000B4
:10BB6000E462A8001E00090000000000CF02780077
:10BB700000000600144580004822DE006124E10038
:10BB800010003A00803381008026F800E0FF9F001B
:10BB90008026F9007026F8004F0078004800DE008B
:10BBA0008026F800F0FF9F008026F9006E26F8003E
:10BBB0007E26F900C45C020000000000FE5D040067
:10BBC00000000000803381008426F800E0FF9F0021
:10BBD0008426F9007026F8004F0078004800DE0047
:10BBE0008426F800F0FF9F008426F9006E26F800F6
:10BBF0008226F900685D02000000000000000600D7
:10BC0000103381001080B20085003200F081B20054
:10BC10008E0032001080B2008C003200F083B2003F
:10BC20008A0032001080B200880032003080B200FA
:10BC3000860032001080B200840032007080B200B2
:10BC4000E00032001080B200DE0032003080B2002E
:10BC5000DC0032001080B200DA003200F080B20066
:10BC6000D80032001080B200D60032003080B2001E
:10BC7000D40032001080B200D20032007080B200D6
:10BC80004E0132001080B2004C0132003080B20010
:10BC90004A0132001080B200480132007082B200C6
:10BCA00046013200F080B200440132001080B20040
:10BCB000420132003080B200400132008081B20087
:10BCC000C20132001080B200C00132007080B200A8
:10BCD000BE0132001080B200BC0132003080B200E0
:10BCE000BA0132001080B200B8013200F080B20018
:10BCF000B60132001080B200B40132003080B200D0
:10BD00001A0232001080B200180232007080B200B5
:10BD1000160232001080B200140232003080B200ED
:10BD2000120232001080B20010023200F081B20024
:10BD30000E0232001080B2000C023200E083B2002A
:10BD4000720232001080B200700232003080B20005
:10BD50006E0232001080B2006C0232007080B200BD
:10BD60006A0232001080B200680232003080B200F5
:10BD7000660232001080B20064023200F080B2002D
:10BD8000D80232001080B200D60232003080B200F9
:10BD9000D40232001080B200D20232007080B200B1
:10BDA000D00232008083B2001A0332007080B200E9
:10BDB00018033200C083B20016033200F087B200CD
:10BDC00014033200E087B200120332003080B20068
:10BDD00010033200C087B2006C0332003080B20022
:10BDE0006A033200D081B2008A033200F083B200CD
:10BDF000970332001080B200A40332003080B200FA
:10BE0000BF0332001080B200CD0332007080B20058
:10BE1000E60332001080B200F40332006A043700F7
:10BE2000203381000004E00004003A00E382A8000F
:10BE3000DF82A900225F040000000000E382A90065
:10BE4000DF82A900E46704000000000020338100C5
:10BE50000004E00028003A00103381007E00E10079
:10BE600003003A00764AA900785F04000000000051
:10BE7000103381007F00E10003003A00766AA900D8
:10BE8000785F0400000000001033810004022000ED
:10BE90000020E10003003A00768AA900785F0400E0
:10BEA0000000000010338100140220000020E10097
:10BEB00003003A0076AAA900785F040000000000A1
:10BEC00010338100240220000020E10003003A002A
:10BED00076CAA900785F04000000000010338100DA
:10BEE000340220000020E10001003A0076EAA900B7
:10BEF000C85F040000000000103381007E00E100F4
:10BF000003003A00764AA800C85F04000000000061
:10BF1000103381007F00E10003003A00766AA80038
:10BF2000C85F0400000000001033810004022000FC
:10BF30000020E10003003A00768AA800C85F0400F0
:10BF40000000000010338100140220000020E100F6
:10BF500003003A0076AAA800C85F040000000000B1
:10BF600010338100240220000020E10003003A0089
:10BF700076CAA800C85F04000000000010338100EA
:10BF8000340220000020E10001003A0076EAA80017
:10BF900064042000743389008033810080C0B300C2
:10BFA0008033890076CABF007026F800F0FF9F003A
:10BFB0007026F900BA5D020000000000E46704008A
:10BFC00000000000203381000004E00038003A0047
:10BFD00010338100440220000020E10003003A00F9
:10BFE000780AA900546004000000000010338100AA
:10BFF000540220000020E10003003A00782AA90042
:10C00000546004000000000010338100640220002E
:10C010000020E10003003A00784AA90054600400BF
:10C020000000000010338100740220000020E100B5
:10C0300003003A00786AA900546004000000000080
:10C0400010338100840220000020E10003003A0048
:10C05000788AA900546004000000000010338100B9
:10C06000940220000020E10003003A0078AAA90011
:10C07000546004000000000010338100A40220007E
:10C080000020E10003003A0078CAA90054600400CF
:10C090000000000010338100B40220000020E10005
:10C0A00001003A0078EAA900C46004000000000022
:10C0B00010338100440220000020E10003003A0018
:10C0C000780AA800C460040000000000103381005A
:10C0D000540220000020E10003003A00782AA80062
:10C0E000C4600400000000001033810064022000DE
:10C0F0000020E10003003A00784AA800C460040070
:10C100000000000010338100740220000020E100D4
:10C1100003003A00786AA800C46004000000000030
:10C1200010338100840220000020E10003003A0067
:10C13000788AA800C4600400000000001033810069
:10C14000940220000020E10003003A0078AAA80031
:10C15000C46004000000000010338100A40220002D
:10C160000020E10003003A0078CAA800C46004007F
:10C170000000000010338100B40220000020E10024
:10C1800001003A0078EAA8006404200074338900B2
:10C190008033810090C0B3008033890078CABF002B
:10C1A0007026F800F0FF9F007026F900BA5D0200CB
:10C1B00000000000E467040000000000203381005C
:10C1C0000004E0003B003A0010338100C40220006C
:10C1D0000020E10003003A007A0AA9005661040039
:10C1E0000000000010338100D40220000020E10094
:10C1F00003003A007A2AA9005661040000000000FA
:10C2000010338100C40220000020E10003003A0046
:10C210007A0AA90056610400000000001033810072
:10C22000E40220000020E10003003A007A4AA9005D
:10C23000566104000000000010338100F402200069
:10C240000020E10003003A007A6AA9005661040068
:10C2500000000000103381006800E10003003A0094
:10C260007ACAA90056610400000000001033810062
:10C270006700E10003003A007AAAA90056610400B1
:10C2800000000000103381006600E10003003A0066
:10C290007A8AA90056610400000000001033810072
:10C2A0006500E10001003A007AEAA900CC610400CF
:10C2B0000000000010338100C40220000020E100D3
:10C2C00003003A007A0AA800CC61040000000000D4
:10C2D00010338100D40220000020E10003003A0066
:10C2E0007A2AA800CC61040000000000103381000D
:10C2F000C40220000020E10003003A007A0AA800EE
:10C30000CC6104000000000010338100E402200032
:10C310000020E10003003A007A4AA800CC61040042
:10C320000000000010338100F40220000020E10032
:10C3300003003A007A6AA800CC6104000000000003
:10C34000103381006800E10003003A007ACAA800B7
:10C35000CC61040000000000103381006700E100A0
:10C3600003003A007AAAA800CC6104000000000093
:10C37000103381006600E10003003A007A8AA800C9
:10C38000CC61040000000000103381006500E10072
:10C3900001003A007AEAA80064042000743389009E
:10C3A00080338100A0C0B300803389007ACABF0007
:10C3B0007026F800F0FF9F007026F900BA5D0200B9
:10C3C00000000000E467040000000000203381004A
:10C3D0000004E0002D003A00103381007B00E100F2
:10C3E00003003A007C4AA9004262040000000000F9
:10C3F000103381007A00E10003003A007C6AA90052
:10C400004262040000000000103381007900E10066
:10C4100003003A007C8AA900426204000000000088
:10C42000103381007800E10003003A007CAAA900E3
:10C430004262040000000000103381007700E10038
:10C4400003003A007CCAA900426204000000000018
:10C45000103381007600E10003003A007CEAA90075
:10C460004262040000000000103381007D00E10002
:10C4700003003A007C0AA9004262040000000000A8
:10C480007C2AA9009C620400000000001033810097
:10C490007B00E10003003A007C4AA8009C62040093
:10C4A00000000000103381007A00E10003003A0030
:10C4B0007C6AA8009C620400000000001033810028
:10C4C0007900E10003003A007C8AA8009C62040025
:10C4D00000000000103381007800E10003003A0002
:10C4E0007CAAA8009C6204000000000010338100B8
:10C4F0007700E10003003A007CCAA8009C620400B7
:10C5000000000000103381007600E10003003A00D3
:10C510007CEAA8009C620400000000001033810047
:10C520007D00E10003003A007C0AA8009C62040040
:10C53000000000007C2AA8006404200074338900F5
:10C5400080338100B0C0B300803389007CCABF0053
:10C550007026F800F0FF9F007026F900BA5D020017
:10C5600000000000E46704000000000020338100A8
:10C570000004E0002D003A00103381007300E10058
:10C5800003003A007E4AA900126304000000000084
:10C59000103381007200E10003003A007E6AA900B6
:10C5A0001263040000000000103381007100E100FC
:10C5B00003003A007E8AA900126304000000000014
:10C5C000103381007000E10003003A007EAAA90048
:10C5D0001263040000000000103381006F00E100CE
:10C5E00003003A007ECAA9001263040000000000A4
:10C5F000103381006E00E10003003A007EEAA900DA
:10C600001263040000000000103381007500E10097
:10C6100003003A007E0AA900126304000000000033
:10C620007E2AA9006C630400000000001033810022
:10C630007300E10003003A007E4AA8006C63040026
:10C6400000000000103381007200E10003003A0096
:10C650007E6AA8006C6304000000000010338100B3
:10C660007100E10003003A007E8AA8006C630400B8
:10C6700000000000103381007000E10003003A0068
:10C680007EAAA8006C630400000000001033810043
:10C690006F00E10003003A007ECAA8006C6304004A
:10C6A00000000000103381006E00E10003003A003A
:10C6B0007EEAA8006C6304000000000010338100D3
:10C6C0007500E10003003A007E0AA8006C630400D4
:10C6D000000000007E2AA800640420007433890052
:10C6E00080338100C0C0B300803389007ECABF00A0
:10C6F0007026F800F0FF9F007026F900BA5D020076
:10C7000000000000E4670400000000002033810006
:10C710000004E00034003A001033810004032000DC
:10C720000020E10003003A00800AA900F063040041
:10C730000000000010338100140320000020E100FD
:10C7400003003A00802AA900F06304000000000002
:10C7500010338100240320000020E10003003A0090
:10C76000804AA900F063040000000000103381003B
:10C77000340320000020E10003003A00806AA90091
:10C78000F063040000000000103381004403200027
:10C790000020E10003003A00808AA900F063040051
:10C7A0000000000010338100540320000020E1004D
:10C7B00003003A0080AAA900F06304000000000012
:10C7C00010338100640320000020E10003003A00E0
:10C7D00080CAA900F06304000000000080EAA900FC
:10C7E000586404000000000010338100040320009E
:10C7F0000020E10003003A00800AA8005864040009
:10C800000000000010338100140320000020E1002C
:10C8100003003A00802AA8005864040000000000C9
:10C8200010338100240320000020E10003003A00BF
:10C83000804AA80058640400000000001033810002
:10C84000340320000020E10003003A00806AA800C1
:10C8500058640400000000001033810044032000ED
:10C860000020E10003003A00808AA8005864040018
:10C870000000000010338100540320000020E1007C
:10C8800003003A0080AAA8005864040000000000D9
:10C8900010338100640320000020E10003003A000F
:10C8A00080CAA800586404000000000080EAA800C4
:10C8B00084042000743389008033810080C0B30079
:10C8C0008033890080CABF007026F800F0FF9F0007
:10C8D0007026F900BA5D020000000000E467040061
:10C8E00000000000203381000004E0001F003A0037
:10C8F00010338100840320000020E10003003A008F
:10C90000820AA900B2640400000000001033810014
:10C91000940320000020E10003003A00822AA900CD
:10C92000B26404000000000010338100A403200062
:10C930000020E10003003A00824AA900B26404002A
:10C940000000000010338100B40320000020E1004B
:10C9500003003A00826AA900B264040000000000EB
:10C96000828AA900F06404000000000010338100F6
:10C97000840320000020E10003003A00820AA8009E
:10C98000F0640400000000001033810094032000D4
:10C990000020E10003003A00822AA800F0640400AD
:10C9A0000000000010338100A40320000020E100FB
:10C9B00003003A00824AA800F0640400000000006E
:10C9C00010338100B40320000020E10003003A008E
:10C9D000826AA800F064040000000000828AA800B7
:10C9E00084042000743389008033810090C0B30038
:10C9F0008033890082CABF007026F800F0FF9F00D4
:10CA00007026F900BA5D020000000000E46704002F
:10CA100000000000203381000004E00028003A00FC
:10CA2000103381006400E10003003A00846AA90029
:10CA30005C65040000000000103381006300E10029
:10CA400003003A00844AA9005C650400000000006D
:10CA500010338100F40320000020E10003003A00BD
:10CA600084CAA9005C650400000000001033810046
:10CA7000040420000020E10003003A0084EAA90039
:10CA80005C6504000000000010338100E403200016
:10CA90000020E10003003A0084AAA9005C650400BC
:10CAA0000000000010338100D40320000020E100CA
:10CAB00001003A00848AA900AC650400000000006F
:10CAC000103381006400E10003003A00846AA8008A
:10CAD000AC65040000000000103381006300E10039
:10CAE00003003A00844AA800AC650400000000007E
:10CAF00010338100F40320000020E10003003A001D
:10CB000084CAA800AC650400000000001033810056
:10CB1000040420000020E10003003A0084EAA80099
:10CB2000AC6504000000000010338100E403200025
:10CB30000020E10003003A0084AAA800AC650400CC
:10CB40000000000010338100D40320000020E10029
:10CB500001003A00848AA80084042000743389000C
:10CB600080338100A0C0B3008033890084CABF0035
:10CB70007026F800F0FF9F007026F900BA5D0200F1
:10CB800000000000E4670400000000002033810082
:10CB90000004E0000A003A00103381001404200071
:10CBA0000020E10003003A00866AA900DC65040069
:10CBB00000000000864AA900F065040000000000A3
:10CBC00010338100140420000020E10003003A002B
:10CBD000866AA800F065040000000000864AA800EC
:10CBE000840420007433890080338100B0C0B30016
:10CBF0008033890086CABF007026F800F0FF9F00CE
:10CC00007026F900BA5D020000000000E46704002D
:10CC100000000000F40F2000F4538800640420009A
:10CC20007433890080338100C0C0B3008033890031
:10CC30007ECABF007026F800F0FF9F007026F90042
:10CC4000BA5D020000000000E4670400000000007C
:10CC5000F40F2000E453880064042000743389003A
:10CC600080338100B0C0B300803389007CCABF002C
:10CC70007026F800F0FF9F007026F900BA5D0200F0
:10CC800000000000E467040000000000F40F200032
:10CC9000C453880064042000743389008033810009
:10CCA00090C0B3008033890078CABF007026F800B6
:10CCB000F0FF9F007026F900BA5D0200000000003E
:10CCC000D05380006F007000D053880064042000AF
:10CCD0007433890080338100A0C0B30080338900A1
:10CCE0007ACABF007026F800F0FF9F007026F90096
:10CCF000BA5D020000000000E467040000000000CC
:10CD0000B4538000C40FB300B453880064042000FF
:10CD1000743389008033810080C0B3008033890080
:10CD200076CABF007026F800F0FF9F007026F90059
:10CD3000BA5D020000000000E4670400000000008B
:10CD4000F40F200004548800840420007433890008
:10CD50008033810080C0B3008033890080CABF0067
:10CD60007026F800F0FF9F007026F900BA5D0200FF
:10CD700000000000820AA8008404200074338900A7
:10CD80008033810090C0B3008033890082CABF0025
:10CD90007026F800F0FF9F007026F900BA5D0200CF
:10CDA00000000000E467040000000000245480003C
:10CDB000040FB300245488008404200074338900D5
:10CDC00080338100A0C0B3008033890084CABF00D3
:10CDD0007026F800F0FF9F007026F900BA5D02008F
:10CDE00000000000E467040000000000C40F200001
:10CDF000B4538800640420007433890080338100B8
:10CE000080C0B3008033890076CABF007026F80066
:10CE1000F0FF9F007026F900BA5D020000000000DC
:10CE2000F40F2000C4538800640420007433890088
:10CE30008033810090C0B3008033890078CABF007E
:10CE40007026F800F0FF9F007026F900BA5D02001E
:10CE500000000000F40F2000D45388006404200078
:10CE60007433890080338100A0C0B300803389000F
:10CE70007ACABF007026F800F0FF9F007026F90004
:10CE8000BA5D020000000000F40F2000E4538800A7
:10CE9000640420007433890080338100B0C0B30083
:10CEA000803389007CCABF007026F800F0FF9F0025
:10CEB0007026F900BA5D020000000000F40F2000A7
:10CEC000F4538800640420007433890080338100A7
:10CED000C0C0B300803389007ECABF007026F8004E
:10CEE000F0FF9F007026F900BA5D0200000000000C
:10CEF000F40F200004548800840420007433890057
:10CF00008033810080C0B3008033890080CABF00B5
:10CF10007026F800F0FF9F007026F900BA5D02004D
:10CF200000000000F4012000145488008404200054
:10CF3000743389008033810090C0B300803389004E
:10CF400082CABF007026F800F0FF9F007026F9002B
:10CF5000BA5D020000000000C40F200024548800C5
:10CF6000840420007433890080338100A0C0B300A2
:10CF70008033890084CABF007026F800F0FF9F004C
:10CF80007026F900BA5D020000000000C400200015
:10CF90003454880084042000743389008033810075
:10CFA000B0C0B3008033890086CABF007026F80085
:10CFB000F0FF9F007026F900BA5D0200000000003B
:10CFC000E46704000000000000000600851F7800F0
:10CFD0000400200004338900F03281003081B20067
:10CFE0000B0032001080B2000D0032003080B20021
:10CFF0000F0032001080B20011003200F081B20048
:10D00000130032001080B200150032001800370003
:10D0100004082000043389003A680400000000007E
:10D0200004042000043389003A6804000000000072
:10D0300004022000043389003A6804000000000064
:10D0400004012000043389003A6804000000000055
:10D0500084002000043389003A68040000000000C6
:10D0600044002000043389003A68040000000000F6
:10D070001200370018E9AE000500370000338100C8
:10D0800000027800F0FF2F000400680000338900E0
:10D0900005338100840420007433890080338100CB
:10D0A000C0C0B300803389007026F800F5FF9F00F0
:10D0B0007026F900BA5D020000000000CF0278007F
:10D0C0000000060004002000643389005033810012
:10D0D000F082B200170032001080B2001800320057
:10D0E0003080B200190032001080B2001A00320005
:10D0F0007080B2001B0032001080B2001C003200B1
:10D100003080B2001D0032001080B2001E003200DC
:10D11000F080B2001F0032001080B2002000320008
:10D120003080B200210032001080B20022003200B4
:10D1300024003700603381000000E800603389007C
:10D14000603381000000E8006033890060338100B3
:10D150000000E80060338900603381000000E800CF
:10D1600060338900603381000000E800603389008B
:10D17000603381000000E800603389006033810083
:10D180000000E80060338900603381000000E8009F
:10D1900060338900603381000000E800603389005B
:10D1A000603381000000E800603389006033810053
:10D1B0000000E80060338900603381000000E8006F
:10D1C000603389006C26F8000000F90000000600BA
:10D1D000851F780004002000E4328900040020004C
:10D1E000F4328900D0328100440220000024E100A2
:10D1F00005003600D032810040C2B300D032890031
:10D200001269040000000000D0328100F402200006
:10D210000024E10003003100D0328100F0C2B300ED
:10D22000D0328900D03281006A26F800E0FF9F00EA
:10D230006A26F900503381000160EF005033890005
:10D240006268020000000000E0328900E0328100E4
:10D250000000E0001F00320004002000F4328900CA
:10D26000F03281006C00E1001A003100E0328100F0
:10D2700061004000E0328900E03281006C00E10092
:10D280000200360014002000E4328900E4328100FC
:10D290000960EF0083962000030042001004E000C4
:10D2A00007003A005C26F8006826F900985A020048
:10D2B00000000000080037006A6904000000000058
:10D2C000F03281000000E800F0328900306904008B
:10D2D000000000000060EF00CF02780000000600B0
:10D2E0004200F8003600F800801F7800200020007F
:10D2F0000C000900B01F780004002000943289005F
:10D30000A032810000C0B300A03289009A60A90059
:10D310002828EC00444180006A20E10068003900C0
:10D320002828EF0004002000943289009032810008
:10D33000240220000020E1006100360090328100CC
:10D34000E4862000040040001004E0005700320092
:10D3500090328100A4822000040040001004E0000C
:10D360004A00320090328100E48620000400400030
:10D370001042780004CEB20023003A0090328100BF
:10D38000140220000020E1001100320090328100E0
:10D39000A482200004004000904278006226F80039
:10D3A000E5FF9F006226F900103381000160EF0065
:10D3B000103389002033810000C0B300203389007E
:10D3C000005E020000000000006A0400000000008F
:10D3D00090328100A4822000040040009042780036
:10D3E0005E26F800E5FF9F005E26F900F03281001E
:10D3F0000160EF00F0328900E667020000000000E3
:10D40000466A04000000000090328100E48620009B
:10D41000040040001042780004CFB20011003A002E
:10D4200090328100A48220000400400090427800E5
:10D430006226F800E5FF9F006226F90010338100A4
:10D440000160EF00103389002033810010C0B30069
:10D4500020338900005E020000000000466A0400DC
:10D460000000000090328100E486200004004000AB
:10D470001042780004CDB20004003A0090328100DE
:10D48000A482200084024000804AEB009032810098
:10D49000A482200084024000804AEB009032810088
:10D4A000E486200084024000804AEB009032810034
:10D4B0000000E80090328900966904000000000036
:10D4C0002628EC0034418000C30320000418E1004A
:10D4D0006F003E002628EF000400200094328900EF
:10D4E00090328100240220000020E1006800360014
:10D4F00090328100A4822000040040001004E0006B
:10D500005E003200903281006D00E10025003200A3
:10D5100090328100A48220000400400090427800F4
:10D5200090328100C4842000040040001043780041
:10D530006226F800E5FF9F006226F90010338100A3
:10D540000160EF00103389006426F800E6FF9F00B9
:10D550006426F900005E02000000000090328100A5
:10D56000C4842000040040001004E00006003200E3
:10D5700090328100C484200084024000804AEB0085
:10D58000CE6A04000000000090328100C4842000B4
:10D590008402400010C0B300804A78003E6B040053
:10D5A000000000003648E20034003A003748E2004C
:10D5B0003200320037C8BF006226F800E0FF9F004B
:10D5C0006226F900103381000160EF0010338900FA
:10D5D0002033810010C0B30020338900005E0200B8
:10D5E0000000000037C8BF005426F800E0FF9F008D
:10D5F0005426F900A03281005A26F800E0FF9F006F
:10D600005A26F900E86802000000000037E8B70079
:10D610003748E20019003200A032810037C8B60056
:10D620000004E00009003A005948E20006003A0010
:10D6300010C0B30059E8B7009A60A8001600370080
:10D64000266B0400000000005968EF0037C8BF00D7
:10D650006226F800E0FF9F006226F9001033810087
:10D660000160EF00103389002033810000C0B30057
:10D6700020338900005E020000000000903281002B
:10D680000000E80090328900706A04000000000089
:10D690008A60A9009A60A8008A60A900A001200001
:10D6A0000C0009004F1078004F0078003600F90098
:10D6B0004200F900004006000000E0004220AF00F8
:10D6C00004003700793E0900000000000000E90076
:10D6D000F9FF370000000600B4B880006124E100C3
:10D6E00004003A00D262A900D662A9007E6B040051
:10D6F00000000000D262A900D662A800D222A900D0
:10D70000D622A800D642A900D242A9001E000900D4
:10D7100000000000D822EF0017D7BF00DCE2B700FE
:10D72000DD62EF001E00090000000000D642A800E4
:10D73000D242A9001E0009000000000000000600FF
:10D7400000CBB30011F7B7001217A80084B880000F
:10D750006924E1000300360080C0B30010F7B70071
:10D760001217A90011D7BF001057B40011F7B70066
:10D7700010C0B30016F7B70011D7BF0017F7B700F6
:10D780006C6B0200000000000040EB001217AF00BD
:10D790000000E800000006001177EF001277EF00AC
:10D7A0001317A80084B8800033082000041CE1008F
:10D7B0000300310030C8B30010F7B7001317A900F9
:10D7C00010D7BF0011F7B70010D7BF0012F7B7008E
:10D7D00012D7BF000160EF000160EF004400DE00DF
:10D7E00012F7B700247121001440A00010C0B3004C
:10D7F00016F7B70012D7BF0017F7B7006C6B02001F
:10D8000000000000A00020005C6B0200000000008F
:10D8100010D7BF0012F7B70012D7BF006F406000EB
:10D8200012F7B70010C0B30016F7B70012D7BF0049
:10D8300017F7B7006C6B020000000000A00020008A
:10D840005C6B0200000000000040EB001317AF000B
:10D850000000E800000006005372EF005472EF0071
:10D86000949280006824E1000400360080C0B30078
:10D8700053F2B700426C04000000000052D2BF0017
:10D8800053F2B70052D2BF0010F7B700A06B0200EE
:10D89000000000001077EF00CC6B020000000000D9
:10D8A0005472EF00A492800043082000041CE100A1
:10D8B000070036001677EF001777EF006C6B020059
:10D8C000000000005472EC00526C040000000000E4
:10D8D00010C0B30000E0B700000006002272EF00A5
:10D8E0002272EF00149180006924E10007003100EA
:10D8F00022D2BF0052F2B7002C6C020000000000E0
:10D900002272EC00726C04000000000000000600AF
:10D9100010C0B30016F7B700E0CAB30017F7B7009E
:10D920006C6B020000000000D282A900D682A90020
:10D930003E01090000000000D282A900D682A800A2
:10D94000803E20005C6B02000000000010C0B300AD
:10D9500016F7B70080C2B30017F7B7006C6B020070
:10D960000000000010C0B30016F7B70020CEB300CF
:10D9700017F7B7006C6B02000000000010C0B30086
:10D9800016F7B70000C1B30017F7B7006C6B0200C1
:10D990000000000010C0B30016F7B7001777EF00C3
:10D9A0006C6B02000000000010C0B30016F7B70057
:10D9B00000CBB30017F7B7006C6B0200000000004B
:10D9C00010C0B30016F7B70000C4B30017F7B700D4
:10D9D0006C6B02000000000010C0B30016F7B70027
:10D9E00010CAB30017F7B7006C6B0200000000000C
:10D9F00010C0B30016F7B70000CCB30017F7B7009C
:10DA00006C6B02000000000010C0B30016F7B700F6
:10DA1000F0CAB30017F7B7006C6B020000000000FB
:10DA2000400620005C6B02000000000010C0B30044
:10DA300016F7B70070CEB30017F7B7006C6B020093
:10DA4000000000006E6C02000000000020032000B7
:10DA50005C6B02000000000000000600851F7800DB
:10DA60001177EF001277EF001377EF0084B8800092
:10DA700003022000041CE10023003E0084B8800063
:10DA8000F3032000041CE1001F00390084B880006B
:10DA90000442B1000440780011F7B7001377EF009B
:10DAA00094B880004822DE006524E10014003100B3
:10DAB00084B880004822DE006520B800800278002B
:10DAC00094B880004822DE000480420044BA20005E
:10DAD0000400400094B880000042900094B8880090
:10DAE0001677EF0012D7BF0017F7B7006C6B020074
:10DAF000000000001377EC00506D040000000000EF
:10DB0000546E04000000000084B88000030420006C
:10DB1000041CE10023003E0084B88000F3052000CF
:10DB2000041CE1001F00390084B880000444B100E7
:10DB30000440780011F7B7001377EF0094B8800025
:10DB40004822DE006524E1001400310084B8800022
:10DB50004822DE006520B8008002780094B880007A
:10DB60004822DE000480420044C42000040040003B
:10DB700094B880000042900094B888001677EF00B7
:10DB800012D7BF0017F7B7006C6B0200000000004F
:10DB90001377EC009E6D040000000000546E04003A
:10DBA0000000000084B8800003062000041CE1008F
:10DBB00023003E0084B88000F3072000041CE1002D
:10DBC0001F00390084B880000446B100044078008A
:10DBD00011F7B7001377EF0094B880004822DE00F9
:10DBE0006524E1001400310084B880004822DE0082
:10DBF0006520B8008002780094B880004822DE00DA
:10DC00000480420044CE20000400400094B880000C
:10DC10000042900094B888001677EF0012D7BF003A
:10DC200017F7B7006C6B0200000000001377EC00E0
:10DC3000EC6D040000000000546E040000000000C1
:10DC40001177EF001377EF0094B880004822DE00D0
:10DC50006524E1001400310084B880004822DE0011
:10DC60006520B8008002780094B880004822DE0069
:10DC70000480420044BA20000400400094B88000B0
:10DC80000042900094B888001677EF0012D7BF00CA
:10DC900017F7B7006C6B0200000000001377EC0070
:10DCA000246E04000000000010C0B30000E0B700C4
:10DCB000CF027800000006000977EF000A77EF0036
:10DCC00004D7BF0010F7B700A06B020000000000EF
:10DCD00005D7BF0010F7B700CC6B020000000000B2
:10DCE0000977EF0009D7BF0044B880000024E100A5
:10DCF0001600360044B880004822DE000400780098
:10DD00000617B40054B880000042900054B8880050
:10DD10000AD7BF0010F7B7002E6D02000000000008
:10DD20001677EF001777EF006C6B02000000000021
:10DD30001677EF001777EF006C6B02000000000011
:10DD40000977EC00726E040000000000000006007D
:10DD5000851F7800C500200003000900B51F78006A
:10DD600000027800810278000203780083037800C3
:10DD70000000EB008000EB000001EB008001EB00F5
:10DD80000800A10007F0A600050037000800A00069
:10DD90000402EA008582EA000683EA008783EA003B
:10DDA0008504720002003A008704730015003200F7
:10DDB000394720000340A7000B0037004200A900AC
:10DDC0000482D2008582D2000683D2008783D200EB
:10DDD0000080D2008180D2000281D2008381D200F3
:10DDE0008904E900F3FF3A00C44CDD004200A900B9
:10DDF00009F0A1000340A10083816C000800A70086
:10DE000003F0A0002501200003000900CF127800D4
:10DE1000CF02780000000600881F7800280120004B
:10DE200004000900B81F78008005EB006066B800A8
:10DE30000304780087047800FA7F20004200A900DC
:10DE40004220A90044C4DE00080465000800E00088
:10DE5000700032004200A9004220A900C4CCDE00BC
:10DE6000890465000900E0006A003200088444006B
:10DE700009B0A70004003700F83FB1006500320088
:10DE800064003900030037001A4020008542450035
:10DE900060003100878669004200A9004220A90085
:10DEA000F300B2000340A000F700B2000740A0005A
:10DEB000881F78000124B800002DB8000A0544002E
:10DEC0008B854C000C80B0000224B8008B05440008
:10DED0000C864C00012CB8008B0544000C864C00CD
:10DEE0000034B8000005EB008B0544000C864C00A4
:10DEF0000A80B0008005EB000324B8000C06440043
:10DF00000A854C000B80B000022CB8000C064400BF
:10DF10000A854C000B80B0000134B8000C064400A8
:10DF20000A854C000B80B000003CB8000C06440091
:10DF30000A854C000B80B0000C0078000006EB0056
:10DF4000032CB8000A0544008B854C000C80B000FF
:10DF50000234B8000A0544008B854C000C80B000E8
:10DF60000334B8008B0544000C864C00013CB8001B
:10DF70000A0544008B854C000C80B000023CB800C0
:10DF80008B0544000C864C00033CB8000C06440092
:10DF90008A0078000B0178008C0178005400200082
:10DFA0004200A9008381D3000281D3008180D30085
:10DFB0000080D3000402E900F9FF3A004F04780022
:10DFC0000804E8000103700001003200020037007D
:10DFD00003037100080032000340A7000600370069
:10DFE0004200A9000080D2008180D2000281D200CC
:10DFF0008381D2000804E9004444DD0003F0A1005D
:10E000000DF0A70003F0A0000340A10083016C0005
:10E01000030037006000B8006001B800000037005E
:10E02000A8012000040009004F1478004F04780074
:10E0300000000600881F7800280120000400090065
:10E04000B81F780087866900030478008704780089
:10E05000FA7F20004200A9004220A90044C4DE004B
:10E06000080465000800E0006C0032004200A900CE
:10E070004220A900C4CCDE00890465000900E0004C
:10E08000660032000005EB00090654000300390069
:10E09000FC3FB00061003100040037001B4020004D
:10E0A0000B0656005D0039005C0032000004EB00F6
:10E0B0008004EB000005EB008005EB00F301B200EB
:10E0C0000340A000F701B2000740A0008C1F7800B9
:10E0D0006C032000040050008580580006015900A0
:10E0E00087815900020033000600310006003A0023
:10E0F00004004000858048000601490087814900EE
:10E10000010037000800A0000C06E9000B003200F7
:10E110004200A9000080D2008180D2000281D2009A
:10E120008381D2004200A9000884D2008984D200F1
:10E130000A85D2008B85D200E6FF37004F067800B3
:10E140000B50A70001003700060037004200A9006D
:10E150008B85D3000A85D3008984D3000884D3003B
:10E16000030037000C06E9004200A9002B00320032
:10E170004200AF00090037000080D2008180D20049
:10E180000281D2008381D2000402500085825800AF
:10E190000603590087835900150039000804E80078
:10E1A00013003A008904E80011003A000A05E8006B
:10E1B0000F003A008B05E8000D003A000C06E8005D
:10E1C000160032000A0037000C06E9001300320086
:10E1D0000B40A700060037004200A9000884D200C7
:10E1E0008984D2000A85D2008B85D200F8FF3700DF
:10E1F0004466DD004200A9000CF0A1000DF0A7006C
:10E200000CF0A0000B40A1008B016E000A01780009
:10E210008900780008007800050037000000200021
:10E220000100200002002000030020000000370051
:10E23000A8012000040009004F1478004F04780062
:10E2400000000600851F7800861F78000302780012
:10E25000030378004200A90044A2DE00F57F2000FD
:10E260000482620003003A006000B8000001EB0085
:10E27000130037000438B100F300B200370020006B
:10E280004200A9000080D2008180D2000281D20029
:10E290008381D2008703E900F9FF3A00010078008A
:10E2A000820078000370A1000480FD004200A900F4
:10E2B0000482D30006F0A70004F0A00003016A0066
:10E2C0004F037800CF02780000000600811F78001D
:10E2D000F18E8000805878008048EB00CF007800F5
:10E2E000DE31EC0000000600851F78008201780016
:10E2F000820278004200A9008381D2000380FD00E1
:10E30000F30FB20003003A006000B8006011B800DB
:10E31000160037000338B000F207B20036002000C4
:10E320000002EB004200A9000281D3008180D300EB
:10E330000080D3004200AF000402E8000603E900B9
:10E34000F8FF3A000270A100C419DD0003F0A1003B
:10E3500005F0A70003F0A000830169000101780027
:10E3600080007800810042000000EB00CF027800BE
:10E3700000000600851F7800C50020000500090088
:10E38000B51F780003047800820378000103780049
:10E3900080027800830478003B472000C499DE00A7
:10E3A000FA7F20008301650083855500F801B200E3
:10E3B0000840A0000000EB008000EB000001EB0033
:10E3C0008001EB004200A9000884D3008783D300BA
:10E3D0000683D3008582D3008381D3000281D300DA
:10E3E0008180D3000080D3008B05E900F5FF3A005F
:10E3F00009F0A600050037000000EA008180EA006D
:10E400000281EA008381EA000000370065012000F4
:10E4100005000900CF127800CF0278000000060046
:10E420008C1F78008D1F78000004EB008004EB0047
:10E430000005EB008005EB000006EB008006EB001A
:10E44000E8002000090020001000FA000C377C00D2
:10E450000884E900FDFF3B0005046A0002003A0061
:10E4600007046B002F0032000004EB000D042000B5
:10E470000D0420004200A9000080D2008180D2005B
:10E480000281D2008381D2000884D2008984D20024
:10E490000A85D2008B85D2000758E10005003A00BA
:10E4A00006D0E10003003A0005C8E10001003A008F
:10E4B00004C0E100050039000404540085845C00B8
:10E4C00006055D0087855D004200A800080F780002
:10E4D000190798002A0798003B0798004E049000FF
:10E4E000DE0490006E059000FE0590000884D200C6
:10E4F0008984D2000A85D2008B85D2004807980013
:10E50000590798006A0798007B0798001E04780056
:10E510009E0490002E059000BE0590008D06E90037
:10E52000D4FF3A004E009000DE0090006E01900093
:10E53000FE0190000080FA0000003700CF0678004E
:10E540004F06780000000600851F7800C5002000F7
:10E5500007000900B51F78002A00FA008802200091
:10E560000006EB000C377C000884E900FDFF3B004F
:10E570000900E0000E003200391798004A17980091
:10E58000470224000003EB006022B800291798001E
:10E59000470224000003EB006022B8000C6F020069
:10E5A00000000000AE1490008904E900F7FF3A0073
:10E5B000BE1490004001200020179800D71C2400B2
:10E5C00056D62C006022B800000F9800110F98005A
:10E5D000220F9800330F9800480120000817980078
:10E5E00004002000859E28004630220077AC2800D9
:10E5F000440F9800550F9800660F9800770F980009
:10E6000003F0A600040037004E1490000804E9004F
:10E6100008D0A0004817980003F0A100BA710200CA
:10E62000000000004E149000BE1490000900E000AD
:10E630004220AF000844E800481798009E1490005C
:10E640008004EB00191798004E0A9000DE0A900033
:10E650006E0B9000FE0B9000107202000000000094
:10E660009E1690000D00A70060003700080F98006C
:10E67000190F98002A0F98003B0F98009E169000E3
:10E680000D00A2001D1798000000E00012003A00E3
:10E69000BE1490008904E8002E159000090455006E
:10E6A0000D003200CE1590000B00E0000E0032008D
:10E6B0007F84650008045500010032003F003100EE
:10E6C0000BF0A7003D0037000BE0A7000600370065
:10E6D0000002200034003700CE1590000C0022000C
:10E6E0008B0566004B179800CE1590000BD0A60046
:10E6F0000E0037000BD0A100BE1490000900E0000E
:10E700004220AE008B05E9008005EB004B17980016
:10E7100000057800D0C2B30066710200000000005E
:10E720000A0078008005EB004B179800BE1490009B
:10E730002E159000090455000B003A008005EB00EF
:10E740004B17980000057800E0C2B3006671020024
:10E7500000000000CE1590000C0022008B05660022
:10E760004B1798000A00780001032000CE15900096
:10E770000BD0A6000C0037000BD0A100BE149000F7
:10E780000900E0004220AE008B05E9008005EB00A7
:10E790004B179800D0C2B300667102000000000061
:10E7A0000000EB000103200000804000801F780083
:10E7B0004F0078006671020000000000AE16900065
:10E7C0008D06E900190032002D1798004E089000C0
:10E7D000DE0890006E099000FE099000A400200061
:10E7E0008002EB006033B8009BFF3700400F9800B9
:10E7F000510F9800620F9800730F98000002780084
:10E800008102780002037800830378000E089000EC
:10E810009E0890002E099000BE0990009E16900060
:10E820000D00A2001D1798008BFF37000080FA0032
:10E83000A501200007000900CF127800CF02780060
:10E8400000000600851F7800E462A8001E00090091
:10E8500000000000E442A8001F00090000000000C2
:10E86000E642AE00FEFF3700E862A900E462A900BC
:10E870001E00090000000000E842A900E442A900CF
:10E880004200F80042E0EF00A1188100165D02008E
:10E89000000000004200F9004200F80042E0EF00F2
:10E8A000B1188100165D0200000000004200F9006E
:10E8B000C51881004200F80042E0EF008540780072
:10E8C000165D0200000000004200F900E462A900A9
:10E8D00000000000E442A800E642AE00FEFF370060
:10E8E0001E000900000000000100090000000000F7
:10E8F000E462A8001E00090000000000CF027800BA
:10E900000000060083002000E462A8001F00090048
:10E9100000000000E442A800E642AE00FEFF37001F
:10E92000E662AF004200A800E662AE004200A90025
:10E930000281D2001E00090000000000E442A9008C
:10E94000E842A9008301E900EFFF3A00E462A80071
:10E950001F00090000000000E862A9000100E000BB
:10E960004220AE00E462A90000000000E442A800DA
:10E97000E642AE00FEFF37001E0009000000000066
:10E98000E842A900E442A9001F00090000000000BD
:10E99000E862A900E462A900020078000000060015
:10E9A000851F7800B833EF00E462A8001E0009005C
:10E9B00000000000E442A8001F0009000000000061
:10E9C000E642AE00FEFF3700E862A900E462A9005B
:10E9D0001E00090000000000E842A900E442A9006E
:10E9E000A59D8000E50FB2004200F80042E0EF0074
:10E9F00085407800165D0200000000004200F9002A
:10EA00004200F80042E0EF00B19D8000165D020078
:10EA1000000000004200F900E462A8001E000900A6
:10EA200000000000E442A8001F00090000000000F0
:10EA3000E642AE00FEFF3700E862A900E462A900EA
:10EA40001E00090000000000E842A900E442A900FD
:10EA5000A09D8000E10270004200F80042E0EF005B
:10EA600085407800165D0200000000004200F900B9
:10EA700001002000811F7800CF007800827402001E
:10EA800000000000B8F3B700B973EF00E462A9001A
:10EA900000000000E442A800E642AE00FEFF37009E
:10EAA0001E00090000000000010009000000000035
:10EAB000E462A8001E00090000000000B8D3BF00F7
:10EAC000CF027800000006002272EF004200F8003A
:10EAD00042E0EF0064042000743389008033810039
:10EAE00080C1B30080338900803381000160EF0072
:10EAF00080338900BA5D0200000000004200F90086
:10EB00004200F80042E0EF00640420007433890002
:10EB10008033810090C1B30080338900803381004D
:10EB20000160EF0080338900BA5D02000000000040
:10EB30004200F9004200F80042E0EF0064042000C7
:10EB40007433890080338100A0C1B3008033890011
:10EB5000803381000160EF0080338900BA5D0200DC
:10EB6000000000004200F9004200F80042E0EF001F
:10EB7000640420007433890080338100B0C1B30085
:10EB800080338900803381000160EF008033890089
:10EB9000BA5D0200000000004200F9004200F800E7
:10EBA00042E0EF0064042000743389008033810068
:10EBB000C0C1B30080338900803381000160EF0061
:10EBC00080338900BA5D0200000000004200F900B5
:10EBD0004200F80042E0EF00640420007433890032
:10EBE0008033810000C2B30080338900803381000C
:10EBF00001E0EF0080338900BA5D020000000000F0
:10EC00004200F9004200F80042E0EF0064042000F6
:10EC1000743389008033810010C2B30080338900CF
:10EC20008033810001E0EF0080338900BA5D02008B
:10EC3000000000004200F9004200F80042E0EF004E
:10EC400064042000743389008033810020C2B30043
:10EC5000803389008033810001E0EF008033890038
:10EC6000BA5D0200000000004200F9004200F80016
:10EC700042E0EF0064042000743389008033810097
:10EC800030C2B300803389008033810001E0EF009F
:10EC900080338900BA5D0200000000004200F900E4
:10ECA0004200F80042E0EF00640420007433890061
:10ECB0008033810040C2B3008033890080338100FB
:10ECC00001E0EF0080338900BA5D0200000000001F
:10ECD0004200F900C40F2000B45388004200F8003D
:10ECE00042E0EF0064042000743389008033810027
:10ECF00080C0B3008033890076CABF007026F80058
:10ED0000F0FF9F007026F900BA5D020000000000CD
:10ED10004200F900F40F2000C45388004200F800BC
:10ED200042E0EF00640420007433890080338100E6
:10ED300090C0B3008033890078CABF007026F80005
:10ED4000F0FF9F007026F900BA5D0200000000008D
:10ED50004200F900F40F2000D45388004200F8006C
:10ED600042E0EF00640420007433890080338100A6
:10ED7000A0C0B300803389007ACABF007026F800B3
:10ED8000F0FF9F007026F900BA5D0200000000004D
:10ED90004200F900F40F2000E45388004200F8001C
:10EDA00042E0EF0064042000743389008033810066
:10EDB000B0C0B300803389007CCABF007026F80061
:10EDC000F0FF9F007026F900BA5D0200000000000D
:10EDD0004200F900F40F2000F45388004200F800CC
:10EDE00042E0EF0064042000743389008033810026
:10EDF000C0C0B300803389007ECABF007026F8000F
:10EE0000F0FF9F007026F900BA5D020000000000CC
:10EE10004200F9004200F80042E0EF0084042000C4
:10EE2000743389008033810080C1B300803389004E
:10EE3000803381000160EF0080338900BA5D0200F9
:10EE4000000000004200F9004200F80042E0EF003C
:10EE500084042000743389008033810090C1B300A2
:10EE600080338900803381000160EF0080338900A6
:10EE7000BA5D0200000000004200F9004200F80004
:10EE800042E0EF0084042000743389008033810065
:10EE9000A0C1B30080338900803381000160EF009E
:10EEA00080338900BA5D0200000000004200F900D2
:10EEB0004200F80042E0EF0084042000743389002F
:10EEC00080338100B0C1B30080338900803381007A
:10EED0000160EF0080338900BA5D0200000000008D
:10EEE0004200F9004200F80042E0EF0084042000F4
:10EEF0007433890080338100C0C1B300803389003E
:10EF0000803381000160EF0080338900BA5D020028
:10EF1000000000004200F9004200F80042E0EF006B
:10EF200084042000743389008033810000C2B30060
:10EF3000803389008033810001E0EF008033890055
:10EF4000BA5D0200000000004200F9004200F80033
:10EF500042E0EF0084042000743389008033810094
:10EF600010C2B300803389008033810001E0EF00DC
:10EF700080338900BA5D0200000000004200F90001
:10EF80004200F80042E0EF0084042000743389005E
:10EF90008033810020C2B300803389008033810038
:10EFA00001E0EF0080338900BA5D0200000000003C
:10EFB0004200F9004200F80042E0EF008404200023
:10EFC000743389008033810030C2B30080338900FC
:10EFD0008033810001E0EF0080338900BA5D0200D8
:10EFE000000000004200F9004200F80042E0EF009B
:10EFF00084042000743389008033810040C2B30050
:10F00000803389008033810001E0EF008033890084
:10F01000BA5D0200000000004200F900F40F200079
:10F02000045488004200F80042E0EF00840420000D
:10F03000743389008033810080C0B300803389003D
:10F0400080CABF007026F800F0FF9F007026F9000C
:10F05000BA5D0200000000004200F900F401200047
:10F06000145488004200F80042E0EF0084042000BD
:10F07000743389008033810090C0B30080338900ED
:10F0800082CABF007026F800F0FF9F007026F900CA
:10F09000BA5D0200000000004200F900C40F200029
:10F0A000245488004200F80042E0EF00840420006D
:10F0B0007433890080338100A0C0B300803389009D
:10F0C00084CABF007026F800F0FF9F007026F90088
:10F0D000BA5D0200000000004200F900C4002000F8
:10F0E000345488004200F80042E0EF00840420001D
:10F0F0007433890080338100B0C0B300803389004D
:10F1000086CABF007026F800F0FF9F007026F90045
:10F11000BA5D0200000000004200F9004404200033
:10F12000A418890084012000B4188900D40F20009D
:10F13000C41889002274020000000000440420006A
:10F14000A418890094012000B4188900F40F20004D
:10F15000C41889002274020000000000440420004A
:10F16000A4188900A4012000B4188900F40F20001D
:10F17000C41889002274020000000000440420002A
:10F18000A4188900B4012000B4188900F40F2000ED
:10F19000C41889002274020000000000440420000A
:10F1A000A4188900C4012000B4188900F40F2000BD
:10F1B000C4188900227402000000000044042000EA
:10F1C000A418890004022000B4188900240020003B
:10F1D000C4188900227402000000000044042000CA
:10F1E000A418890014022000B4188900040020002B
:10F1F000C4188900227402000000000044042000AA
:10F20000A418890024022000B418890004002000FA
:10F21000C418890022740200000000004404200089
:10F22000A418890034022000B418890004002000CA
:10F23000C418890022740200000000004404200069
:10F24000A418890044022000B4188900040020009A
:10F25000C41889002274020000000000C4042000C9
:10F26000A418890084012000B4188900F40F20003C
:10F27000C41889002274020000000000C4042000A9
:10F28000A418890094012000B4188900F40F20000C
:10F29000C41889002274020000000000C404200089
:10F2A000A4188900A4012000B4188900F40F2000DC
:10F2B000C41889002274020000000000C404200069
:10F2C000A4188900B4012000B4188900E40F2000BC
:10F2D000C41889002274020000000000C404200049
:10F2E000A4188900C4012000B4188900F40F20007C
:10F2F000C41889002274020000000000C404200029
:10F30000A418890004022000B41889000400200019
:10F31000C41889002274020000000000C404200008
:10F32000A418890014022000B418890004002000E9
:10F33000C41889002274020000000000C4042000E8
:10F34000A418890024022000B418890004002000B9
:10F35000C41889002274020000000000C4042000C8
:10F36000A418890034022000B41889001400200079
:10F37000C41889002274020000000000C4042000A8
:10F38000A418890044022000B41889000400200059
:10F39000C41889002274020000000000C404200088
:10F3A000A49D880034002000B49D8800D074020021
:10F3B0000000000088EAB700896AEF00445480002A
:10F3C000040FB20044548800C4042000A49D8800A7
:10F3D00044002000B49D8800D074020000000000AA
:10F3E0008AEAB7008B6AEF0044042000A49D8800DD
:10F3F000B633EF00D07402000000000022F2B70024
:10F4000044042000A49D880014002000B49D8800BE
:10F41000D07402000000000022F2B7004404200073
:10F42000A49D880024002000B49D8800D0740200B0
:10F430000000000022F2B70044042000A49D8800D0
:10F4400034002000B49D8800D07402000000000049
:10F4500022F2B70044042000A49D8800440020004C
:10F46000B49D8800D07402000000000022F2B700B2
:10F47000C4042000A49D8800B633EF00D0740200BD
:10F480000000000022F2B700C4042000A49D880000
:10F4900014002000B49D8800D07402000000000019
:10F4A00022F2B700C4042000A49D8800240020009C
:10F4B000B49D8800D07402000000000022F2B70062
:10F4C000C4042000A49D880034002000B49D88005E
:10F4D000D07402000000000022F2B700C404200033
:10F4E000A49D880044002000B49D8800D0740200D0
:10F4F0000000000022F2B70000000600851F78001F
:10F500006432EF00A348E20004003A0040CBB300AD
:10F5100018E9B700927A04000000000040C3B3006D
:10F5200018E9B70000C1B30019E9B70040C0B30043
:10F530001AE9B7001B69EF00A0C0B3001CE9B700CF
:10F5400010C0B3001EE9B70010C0B3001FE9B70038
:10F5500020C1B30021E9B700F0C0B30020E9B70033
:10F5600040C0B30022E9B70040C0B30023E9B700B0
:10F5700040C0B30024E9B70090C1B30025E9B7004B
:10F5800040C1B30046E9B70040C1B30047E9B70046
:10F5900040C1B30048E9B7002E69EF002F69EF00C2
:10F5A0003069EF0080C1B30031E9B70080C1B3001A
:10F5B00032E9B70080C1B30033E9B70080C1B300BE
:10F5C00034E9B70080C1B30035E9B70080C1B300AA
:10F5D00036E9B70080C1B30037E9B70040C1B300D6
:10F5E00038E9B70040C1B30039E9B70040C1B30002
:10F5F0003AE9B70040C1B3003BE9B70040C1B300EE
:10F600003CE9B70040C1B3003DE9B70040C1B300D9
:10F610003EE9B70070C0B3003FE9B70070C0B30067
:10F6200040E9B70070C0B30041E9B70070C0B30053
:10F6300042E9B70070C0B30043E9B70070C0B3003F
:10F6400044E9B70070C0B30045E9B70020C0B3007B
:10F6500049E9B70020C0B3004AE9B70020C0B300B1
:10F660004BE9B70020C0B3004CE9B70020C0B3009D
:10F670004DE9B70020C0B3004EE9B70020C0B30089
:10F680004FE9B70020C0B30050E9B70020C0B30075
:10F6900051E9B7002669EF002769EF002869EF00FC
:10F6A0002969EF002A69EF002B69EF0010C0B30051
:10F6B0002CE9B70010C0B3002DE9B70000C1B300BA
:10F6C0001DE9B7005269EF005369EF005469EF007C
:10F6D0005569EF005669EF005769EF005869EF0070
:10F6E00050C3B30059E9B7006432EF00249380009F
:10F6F0006D20E100070031008496200023938000F4
:10F7000084824100804AEB006432EC00767B040086
:10F7100000000000CF02780000000600851F78007E
:10F72000E462A8001E00090000000000E442A800F6
:10F730001F00090000000000E642AE00FEFF370097
:10F74000E862A900E462A9001E00090000000000B0
:10F75000E842A900E442A9009E0009000000000060
:10F76000A018810080027800E50FB2004200F80086
:10F7700042E0EF0085407800165D020000000000C6
:10F780004200F9009E00090000000000B518810049
:10F790004200F80042E0EF0085407800165D02006C
:10F7A000000000004200F9009E0009000000000077
:10F7B000E462A90000000000E442A800E642AE00B6
:10F7C000FEFF37001E0009000000000001000900D4
:10F7D00000000000E462A8001E0009000000000014
:10F7E000BE00090000000000CF0278000000060003
:10F7F000851F78009033EF0014002000849C88005F
:10F80000849C80006720E100140031000000370074
:10F81000849C80006702420084027800040E20006D
:10F82000A4188900B51889008E7B02000000000032
:10F83000A4092000A4188900E4012000B41889005C
:10F84000640B2000C418890022740200000000002C
:10F850009033EC00007C040000000000D3E2A9001B
:10F86000D7E2A80014002000849C8800849C8000BB
:10F870006720E1001A00310000003700849C8000FE
:10F880006702420084027800040E2000A418890058
:10F89000B51889008E7B0200000000005000200097
:10F8A0005C6B02000000000024042000A418890002
:10F8B000F4002000B418890044042000C418890012
:10F8C0002274020000000000500020005C6B020067
:10F8D000000000009033EC00367C040000000000C3
:10F8E000CF02780000000600AA33EF00AC33EF002F
:10F8F000AE73EF00AF73EF00B073EF00449D800074
:10F90000F37F20000418E100020031000060EF00E6
:10F9100028003700449D8000F30F20000418E10008
:10F9200005003600AA33EF00A813F800AC13F90065
:10F93000B27C040000000000449D8000F30F200012
:10F94000110009000382D800509D8800549D80005A
:10F95000F30F20000320B800449D800000005200F7
:10F96000609D8800ACD3BF00AFF3B700AA33D400CA
:10F97000040A2000539D800004804100509D8800AF
:10F98000AAD3BF00B0F3B700B0D3BF00B4F3B70041
:10F99000B573EF00AFD3BF00B6F3B700B773EF0096
:10F9A000D074020000000000AEF3B700AED3BF0079
:10F9B00000E0B70000000600851F78003E52E2001C
:10F9C00021003200D091800090427800E0918000C8
:10F9D0000002780014407800002CE1000E00320094
:10F9E000D091800090427800E09180000002780081
:10F9F00014407800002CE1000300310000C0EB004F
:10FA0000067D04000000000010C0B3000F003700A6
:10FA1000167D040000000000D09180001004E0007A
:10FA200002003A000060EF0008003700D09180002B
:10FA30003A32EC00E09180003C32EC003E72ED0086
:10FA4000DE7C0400000000000060EF00CF027800C0
:10FA500000000600851F78002232EF002472EF00BC
:10FA60002572EF0004022200349188000402220073
:10FA7000449188000402220054918800040222006C
:10FA8000649188000402220074918800040222001C
:10FA900084918800040222009491880004022200CC
:10FAA000A491880004022200B49188003872EF000B
:10FAB000F47C2000149188002472EF0024918000CF
:10FAC0007224E10014003D002212F800A813F9008E
:10FAD000747C02000000000025F2B70050002000F6
:10FAE0005C6B02000000000024D2BF000000FB009D
:10FAF000642221008402400025D2BF00804A7800A1
:10FB00001491800061024200149188002472EC007C
:10FB10005E7D0400000000003872EF0020C1B300D9
:10FB20003EF2B70064222100D4918800448A20006C
:10FB3000E4918800DC7C0200000000000004E0008A
:10FB400005003A0010C0B30000E0B7000400370021
:10FB5000B07D04000000000000E0EF00000037006E
:10FB6000CF02780000000600851F78000417F80017
:10FB70000A17F9000857E2000C00320030B8800084
:10FB80001004E0000900320050B880000A37EC0091
:10FB90008002780030B880000637EC00904A780088
:10FBA0000877ED00BA7D0400000000000857E2006D
:10FBB0000700320050B880000A37EC00800278005D
:10FBC000804AEB000877ED00D67D040000000000BD
:10FBD0000417F8000000F900CF02780000000600CA
:10FBE000016F210002002000120009008058EB0084
:10FBF00020C1B30008F7B700046F210024B88800C3
:10FC0000EE16F8000617F900B47D020000000000AF
:10FC100070C0B30004F7B7000577EF0020C1B30050
:10FC200008F7B700046F210034B888005C6E02004A
:10FC300000000000000006009E32EF00A032EF003E
:10FC40009D72EF00A272EF00D4948000F37F200039
:10FC50000418E1000100310038003700D49480001E
:10FC6000F30F20000418E100050036009E32EF007B
:10FC70009A12F800A012F900587E0400000000005B
:10FC8000D4948000F30F2000110009000382D800F3
:10FC90009EF2B7009F72EF00F4948000F30F2000F3
:10FCA0000320B800D4948000000052000095880022
:10FCB000A0D2BF009DF2B7009E32D400040A2000FB
:10FCC000F394800004804100F09488009ED2BF002D
:10FCD000A2F2B700A2D2BF001423F800E0FF9F00F9
:10FCE0001423F900A01881000160EF00A01889001A
:10FCF0009DD2BF001623F800E0FF9F001623F900F5
:10FD0000B01881000160EF00B01889009CD2BF00DC
:10FD10001823F800E0FF9F001823F900C0188100A5
:10FD20000160EF00C018890022740200000000008A
:10FD3000500020005C6B0200000000000000060084
:10FD40009C32EF009B72EF009C32EF00E094800049
:10FD5000D49480000960EF000020E1000B00360021
:10FD6000E09480009812B4000002780014407800FB
:10FD70009B72B400500020005C6B02000000000089
:10FD80009C32EC00A67E040000000000D4948000A9
:10FD90004822DE00F4CFB200044078009BF2B700A6
:10FDA000D49480004822DE00614242000440780082
:10FDB0009BF2B7009BD2BF0000000600851F7800B1
:10FDC0007E32EF007D72EF009472EF009512A90071
:10FDD0007E32EF00F0938000E49380000960EF0032
:10FDE0000020E1001F0036007E12F800A813F90081
:10FDF000747C02000000000094F2B700F0938000D1
:10FE00007A12B40000027800144078009452E300A3
:10FE100011003200A00020005C6B02000000000016
:10FE2000F09380007A12B400904278009C12F8009F
:10FE3000E5FF9F009C12F9007E12F8009A12F9006B
:10FE40001C7E020000000000A00020005C6B02008D
:10FE5000000000009512A8007E32EC00EA7E04004B
:10FE6000000000009512AE003A00370002002000AA
:10FE70000128210002007800320402000000000086
:10FE8000805878000201E8000004E0004220AE0043
:10FE9000F8FF37000428210074B78800F07D0200C5
:10FEA000000000001929AE000D00370001002000FD
:10FEB0000100780052040200000000008100E80008
:10FEC000811F78002322AF00FEFF37002011880039
:10FED000CF007800D00020000008E600F4FF3700D3
:10FEE0007CD2BF009AF2B7007A12F8009812F9009B
:10FEF000A07E0200000000007DF2B7007CD2BF00AF
:10FF0000A8F3B700A973EF00747C020000000000A2
:10FF100094F2B70094D2BF007D52E3000D0032008E
:10FF2000A00020005C6B0200000000007CD2BF003B
:10FF30009AF2B7009B72EF007DD2BF009CF2B7002F
:10FF40001C7E020000000000A00020005C6B02008C
:10FF500000000000CF02780000000600851F780036
:10FF6000861F78000001EB000103780064C11000D7
:10FF70004211DD000200DD00800278000C60EC0020
:10FF80000C60ED000D00320005007800C42ADD0091
:10FF90004C00DE00F000B2000003B000A20320001D
:10FFA0000200E100010039000D40B4002322AF003F
:10FFB000FEFF370020118800F1FF37004F03780063
:10FFC000CF02780000000600851F78007E32EF0027
:10FFD0008032EF007D72EF008272EF008032EF001E
:10FFE000049480006220E100550031007E32EF0071
:10FFF000F0938000E49380000960EF000020E100AE
:020000040001F9
:100000000E003600F09380007A12B400800278006F
:100010007E12F800A813F900747C020000000000B2
:10002000804A7800500020005C6B02000000000055
:100030007E32EC00F87F0400000000007CD2BF009C
:10004000A8F3B700A973EF00747C02000000000061
:1000500082F2B7007CD2BF009AF2B7007A12F800A1
:100060009812F900A07E0200000000007DF2B700A7
:1000700082D2BF007D52E3002E003200010020003A
:100080000100780002040200000000008100E80086
:10009000811F78002322AF00FEFF37002011880067
:1000A000CF007800D00020000008E600F4FF370001
:1000B00082D2BF000160EF0021702200AE7F0200FB
:1000C000000000001101200001007800020402007D
:1000D000000000008100E800811F78002322AF00AB
:1000E000FEFF370020118800CF007800D0012000EB
:1000F0000008E600F4FF37007DD2BF000160EF008A
:1001000021702200AE7F0200000000002322AF0019
:10011000FEFF3700A4002000241188002322AF0036
:10012000FEFF3700D4002000241188000060EF009B
:10013000050037008032EC00F07F04000000000072
:1001400010C0B30000E0B700CF0278000000060046
:10015000851F78007A32EF007C32EF007E32EF00AC
:100160008032EF0004052000D49388007C32EF0039
:10017000E49380006620E1001B0031007E32EF0036
:10018000F49380006C20E100140031008032EF0015
:10019000049480006E20E1000D003100D0938000B7
:1001A0007A32EC00800278009C72EF00D5948800CF
:1001B0001C7E020000000000500020005C6B02006A
:1001C000000000008032EC00C88004000000000045
:1001D0007E32EC00C0800400000000007C32EC00A5
:1001E000B8800400000000007C32EF00E49380003F
:1001F0006D20E1000700310084962000E393800029
:1002000084824100804AEB007C32EC00F6800400DE
:100210000000000034042000D49388007C32EF00FA
:10022000E49380006D20E1000D003100D093800048
:100230007A32EC00800278009CF2EF00D5948800BE
:100240001C7E020000000000500020005C6B0200D9
:10025000000000007C32EC0010810400000000006F
:10026000CF02780000000600851F78002632EF00DC
:100270002832EF002A32EF00041323007493880021
:10028000D4A224008493880054E726009493880025
:10029000D4022300A493880094032000B493880020
:1002A0007872EF00A348E20004003A0040CBB300AC
:1002B0002CF2B700628104000000000040C3B300CC
:1002C0002CF2B70000C1B3002DF2B70040C0B3005C
:1002D0002EF2B7002F72EF00A0C0B30030F2B700CB
:1002E00010C0B30031F2B70010C0B30032F2B70053
:1002F00020C1B30033F2B700F0C0B30034F2B7004E
:1003000040C0B30035F2B70040C0B30036F2B700CA
:1003100040C0B30037F2B70090C1B30038F2B70065
:1003200040C1B30039F2B70040C1B3003AF2B700A0
:1003300040C1B3003BF2B7003C72EF003D72EF00EA
:100340003E72EF0080C1B3003FF2B70080C1B3003E
:1003500040F2B70080C1B30041F2B70080C1B300E2
:1003600042F2B70080C1B30043F2B70080C1B300CE
:1003700044F2B70080C1B30045F2B70040C1B300FA
:1003800046F2B70040C1B30047F2B70040C1B30026
:1003900048F2B70040C1B30049F2B70040C1B30012
:1003A0004AF2B70040C1B3004BF2B70040C1B300FE
:1003B0004CF2B70070C0B3004DF2B70070C0B3008C
:1003C0004EF2B70070C0B3004FF2B70070C0B30078
:1003D00050F2B70070C0B30051F2B70070C0B30064
:1003E00052F2B70070C0B30053F2B70020C0B300A0
:1003F00054F2B70020C0B30055F2B70020C0B300DC
:1004000056F2B70020C0B30057F2B70020C0B300C7
:1004100058F2B70020C0B30059F2B70020C0B300B3
:100420005AF2B70020C0B3005BF2B70020C0B3009F
:100430005CF2B7005D72EF005E72EF005F72EF007A
:100440006072EF006172EF006272EF0010C0B300E3
:1004500063F2B70010C0B30064F2B70000C1B3008C
:1004600065F2B7006672EF006772EF006872EF0026
:100470006972EF006A72EF006B72EF006C72EF004E
:1004800050C3B3006DF2B70020C4B3007CF2B700D4
:10049000C4222100D4938800DE7E02000000000008
:1004A00020C4B3007CF2B700C4222100D49388009A
:1004B000E47F0200000000006104E1001B00320044
:1004C00020C4B3007CF2B700C4222100D49388007A
:1004D000DE7E02000000000020C4B3007CF2B70002
:1004E000C4222100D4938800E47F020000000000B1
:1004F0006104E1000D0032000100200001007800DD
:100500006E040200000000008100E800811F7800F6
:100510002322AF00FEFF370020118800CF007800B3
:10052000D00120000008E600F4FF3700A880020098
:1005300000000000F47C2000349188002A32EF0093
:10054000549180007320E10017003100448A20009C
:100550005391800004804100C493800000429000C9
:10056000C493880078D2BF009CF2B7002612F8002E
:100570009A12F9001C7E0200000000002612F8000A
:10058000A813F900747C02000000000078F2B700A4
:100590003491800061024200349188002A32EC00DC
:1005A000A082040000000000147E20003491880026
:1005B0002832EF002A32EF00549180007320E100CE
:1005C00032003100048920005391800004804100F2
:1005D00090427800040320000524E10004003E005E
:1005E000940320000524E1000100390003003700D6
:1005F0000040EB00008304000000000010C0B300C6
:100600006104E1001E003A00449180006520E10091
:100610001B003E00048920005391800004804100AB
:10062000C493800000429000C493880078D2BF0039
:100630009CF2B7002612F8009A12F9001C7E020004
:1006400000000000500020005C6B02000000000071
:100650002612F800A813F900747C020000000000C4
:1006600078F2B700500020005C6B02000000000030
:100670002832EC00349180006102420034918800FD
:100680002A32EC00DC82040000000000747E2000AE
:10069000349188002A32EF00549180006920E100F3
:1006A0001D003100E42621005391800004804100A8
:1006B000C493800000429000C493880078D2BF00A9
:1006C0009CF2B7002612F8009A12F9001C7E020074
:1006D00000000000500020005C6B020000000000E1
:1006E0002612F800A813F900747C02000000000034
:1006F00078F2B700500020005C6B020000000000A0
:100700003491800061024200349188002A32EC006A
:100710004C83040000000000CF02780000000600B7
:10072000851F780020C4B3007CF2B700242221008A
:10073000D4938800E47F0200000000000004E00081
:100740001A003A0020C4B3007CF2B7002422210032
:10075000D4938800E47F0200000000000004E00061
:1007600012003A001929AE001000370001002000E5
:10077000010078009A040200000000008100E800F7
:10078000811F78002322AF00FEFF37002011880070
:10079000CF007800300120000008E600F4FF3700A9
:1007A0007E7A0200000000008400370022D2BF00E1
:1007B00018E9B70023D2BF0019E9B70024D2BF005F
:1007C0001AE9B70025D2BF001BE9B70026D2BF0047
:1007D0001CE9B70027D2BF001EE9B70028D2BF002E
:1007E0001FE9B70029D2BF0021E9B7002AD2BF0014
:1007F00020E9B7002BD2BF0022E9B7002CD2BF00FE
:1008000023E9B7002DD2BF0024E9B7002ED2BF00E4
:1008100025E9B7002FD2BF0046E9B70030D2BF00AC
:1008200047E9B70031D2BF0048E9B70032D2BF0074
:100830002EE9B70033D2BF002FE9B70034D2BF0092
:1008400030E9B70035D2BF0031E9B70036D2BF007A
:1008500032E9B70037D2BF0033E9B70038D2BF0062
:1008600034E9B70039D2BF0035E9B7003AD2BF004A
:1008700036E9B7003BD2BF0037E9B7003CD2BF0032
:1008800038E9B7003DD2BF0039E9B7003ED2BF001A
:100890003AE9B7003FD2BF003BE9B70040D2BF0002
:1008A0003CE9B70041D2BF003DE9B70042D2BF00EA
:1008B0003EE9B70043D2BF003FE9B70044D2BF00D2
:1008C00040E9B70045D2BF0041E9B70046D2BF00BA
:1008D00042E9B70047D2BF0043E9B70048D2BF00A2
:1008E00044E9B70049D2BF0045E9B7004AD2BF008A
:1008F00049E9B7004BD2BF004AE9B7004CD2BF006C
:100900004BE9B7004DD2BF004CE9B7004ED2BF0053
:100910004DE9B7004FD2BF004EE9B70050D2BF003B
:100920004FE9B70051D2BF0050E9B70052D2BF0023
:1009300051E9B70053D2BF0026E9B70054D2BF0037
:1009400027E9B70055D2BF0028E9B70056D2BF004B
:1009500029E9B70057D2BF002AE9B70058D2BF0033
:100960002BE9B70059D2BF002CE9B7005AD2BF001B
:100970002DE9B7005BD2BF001DE9B7005CD2BF0014
:1009800052E9B7005DD2BF0053E9B7005ED2BF00A5
:1009900054E9B7005FD2BF0055E9B70060D2BF008D
:1009A00056E9B70061D2BF0057E9B70062D2BF0075
:1009B00058E9B70063D2BF0059E9B700CF02780009
:1009C000000006008E2BEF008E0BF800900BF90054
:1009D00001A9200002002000FD0009008058EB0062
:1009E000F849A90000000600851F780097D4BF00D1
:1009F0000160EF001082B200430032001080B200AC
:100A000041003200F083B2003F0032001080B2009B
:100A10003D0032003080B2003B0032001080B20056
:100A2000390032007080B200370032001080B2000E
:100A3000350032003080B200330032001080B20046
:100A400031003200F080B2002F0032001080B2007E
:100A50002D0032003080B2002B0032001080B20036
:100A6000290032007080B200270032001080B200EE
:100A7000250032003080B200230032001080B20026
:100A800021003200F081B2001F0032001080B2005D
:100A90001D0032002080B2001B0032007080B200C6
:100AA000190032001080B200170032003080B2000E
:100AB000150032001080B20013003200F080B20046
:100AC000110032001080B2002A0032003080B200E3
:100AD000280032001080B200260032007080B20080
:100AE000240032001080B200220032003080B200B8
:100AF000200032001080B2001E003200D080B20010
:100B00002A00320042003700B4A480004822DE00F0
:100B1000A38220008302420096D4BF008042980046
:100B2000C4A480006224E100100032009854E20066
:100B300008003A00B4A480004822DE00E3862000CA
:100B40008302420000CEB300804A7800B6850400DC
:100B500000000000B4A480004822DE00E3862000EC
:100B60008302420000CFB300804A78000886040068
:100B700000000000B4A480004822DE00A382200010
:100B80008302420096D4BF0080429800B4A4800043
:100B90004822DE00E38620008302420000CFB3003B
:100BA000804A78000886040000000000C4A4800089
:100BB0006224E10008003A00B4A480004822DE006C
:100BC000A38220008302420096D4BF008042980096
:100BD0000486040000000000B4A480004822DE0067
:100BE000A3822000030042001004E000060032004F
:100BF000B4A480004822DE00E38620008302420085
:100C000000CDB300804A7800088604000000000090
:100C1000CF02780000000600851F7800C500200084
:100C200003000900B51F7800800378008404780071
:100C300004F0A1000400E00006003A0009F0A7005B
:100C400002003700050020001000370005002000DA
:100C50000E003700E64252000B003900000320006E
:100C600009F0A60000022000801F78004F007800E5
:100C700066710200000000008502E900FAFF3B00F7
:100C80005500200001003700840278006400200035
:100C900005E0A00009F0A70005F0A00008712200FF
:100CA000110009008883D8008A8602000000000035
:100CB00081037800883E2000110009008883D80055
:100CC0008A860200000000008103780048062000A8
:100CD000110009008883D8008A8602000000000005
:100CE00081037800A8002000110009008883D80043
:100CF0008A860200000000000003200000C04000BF
:100D0000801F78004F00780066710200000000002C
:100D10001A003700060320000000E0000E003A0031
:100D200005E0A6000D0037000402E9000524E100FB
:100D3000020032004200AF00000006000000E000A8
:100D400005003A0005E0A6000400370005F0A60003
:100D5000060220000100370005E0A100004043002A
:100D6000811F7800801F78004F00780066710200B4
:100D700000000000CF0078000000060025012000E0
:100D800003000900CF127800CF02780000000600AF
:100D9000851F7800C500200003000900B51F7800FA
:100DA000800378008404780004F0A1000400E000CF
:100DB00006003A0009F0A7000200370005002000F5
:100DC0000F003700050020000D003700E6425200FA
:100DD0000A0039000003200009F0A60000022000EC
:100DE0002322AF00FEFF3700201188008502E900B2
:100DF000FBFF3B0055002000010037008402780013
:100E00006400200005E0A00009F0A70005F0A000A4
:100E100008712200110009008883D800428702006F
:100E20000000000081037800883E200011000900C6
:100E30008883D80042870200000000008103780008
:100E400048062000110009008883D800428702006C
:100E50000000000081037800A800200011000900B4
:100E60008883D800428702000000000000032000B1
:100E700000C040002322AF00FEFF37002011880091
:100E800019003700060320000000E0000E003A00C1
:100E900005E0A6000D0037000402E9000524E1008A
:100EA000020032004200AF00000006000000E00037
:100EB00005003A0005E0A6000400370005F0A60092
:100EC000060220000100370005E0A10000404300B9
:100ED000811F78002322AF00FEFF37002011880019
:100EE000CF00780000000600250120000300090063
:100EF000CF127800CF02780000000600851F78002E
:100F00009233EF009473EF009573EF001490280074
:100F1000B49C880024002800C49C880034002E0063
:100F2000D49C880044002800E49C8800545025008C
:100F3000F49C880064002000049D880074D0250083
:100F4000149D880084002000249D88009450250072
:100F5000349D8800A4002000449D8800B400240033
:100F6000549D8800C4002000649D8800D4002400A3
:100F7000749D8800E4002000849D8800F400240013
:100F8000949D880004012000A49D88001401220083
:100F9000B49D880024812100C49D88003401220072
:100FA000D49D880044812100E49D880054A1200044
:100FB000F49D880064412000049E88007441200054
:100FC000149E880084A12200249E880094D12200CF
:100FD000349E8800A4412100449E8800B43127003B
:100FE000549E8800C4F12F00649E8800D48127009D
:100FF000749E8800E4412A00849E8800F4612900E0
:10100000949E880004F22000A49E8800140222000E
:10101000B49E880024222300C49E880034622100EC
:10102000D49E880044822000E49E880054F22C0064
:10103000F49E880064022100049F88007402260048
:10104000149F880084F22B00249F880094222000A3
:10105000349F8800A4022800449F8800B402200026
:10106000549F8800C4022000649F8800D4822E0010
:10107000749F8800E4022E00849F880014502A0088
:10108000949F880024002000A49F880034002E0034
:10109000B49F880044002800C49F88005450250055
:1010A000D49F880064002000E49F880074D025004D
:1010B000F49F88008400200004A08800945025003C
:1010C00014A08800A400200024A08800B4002400FC
:1010D00034A08800C400200044A08800D40024006C
:1010E00054A08800E400200064A08800F4002400DC
:1010F00074A088000401200084A08800140122004C
:1011000094A0880024812100A4A08800340122003A
:10111000B4A0880044812100C4A0880054A120000C
:10112000D4A0880064412000E4A08800744120001D
:10113000F4A0880084A1220004A1880094D1220098
:1011400014A18800A441210024A18800B431270003
:1011500034A18800C4F12F0044A18800D481270065
:1011600054A18800E4412A0064A18800F4612900A8
:1011700074A1880004F2200084A1880014022200D7
:1011800094A1880024222300A4A1880034622100B5
:10119000B4A1880044822000C4A1880054F22C002D
:1011A000D4A1880064022100E4A188007402260012
:1011B000F4A1880084F22B0004A28800942220006D
:1011C00014A28800A402280024A28800B4022000EF
:1011D00034A28800C402200044A28800D4822E00D9
:1011E00054A28800E4022E0064A288001490280013
:1011F00074A288002400280084A2880034002A00F9
:1012000094A2880054502500A4A288006400200005
:10121000B4A2880074D02500C4A2880084002000F5
:10122000D4A2880094502500E4A28800A4002000E5
:10123000F4A28800B400240004A38800C4002000A5
:1012400014A38800D400240024A38800E400200014
:1012500034A38800F400240044A388000401200083
:1012600054A388001401220064A388002481210073
:1012700074A388003401220084A3880044812100E3
:1012800094A3880054A12000A4A3880064412000F6
:10129000B4A3880074412000C4A3880084A1220064
:1012A000D4A3880094D12200E4A38800A4412100A3
:1012B000F4A38800B431270004A48800C4F12F00EF
:1012C00014A48800D481270024A48800E4412A00C3
:1012D00034A48800F461290044A4880004F22000AA
:1012E00054A488001402220064A48800242223004D
:1012F00074A488003462210084A488004482200001
:1013000094A4880054F22C00A4A488006402210054
:10131000B4A4880074022600C4A4880084F22B00C0
:10132000D4A4880094222000E4A48800A402280009
:10133000F4A48800B402200004A58800C4022000A0
:1013400014A58800D4822E0024A58800E4022E0073
:1013500034A58800A834EF0014402A0054A5880062
:1013600024002F0064A5880034002A0074A588009A
:101370005450250084A588006400200094A58800AE
:1013800074D02500A4A5880084002000B4A588009E
:1013900094502500C4A58800A4002000D4A588008E
:1013A000B4002400E4A58800C4002000F4A588004F
:1013B000D400240004A68800E400200014A68800BD
:1013C000F400240024A688000401200034A688002C
:1013D0001401220044A688002481210054A688001C
:1013E0003401220064A688004481210074A688008C
:1013F00054A1200084A688006441200094A688009F
:1014000074412000A4A6880084A12200B4A688000C
:1014100094D12200C4A68800A4412100D4A688004B
:10142000B4312700E4A68800C4F12F00F4A6880098
:10143000D481270004A78800E4412A0014A788006B
:10144000F461290024A7880004F2200034A7880052
:101450001402220044A788002422230054A78800F5
:101460003462210064A788004482200074A78800A9
:1014700054F22C0084A788006402210094A78800FD
:1014800074022600A4A7880084F22B00B4A7880069
:1014900094222000C4A78800A4022800D4A78800B2
:1014A000B4022000E4A78800C4022000F4A788004A
:1014B000D4822E0004A88800E4022E0014A888001C
:1014C0000435EF001470260034A8880024002200A0
:1014D00044A8880034802A0054A8880044002800CA
:1014E00064A888005450250074A888006400200077
:1014F00084A8880074D0250094A888008400200067
:10150000A4A8880094502500B4A88800A400200056
:10151000C4A88800B4002400D4A88800C400200017
:10152000E4A88800D4002400F4A88800E400200087
:1015300004A98800F400240014A9880004012000F4
:1015400024A988001401220034A9880024812100E4
:1015500044A988004481210054A9880054A1200096
:1015600064A988006441200074A9880074412000A7
:1015700084A9880084A1220094A9880094D1220023
:10158000A4A98800A4412100B4A98800B43127008F
:10159000C4A98800C4F12F00D4A98800D4812700F1
:1015A000E4A98800E4412A00F4A98800F461290034
:1015B00004AA880004F2200014AA88001402220061
:1015C00024AA88002422230034AA8800344221005F
:1015D00044AA88004482200054AA880054F22C00B7
:1015E00064AA88006402210074AA8800740226009C
:1015F00084AA880084F22B0094AA880094222000F8
:10160000A4AA8800A4022800B4AA8800B40220007A
:10161000C4AA8800C4022000D4AA8800D4822E0064
:10162000E4AA8800E4022E00F4AA88006035EF00E6
:1016300014B0270014AB880024002C0024AB8800D1
:1016400034802A0034AB88004400280044AB880072
:101650005450250054AB88006400200064AB88001F
:1016600074D0250074AB88008400200084AB88000F
:101670009450250094AB8800A4002000A4AB8800FF
:10168000B4002400B4AB8800C4002000C4AB8800C0
:10169000D4002400D4AB8800E4002000E4AB880030
:1016A000F4002400F4AB88000401200004AC88009E
:1016B0001401220014AC88002481210024AC88008D
:1016C0004481210034AC880054A1200044AC88003F
:1016D0006441200054AC88007441200064AC880050
:1016E00084A1220074AC880094D1220084AC8800CC
:1016F000A441210094AC8800B4312700A4AC880038
:10170000C4F12F00B4AC8800D4812700C4AC880099
:10171000E4412A00D4AC8800F4612900E4AC8800DC
:1017200004F22000F4AC88001402220004AD88000A
:101730002422230014AD88003442210024AD880007
:101740004482200034AD880054F22C0044AD88005F
:101750006402210054AD88007402260064AD880044
:1017600084F22B0074AD88009422200084AD8800A0
:10177000A402280094AD8800B4022000A4AD880023
:10178000C4022000B4AD8800D4822E00C4AD88000D
:10179000E4022E00D4AD8800BC35EF0014202300F5
:1017A000F4AD88002400200004AE8800340022003C
:1017B00014AE880044002C0024AE8800540024009D
:1017C00034AE88006400200044AE88007400240019
:1017D00054AE88008400200064AE88009400240089
:1017E00074AE8800A400200084AE8800B4002000FD
:1017F00094AE8800C4002800A4AE8800D400200065
:10180000B4AE8800E4002800C4AE8800F4002000D4
:10181000D4AE880004012800E4AE880044212000F2
:10182000F4AE880054A1200004AF88006421200099
:1018300014AF88007421200024AF880084012200A6
:1018400034AF88009481200044AF8800A441210077
:1018500054AF8800B431270064AF8800C4F12F0072
:1018600074AF8800D481270084AF8800E441280049
:1018700094AF8800F4612900A4AF880004F220002E
:10188000B4AF880014022200C4AF880024222300D1
:10189000D4AF880034622100E4AF880044422500C0
:1018A000F4AF88005492200004B088006402220043
:1018B00014B0880074022D0024B0880084F22B003C
:1018C00034B088009422200044B08800A40228008C
:1018D00054B08800B402200064B08800C402200024
:1018E00074B08800D4822E0084B08800E4022E00F8
:1018F00094B088001436EF0014402300B4B0880080
:1019000024002800C4B0880034802200D4B08800AD
:1019100044002C00E4B0880054002400F4B0880097
:101920006400200004B188007400240014B1880011
:101930008400200024B188009400240034B1880081
:10194000A400200044B18800B400200054B18800F5
:10195000C400280064B18800D400200074B188005D
:10196000E400280084B18800F400200094B18800CD
:1019700004012800A4B1880044212000B4B18800EB
:1019800054A12000C4B1880064212000D4B1880093
:1019900074212000E4B1880084012200F4B18800A1
:1019A0009481200004B28800A441210014B2880070
:1019B000B431270024B28800C4F12F0034B288006B
:1019C000D481270044B28800E441280054B2880042
:1019D000F461290064B2880004F2200074B2880027
:1019E0001402220084B288002422230094B28800CA
:1019F00034622100A4B2880044422500B4B28800B9
:101A000054922000C4B2880064022200D4B288003C
:101A100074022D00E4B2880084F22B00F4B2880036
:101A20009422200004B38800A402280014B3880084
:101A3000B402200024B38800C402200034B388001C
:101A4000D4822E0044B38800E4022E0054B38800F0
:101A50006C36EF001420240074B3880024002000AA
:101A600084B388003400260094B3880044002C001E
:101A7000A4B3880054202700B4B388006400240075
:101A8000C4B3880074902600D4B3880084002C006E
:101A9000E4B3880094702700F4B38800A400280001
:101AA00004B48800B4D0250014B48800C400200019
:101AB00024B48800D450210034B48800E400240009
:101AC00044B48800F420260054B4880004012000A7
:101AD00064B488004421200074B4880054A120001C
:101AE00084B488006421200094B48800742120000C
:101AF000A4B4880084012200B4B4880094D12000EA
:101B0000C4B48800A4412100D4B48800B4312700B3
:101B1000E4B48800C4F12F00F4B48800D481270015
:101B200004B58800E441280014B58800F461290058
:101B300024B5880004F2200034B588001402220085
:101B400044B588002422230054B5880034A2210023
:101B500064B588004442250074B588005492200082
:101B600084B588006402220094B5880074022D00B8
:101B7000A4B5880084F22B00B4B58800942220001C
:101B8000C4B58800A4022800D4B58800B40220009F
:101B9000E4B58800C4022000F4B58800D4822E0089
:101BA00004B68800E4022E0014B68800C436EF00A4
:101BB0001440250034B688002400200044B6880074
:101BC00034802A0054B6880044002C0064B6880093
:101BD0005420270074B688006400240084B688006E
:101BE0007490260094B6880084002C00A4B6880067
:101BF00094702700B4B68800A4002800C4B68800FA
:101C0000B4D02500D4B68800C4002000E4B6880013
:101C1000D4502100F4B68800E400240004B7880002
:101C2000F420260014B788000401200024B788009F
:101C30001401220034B788002481290044B78800A9
:101C40003401220054B7880044C1290064B78800D9
:101C500054A1200074B788006421200084B7880054
:101C60007421200094B7880084012200A4B7880062
:101C700094412000B4B78800A4412100C4B7880073
:101C8000B4312700D4B78800C4F12F00E4B788002E
:101C9000D4812700F4B78800E4612B0004B88800E1
:101CA000F441290014B8880004F2200024B8880008
:101CB0001402220034B888002422230044B888008B
:101CC0003462210054B888004442250064B888007A
:101CD0005492200074B888006402220084B88800FE
:101CE00074022D0094B8880084F22B00A4B88800F8
:101CF00094222000B4B88800A4022800C4B8880048
:101D0000B4022000D4B88800C4022000E4B88800DF
:101D1000D4822E00F4B88800E4022E0004B98800B2
:101D20002237EF001420250024B988002400200069
:101D300034B9880034802A0044B9880044002C005B
:101D400054B988005420270064B988006400240036
:101D500074B988007490260084B9880084002C002F
:101D600094B9880094702700A4B98800A4002800C2
:101D7000B4B98800B4D02500C4B98800C4002000DC
:101D8000D4B98800D4502100E4B98800E4002400CC
:101D9000F4B98800F420260004BA88000401200069
:101DA00014BA88001401220024BA88002481290072
:101DB00034BA88003401220044BA880044C12900A2
:101DC00054BA880054A1200064BA8800642120001D
:101DD00074BA88007421200084BA8800840122002B
:101DE00094BA880094412000A4BA8800A44121003C
:101DF000B4BA8800B4312700C4BA8800C4F12F00F7
:101E0000D4BA8800D4812700E4BA8800E4612B00AA
:101E1000F4BA8800F441290004BB880004F22000D1
:101E200014BB88001402220024BB88002422230053
:101E300034BB88003462210044BB88004442250042
:101E400054BB88005492200064BB880064022200C6
:101E500074BB880074022D0084BB880084F22B00C0
:101E600094BB880094222000A4BB8800A402280010
:101E7000B4BB8800B4022000C4BB8800C4022000A8
:101E8000D4BB8800D4822E00E4BB8800E4022E007C
:101E9000F4BB88008037EF001490260014BC880043
:101EA0002400280024BC880034002B0034BC8800A7
:101EB00044002C0044BC88005420270054BC8800F7
:101EC0006400240064BC88007490260074BC880000
:101ED00084002C0084BC88009470270094BC880087
:101EE000A4002800A4BC8800B4D02500B4BC88009D
:101EF000C4002000C4BC8800D4502100D4BC880099
:101F0000E4002400E4BC8800F4202600F4BC88002F
:101F10000401200004BD88001401220014BD8800C3
:101F20002481290024BD88003401220034BD8800AA
:101F300044C1290044BD880054A1200054BD88003C
:101F40006421200064BD88007421200074BD8800D5
:101F50008401220084BD88009441200094BD880043
:101F6000A4412100A4BD8800B4312700B4BD88007D
:101F7000C4F12F00C4BD8800D4812700D4BD8800DF
:101F8000E4612B00E4BD8800F4412900F4BD880021
:101F900004F2200004BE88001402220014BE88004F
:101FA0002422230024BE88003462210034BE88002D
:101FB0004442250044BE88005492200054BE88004C
:101FC0006402220064BE880074022D0074BE880082
